:020000040800F2
:10000000F0FF0120D5760408011F030835D101084F
:10001000497704084977040849770408000000007C
:100020000000000000000000000000000D1F030899
:10003000091F030800000000051F0308F99E0108BE
:100040004977040849770408497704084977040880
:100050004977040849770408A9DE0108D5DF0108BB
:1000600099DF01085DDF010821DF0108F5D70008ED
:10007000E5D70008D5D70008C5D70008B1D70008D4
:100080009DD7000889D700084977040800000000C0
:10009000000000000000000000000000E5DE010894
:1000A000418901082D8D010849770408ED8D01086B
:1000B0006D8C0108AD8B0108E18A010879DF000829
:1000C00081DF00086DDF000875DF0008497704084C
:1000D00049770408D59F0108399F010800000000F6
:1000E0006DDE010849770408C162030800000000C2
:1000F00000000000000000000000000075D70008AC
:100100000000000049770408118A010849770408B3
:1001100000000000000000000000000000000000DF
:1001200061D700084DD7000839D7000825D7000847
:1001300011D70008000000000000000000000000CF
:10014000000000000000000000000000812D0308F6
:10015000FDD60008E9D60008D5D60008497704087E
:1001600061DF000869DF00080000000000000000F7
:10017000000000000000000000000000000000007F
:1001800000000000497704080000000000000000A3
:080190004977040849770408CF
:080198006C720400010000007C
:1001A00010020100882B0020842B0020000000009A
:1001B000F006000818020200D0360020B8370020F0
:1001C000000000000000000017020B00C5360020F0
:1001D000BC37002000000000258400080702020050
:1001E00074370020C837002000000000F206000825
:1001F00002000C004C370020CC370020000000002B
:100200000000000006020C0040370020D837002014
:10021000000000007591000808120900BC3600209B
:10022000E43700200000000069840008F7010600A0
:10023000B6360020F037002000000000F406000869
:100240000A020A00B8310020F83700200000000040
:10025000FA06000803000100B82C00200438002032
:1002600000000000000000001A023C0004390020D9
:10027000043D002000000000E59000082700040075
:1002800000390020403D0020000000000407000865
:100290000312330000440020D44B00200000000073
:1002A0000807000825009600884A00201E4B002001
:1002B0000000000000000000F6210C00544800205F
:1002C000044A0020000000003C07000815007000F0
:1002D0002449002094490020000000000000000094
:1002E0002A00600064480020C4480020000000008C
:1002F0005DF503082C001000B44B0020C44B002017
:1003000000000000510F02082B0024002B4C00209D
:10031000074C002000000000210F0208291078007F
:1003200064470020104A0020000000000000000088
:10033000140003001C46002060480020000000005C
:10034000480700081010020098440020944C002038
:10035000000000004C07000828101000884400200E
:10036000984C0020000000008DF3010823001000CD
:1003700034410020A84C002000000000A5F3010833
:10038000F82106007E420020B84C0020000000004A
:100390004E0700080E502001BC5D0020386500208B
:1003A0000000000085F5030813000400BC62002073
:1003B00058660020000000005407000801010400F6
:1003C000365D00205C660020000000000000000098
:1003D000000104002E5D0020606600200000000087
:1003E0005807000802010300295D00206466002010
:1003F0000000000069E9000809020100E064002033
:1004000068660020000000005C0700080C106C000B
:10041000065F00206C6600200000000041E9000833
:10042000010205003E5D0020D866002000000000AB
:10043000E58D02080002050050620020E066002001
:1004400000000000000000001B0208002C620020D9
:10045000E866002000000000198400080120080060
:10046000A0630020F0660020000000005E07000886
:100470001900050050640020F8660020000000000C
:100480006607000837001E0028640020006700206F
:10049000000000006C0700081E0005000C60002032
:1004A00020670020000000008A0700081B00F400FD
:1004B000C84C00202867002000000000799E020838
:1004C0000E020200386300201C68002000000000BB
:1004D000900700082F0011001865002020680020F8
:1004E000000000009207000805100600347E00207E
:1004F0002483002000000000A4070008F5317000EC
:10050000947D00202C830020000000001998020830
:1005100026000E00AC8300209C8300200000000019
:10052000391203080B2010009C7B0020E083002080
:1005300000000000AA0700081F201C00EC72002029
:10054000F083002000000000BA0700080502040044
:100550005C7D00200C84002000000000D60700080D
:1005600003010A00547B00201084002000000000DA
:10057000DA07000813020300607100201C840020C9
:1005800000000000E407000816000800A084002016
:10059000A884002000000000E80700080400800094
:1005A000F8B90020B0BA00200000000000000000F0
:1005B0000D002C006CB8002030BB002000000000B3
:1005C0008D630308F9010400BCAF00205CBB002070
:1005D000000000001D770108FD01240098AF0020F5
:1005E00060BB002000000000A576010818202C0048
:1005F00068AF002084BB0020000000008D9100083F
:1006000006101800B4A20020B0BB002000000000BB
:10061000E1F50308FB010100ECA10020C8BB0020AC
:1006200000000000F1910008FC010900B8A00020C2
:10063000CCBB002000000000019200080A4020000E
:1006400080A00020D8BB002000000000F0070008B8
:100650003400100028990020F8BB002000000000A2
:10066000B5F50308110208000099002008BC00201D
:10067000000000001008000812120400F898002082
:1006800010BC0020000000001808000812200E0016
:10069000E898002014BC0020000000001C0800089E
:1006A000020203000485002024BC0020000000009A
:1006B000000000000C020300C084002028BC0020C1
:1006C0000000000089840008FE0109003087002036
:1006D0002CBC002000000000998400081A000E00C5
:1006E0001CC00020C4C10020000000002A0800082F
:1006F0000000013C22010000000000004A01B4009B
:10070000D6010000200300000000000000000000EF
:1007100000000000000000000000000000000000D9
:1007200000000000000000000000000000000000C9
:1007300000000000000000000000010000000000B8
:100740000100000002020000030000000005040197
:10075000F401190048040430900100000000E8038F
:100760006400040A0001000028010000200032009B
:10077000C800D0079600140032002800B0044006DC
:100780000005500014000F000801000001000000E7
:100790000000000000000000000000000000000059
:1007A000000000002000030100002B21231E640133
:1007B0000100000001000A01290000000000000102
:1007C000000000050000010203000000000000001E
:1007D00000000000000000000000040101006C1691
:1007E0000000000000000000C409000019012828D2
:1007F000003001000000000064002C010000000037
:10080000000000000000020000019E077D0046324B
:100810000000000001010101FFFFFFFF00000001D7
:10082000000005465344343100007E05EA05B40556
:080830003200E803D0070000CC
:100838000100000080010000080000000400000022
:100848000000000000000000010203040607080978
:10085800010000000000803F0000000000000000D0
:1008680000000000FF00000000000000A837002082
:100878000800000000000000983700200800000071
:1008880018960408050804000000000084BF040846
:100898004CC0040870BF04080000000000000000FD
:1008A8004496040805080A000000000084BF0408F4
:1008B8004CC0040850BE04080000000000000000FE
:1008C800685E0C00010102FFFF000000D601010074
:1008D800000101010001FFFFFFFFFFFF0100000011
:1008E80000000100E001010101000000BD910208C3
:1008F80000000000300200207C18050800000000FD
:10090800000000000000000000000000D3200508DF
:100918000000000000000000C602002004000000E3
:10092800281805080D00000009BD02089C1C0020BD
:10093800000000008C1105080D00000031BD020800
:10094800901C002000000000F412050808000000B8
:1009580000000000841C002004000000F8110508B5
:100968000D00000071920208781C002000000000B1
:10097800A81205080300000005C002086C1C00202E
:10098800000000008C1805080300000005C00208DC
:10099800601C002000000000280E0508010000006F
:1009A800000000000000000000000000000000003F
:1009B8000E00000000000000000000000000000021
:1009C8007C1805080000000000000000000000007E
:1009D80000000000D320050800000000000000000F
:1009E800C602002004000000D41705080300000018
:1009F80009990208541C002008000000F811050895
:100A08000D00000071920208781C00200000000010
:100A1800A81205080300000005C002086C1C00208D
:100A2800000000008C1805080300000005C002083B
:100A3800601C002000000000280E050801000000CE
:100A4800000000000000000000000000000000009E
:100A58000E00000000000000000000000000000080
:100A680094180508000000000000000000000000C5
:100A780000000000D320050800000000000000006E
:100A8800C602002004000000DC170508030000006F
:100A980005C00208A81C002000000000280E050858
:100AA800010000000000000000000000000000003D
:100AB800000000000E000000000000000000000020
:100AC8000000000020700020702D7200FFFFFFFF63
:100AD800010000000000803F080000000000000046
:100AE8000000000010180020FA00000001000000BB
:100AF80001000000FFFF2D202D2D202D2D2D2D2054
:100B08002D2D2D0000000000000000000000000056
:100B180000000000000000000000803F0000803F4F
:100B2800FFFFFFFFFC0D0508040E0508200E050851
:100B380000000000000000000000000000000000AD
:100B4800CE0B050804000000D1BA0208000000001E
:100B580000000000280E0508010000000000000049
:100B68000000000000000000000000000E0000006F
:100B780000000000000000000000000098BA0020FB
:100B88000100C4090000000096BA00200100C40951
:100B98000000000094BA00200100C4090000000011
:100BA80092BA00200100C409000000008EBA00209B
:100BB8000100C4090000000090BA00200100C40927
:100BC800000000008CBA00200100C40900000000E9
:100BD8008ABA00200100C40900000000505D00200E
:100BE8000100C800010000004E5D00203200307591
:100BF800320000004C5D0020055A0500495D0020C8
:100C080000FF01004B5D002001000000F4020020FD
:100C1800475D00200200000078C00408485D0020FD
:100C280000FF01004A5D002001000000F4020020DE
:100C3800465D00200200000078C004083C5D0020EA
:100C480080C1803E050000003A5D002080C1803EE2
:100C580005000000345D002080C1803E05000000D2
:100C6800325D002080C1803E050000002C5D002020
:100C780000FF0100285D00200A320100275D0020E6
:100C88000400000030BE0408265D002002000000B9
:100C980044BE04080000000000000000FC02002020
:100CA8000C7D00209CFF2C0100000000B6000020F5
:100CB8000A00000050BE04081C5D0020E0150C1757
:100CC80000000000B8000020080000004CC0040824
:100CD800B70000200500000084BF04081E5D002046
:100CE8000200000068BE04088C5F00200100FF7F3E
:100CF800010000008B5F00200200000074BE0408A1
:100D0800AF5D00200300000084BE0408AE5D002033
:100D18000300000084BE0408E65E00200000F40121
:100D280001000000E45E00200000F4010100000062
:100D3800E25E00200000F40101000000E05E0020F7
:100D48000000F40101000000DE5E00200000803E8B
:100D580001000000DC5E00200000803E0100000071
:100D6800025F0020E803D0070A000000005F0020AF
:100D7800006401000A000000F55E00200064010024
:100D8800F45E002000640100FC5E002000640100A5
:100D98000A000000FB5E0020006401000A00000059
:100DA800FA5E0020006401000A000000FF5E0020D7
:100DB800006401000A000000FE5E002000640100DB
:100DC8000A000000FD5E0020006401000A00000027
:100DD800F95E002000FF01000A000000F85E002014
:100DE80000FF01000A000000F75E002000FF01007C
:100DF8000A000000B85D00200000F40101000000B6
:100E0800B65D00200000F40101000000B45D002080
:100E18000000F40101000000B25D00200000F401B0
:100E280001000000B05D00200000F4010100000096
:100E3800F25E002000640100F05E00201400E80368
:100E480001000000EE5E0020E80330750A00000093
:100E5800EC5E002000C80100EB5E002000C8010025
:100E6800EA5E002000C80100E95E0020006401007D
:100E78000A000000805F00200000D0070100000089
:100E88007B5F002000C801007A5F002000C80100D5
:100E9800795F002000C801007E5F00200000D007B5
:100EA80001000000785F002000C80100775F002083
:100EB80000C80100765F002000C801007C5F0020A8
:100EC8000000D00701000000755F002000C8010085
:100ED800745F002000C80100735F002000C8010093
:100EE800500E05080000000000000000000000008F
:100EF8000000000064E2040809000000000000008F
:100F0800A0030020040000006CE2040809000000AF
:100F1800000000009403002004000000AC15050840
:100F28000900000000000000880300200400000001
:100F3800CB0C050809000000000000007C0300201D
:100F480004000000600E0508090000000000000011
:100F58007003002004000000680E05080900000066
:100F6800000000006403002004000000700E050863
:100F780009000000000000005803002004000000E1
:100F8800780E050809000000000000004C0300204E
:100F980004000000280E0508010000000000000001
:100FA8000000000000000000000000000E0000002B
:100FB8000000000000000000000000007810050894
:100FC8000000000000000000000000000000000019
:100FD800E4FF04080700000000000000C40300202C
:100FE800000000008810050808000000000000004C
:100FF800B803002000000000941005080800000055
:1010080000000000AC03002000000000280E0508C6
:1010180001000000000000000000000000000000C7
:10102800000000000E0000000000000000000000AA
:10103800000000009C1005080000000000000000EF
:101048000000000000000000AC1005080D000000C2
:10105800000000000004002000000000B410050893
:101068000D00000000000000F40300200000000054
:10107800BC1005080700000000000000EC03002079
:1010880000000000C41005080D000000000000006A
:10109800E003002000000000CC1005080D0000004F
:1010A80000000000D403002000000000D410050850
:1010B8000700000000000000CC0300200000000032
:1010C800280E0508010000000000000000000000D4
:1010D80000000000000000000E00000000000000FA
:1010E8000000000000000000DC10050800000000FF
:1010F800000000000000000000000000E4FF0408F9
:101108000C00000000000000525D002000000000FC
:10111800F01005080C00000000000000545D0020DD
:1011280000000000001105080C000000000000008D
:101138008A5D002000000000101105080C00000066
:10114800000000007E5D002000000000241105085A
:101158000C00000000000000565D002000000000A8
:10116800301105080C00000000000000585D002048
:1011780000000000381105080C0000000000000005
:101188005A5D0020000000004C1105080C0000000A
:10119800000000005C5D00200000000054110508FC
:1011A8000C000000000000005E5D00200000000050
:1011B8005C1105080C000000000000009C5D002088
:1011C80000000000741105080C0000000000000079
:1011D800605D002000000000801105080C00000080
:1011E80000000000625D00200000000074E20408B6
:1011F8000C00000000000000645D002000000000FA
:10120800881105080C00000000000000665D002041
:1012180000000000941105080C0000000000000008
:10122800685D002000000000A01105080C00000007
:10123800000000006A5D002000000000AC110508F5
:101248000C000000000000006C5D002000000000A1
:10125800B81105080C000000000000006E5D0020B9
:1012680000000000C41105080C0000000000000088
:10127800825D002000000000CC1105080C00000071
:1012880000000000805D002000000000D411050867
:101298000C000000000000008E5D0020000000002F
:1012A800E01105080C00000000000000905D00201F
:1012B80000000000EC1105080C0000000000000010
:1012C800965D0020000000001C0F05080C000000BF
:1012D80000000000705D002000000000F811050803
:1012E8000C00000000000000785D002000000000F5
:1012F800001205080C00000000000000725D0020CC
:10130800000000000C1205080C000000000000009E
:10131800745D002000000000181205080C00000091
:1013280000000000765D0020000000002012050883
:101338000C000000000000007A5D002000000000A2
:10134800040005080C00000000000000845D002077
:10135800000000002C1205080C000000000000002E
:101368007C5D0020000000006A0D05080C000000EC
:10137800000000008C5D0020000000003812050805
:101388000C00000000000000865D00200000000046
:10139800401205080C00000000000000885D0020D5
:1013A80000000000481205080C00000000000000C2
:1013B800925D002000000000501205080C0000009B
:1013C80000000000945D002000000000581205088D
:1013D8000C00000000000000A65D002000000000D6
:1013E800280E0508010000000000000000000000B1
:1013F80000000000000000000E00000000000000D7
:101408000000000000000000601205080000000055
:101418000000000000000000000000006C12050839
:101428000D0000000000000058040020000000002B
:10143800741205080D000000000000004C04002094
:10144800000000007C1205080700000000000000F2
:10145800440400200000000088120508070000006E
:10146800000000003C040020000000009412050861
:101478000900000000000000300400200000000007
:10148800A012050809000000000000002404002044
:1014980000000000AC120508090000000000000070
:1014A8001804002000000000BC1205080900000014
:1014B800000000000C04002000000000280E0508B1
:1014C8000100000000000000000000000000000013
:1014D800000000000E0000000000000000000000F6
:1014E80000000000D0120508000000000000000005
:1014F8000000000000000000E012050805000000E0
:1015080000000000AD5D002000000000280E050866
:1015180001000000000000000000000000000000C2
:10152800000000000E0000000000000000000000A5
:1015380000000000E812050800000000000000009C
:101548000000000000000000D32005080000000093
:1015580000000000241E002004000000C70C05083D
:101568000D00000035BB0208AC040020000000009C
:10157800281805080D00000075910208A004002035
:10158800000000008C1105080D00000059910208A8
:101598009404002000000000F41205080800000070
:1015A800000000008804002004000000F81105086D
:1015B8000D000000A19002087C040020000000003B
:1015C800FC1205080900000000000000700400205B
:1015D80004000000A81205080300000005C0020866
:1015E8006404002000000000280E05080100000027
:1015F80000000000000000000000000000000000E3
:101608000E000000000000000000000000000000C4
:10161800041305080000000000000000000000009E
:1016280000000000141305080D0000000000000071
:10163800C4040020000000001C1305080A00000074
:1016480000000000BA5F0020000000002813050811
:101658000A00000000000000C25F00200000000037
:10166800301305080A00000000000000CA5F0020CF
:101678000000000038130508080000000000000002
:10168800B804002000000000280E05080100000032
:101698000000000000000000000000000000000042
:1016A8000E00000000000000000000000000000024
:1016B80040130508000000000000000000000000C2
:1016C80000000000541305080D0000000000000091
:1016D800DC0400200000000064130508040000007A
:1016E800ADBD020800000000000000006C130508F2
:1016F8000D00000000000000D004002000000000E1
:10170800801305080400000089BD020800000000DD
:1017180000000000280E050801000000000000007D
:101728000000000000000000000000000E000000A3
:1017380000000000000000000000000088130508F9
:101748000000000000000000000000000000000091
:101758009C13050808000000000000002405002074
:1017680000000000A81305080800000000000000A1
:101778001805002000000000B41305080800000048
:10178800000000000C05002000000000C013050840
:101798000800000000000000000500200000000014
:1017A800CC1305080800000000000000F404002025
:1017B80000000000D8130508080000000000000021
:1017C800E804002000000000280E050801000000C1
:1017D8000000000000000000000000000000000001
:1017E8000E000000000000000000000000000000E3
:1017F800E413050800000000000000009702002024
:1018080000000000F01305080B00000000000000B5
:10181800B805002000000000FC1305080B000000BC
:1018280000000000AC0500200000000008140508B6
:101838000B00000000000000A005002000000000D0
:10184800141405080B000000000000009405002097
:1018580000000000201405080B0000000000000034
:1018680088050020000000002C1405080B0000006B
:10187800000000007C050020000000003814050866
:101888000B000000000000007005002000000000B0
:10189800441405080B000000000000006405002047
:1018A80000000000501405080B00000000000000B4
:1018B80058050020000000005C140508070000001F
:1018C8000000000050050020000000006414050816
:1018D800070000000000000048050020000000008C
:1018E800701405080B000000000000003C050020F3
:1018F800000000007C14050808000000000000003B
:101908003005002000000000280E05080100000036
:1019180000000000000000000000000000000000BF
:101928000E000000000000000000000000000000A1
:1019380088140508000000000000000000000000F6
:10194800000000009C1405080800000000000000CA
:10195800F405002000000000A81405080800000095
:1019680000000000E805002000000000B41405088D
:101978000800000000000000DC0500200000000056
:10198800C01405080800000000000000D005002071
:1019980000000000CC14050808000000000000004A
:1019A800C405002000000000280E05080100000002
:1019B800000000000000000000000000000000001F
:1019C8000E00000000000000000000000000000001
:1019D800D414050800000000000000009402002054
:1019E80000000000E41405080B00000000000000DF
:1019F8003806002000000000F01405080700000069
:101A0800000000003006002000000000FC1405085B
:101A18000700000000000000280600200000000069
:101A28000815050807000000000000002006002037
:101A38000000000014150508080000000000000060
:101A480014060020000000001C150508080000000E
:101A5800000000000806002000000000241505080A
:101A68000700000000000000000600200000000041
:101A7800280E05080100000000000000000000001A
:101A880000000000000000000E0000000000000040
:101A980000000000000000003015050800000000EC
:101AA8000000000094020020000000003C1505081A
:101AB8000700000000000000A80600200000000049
:101AC800441505080700000000000000A0060020DB
:101AD800000000004C150508070000000000000089
:101AE80098060020000000005415050808000000B2
:101AF800000000008C060020000000005C150508AE
:101B0800070000000000000084060020000000001C
:101B18006415050807000000000000007C0600208E
:101B2800000000006C150508070000000000000018
:101B38007406002000000000741505080800000065
:101B48000000000068060020000000007C15050861
:101B580007000000000000006006002000000000F0
:101B68008415050807000000000000005806002042
:101B7800000000008C1505080700000000000000A8
:101B88005006002000000000941505080800000019
:101B9800000000004406002000000000280E050890
:101BA800010000000000000000000000000000002C
:101BB800000000000E00000000000000000000000F
:101BC8000000000000000000E5940208B0060020B4
:101BD800AB5D00202B00000094BE0408AA5D002025
:101BE80000C80100A85D0020E803D007010000003C
:101BF80046554C4C5350454544463431310000005D
:101C0800455D002000030100445D00200003010041
:101C18002D940208059402088C070020C19302083D
:101C280075930208040800206D9402085594020870
:101C3800B8080020E192020895920208D80B00200B
:101C4800FB94020859BD0208B40C0020E190020878
:101C580000000000040D0020499902086997020855
:101C6800E00D00202195020800000000800E0020F1
:101C7800C9950208959502080C0F00205196020894
:101C88009D960208C00F0020F35E002001060100A7
:101C9800659502083595020800110020FD95020897
:101CA800D1BD0208A0110020CD96020821BE02086D
:101CB80068120020E85E0020010301009C15050859
:101CC800000000000000000000000000000000000C
:101CD800A81505080800000000000000B413002043
:101CE80000000000B0150508070000000000000013
:101CF800AC13002000000000C01505080D0000000E
:101D080000000000A013002000000000CC1505080A
:101D18000300000005C00208941300200000000022
:101D2800280E050801000000000000000000000067
:101D380000000000000000000E000000000000008D
:101D48000000000000000000D41505080000000095
:101D5800000000000000000000000000E415050875
:101D68000A00000000000000EC1505080000000053
:101D7800F41505080A00000000000000BFCE0408A2
:101D880000000000FC1505080A0000000000000023
:101D9800825F002000000000041605080A00000009
:101DA80000000000C013002000000000280E0508F5
:101DB800010000000000000000000000000000001A
:101DC800000000000E0000000000000000000000FD
:101DD800000000000C1605080000000000000000CC
:101DE80000000000000000001816050803000000AD
:101DF80005C00208F813002000000000241605089A
:101E08000300000005C00208EC13002000000000D9
:101E18002C1605080300000005C00208E013002086
:101E2800000000003416050805000000000000004E
:101E3800435D0020000000003C1605080700000074
:101E480000000000D8130020000000004816050814
:101E58000700000000000000D01300200000000070
:101E6800280E050801000000000000000000000026
:101E780000000000000000000E000000000000004C
:101E880000000000000000005416050800000000D3
:101E980000000000000000000000000068160508AF
:101EA8000300000005C002082814002000000000FC
:101EB800741605080300000005C00208BC000020D5
:101EC800000000007C1605080300000005C0020899
:101ED8001C14002000000000841605080300000000
:101EE80005C002081014002000000000F8110508C1
:101EF8000300000005C002080414002000000000D0
:101F0800280E050801000000000000000000000085
:101F180000000000000000000E00000000000000AB
:101F280000000000000000009016050800000000F6
:101F3800000000000000000000000000A0160508D6
:101F4800070000007DBE0208841400200000000085
:101F58001C1205080300000005C0020878140020C0
:101F680000000000AC1605080300000005C00208C8
:101F78006C14002000000000B416050803000000DF
:101F880005C002086014002000000000BC16050807
:101F98000700000061BE020858140020000000007D
:101FA800C01A05080300000005C002084C140020F0
:101FB80000000000C81605080300000005C002085C
:101FC8004014002000000000D4160508030000009B
:101FD80005C002083414002000000000280E05087F
:101FE80001000000000000000000000000000000E8
:101FF800000000000E0000000000000000000000CB
:1020080000000000B5940208859402088C14002092
:102018004997020800000000181500205193020893
:102028002D930208A4150020000000000000000005
:10203800581600202197020899BE0208F8160020B9
:10204800E016050800000000000000000000000085
:1020580000000000EC1605080300000005C0020897
:102068000418002000000000F41605080300000012
:1020780005C00208F817002000000000FC00050851
:102088000300000005C00208EC1700200000000053
:10209800001705080300000005C00208E01700202B
:1020A800000000000C1705080300000005C0020826
:1020B800D4170020000000001417050802000000D3
:1020C800B5BE020800000000000000001C1705084B
:1020D80002000000B5BE0208010000000000000078
:1020E8002817050802000000B5BE0208020000001B
:1020F80000000000000000000E00000000000000CA
:102108000000000000000000225D002088136F1707
:1021180001000000245D002088136F1700000000F4
:10212800341705080000000000000000000000004F
:102138000000000044170508080000000000000027
:10214800E4180020040000005017050808000000EB
:1021580000000000D818002000000000A8120508A0
:10216800040000005DBB0208000000000000000041
:10217800280E050801000000000000000000000013
:1021880000000000000000000E0000000000000039
:102198000000000000000000205D002088136F1779
:1021A80001000000487D002088136F170000000020
:1021B8002592020800000000F0180020B9620020F3
:1021C8000100000044BF04084A7D0020010000000F
:1021D80050BF0408407D00200200000058BF0408DA
:1021E8003E73002000000000000000003C73002047
:1021F80000000000000000003A730020000000000A
:1022080000000000387300200000000000000000FB
:102218003673002000000000000000003473002026
:1022280000000000000000005C1E0020000000000C
:10223800000000001F5D00200200000064BF0408C9
:102248008C170508000000000000000000000000D6
:102258000000000044170508080000000000000006
:102268007419002004000000501705080800000039
:10227800000000006819002000000000A8120508EE
:1022880004000000F59102080000000000000000B2
:10229800280E0508010000000000000000000000F2
:1022A80000000000000000000E0000000000000018
:1022B80000000000000000009C1705080000000056
:1022C800000000000000000000000000AC17050836
:1022D8000D000000ADBC0208A41900200400000095
:1022E800B81705080D0000004D9202089819002043
:1022F80004000000C41705080D00000071BC0208A6
:102308008C19002000000000D01705080300000009
:10231800299902088019002008000000DC17050828
:102328000300000005C00208A81C002000000000EF
:10233800280E050801000000000000000000000051
:1023480000000000000000000E0000000000000077
:102358000000000000000000200E0508000000003A
:10236800000000000000000000000000CE0B05087F
:102378000400000075BB0208000000000000000017
:10238800280E050801000000000000000000000001
:1023980000000000000000000E0000000000000027
:1023A80000000000000000003018050800000000D0
:1023B80000000000000000000000000068E60408BB
:1023C8000D00000000000000041A002004000000B6
:1023D800401805080800000000000000F819002057
:1023E800040000004C180508080000000000000068
:1023F800EC1900200400000054180508080000002B
:1024080000000000E0190020040000005C18050826
:102418000800000000000000D4190020040000009B
:10242800641805080800000000000000C819002012
:10243800040000006C1805080800000000000000F7
:10244800BC190020040000007418050808000000EA
:1024580000000000B019002004000000280E050844
:102468000100000000000000000000000000000063
:10247800000000000E000000000000000000000046
:10248800000000000D92020800000000101A002051
:102498000000000000000000881A00200000000072
:1024A80000000000281B0020467D002004000000DA
:1024B80070BF0408447D0020E0150C1700000000E0
:1024C800437D0020080000004CC00408427D002025
:1024D8000500000084BF04080000000000000000A0
:1024E800781B00200403090412010002EF020140D6
:1024F80083045632000201020301000012010002A7
:102508000202004083044057000201020301000058
:1025180009026400030100C032090400000103003D
:102528000000092111010001222600070583030884
:10253800000A080B0102020201000904010001025D
:1025480002010005240010010524010002042402F0
:10255800020524060102070582030800FF09040298
:1025680000020A000000070501024000000705817B
:102578000240000009024300020100C032090400C1
:1025880000010202010005240010010524010001D8
:10259800042402020524060001070582030800FF3F
:1025A80009040100020A00000007050102400000BA
:1025B8000705810240000000FF00000000FFFF0047
:1025C80000000000AA5505010000010005010905E9
:1025D800A101A10005010930093109320933093582
:1025E8000934094009381581257F75089508810245
:1025F800C0C0000009022200010100E03209040005
:10260800000103010200092111010001222600072F
:1026180005830308000A000000000000010203040B
:102628000102030406070809492203084D2103088B
:102638008D240308CD060308110A0308DD060308E4
:10264800F9060308A506030895060308000000001C
:10265800000000002D202D2D202D2D2D2D202D2D7D
:102668002D2D000000000000000000000000000008
:10267800000000AA550B010000AA5507010000AA96
:10268800550902000000000001000000C012AA5510
:1026980003009F00FF1FFF1F01000000BC830020F4
:1026A80000000000C42300200400000030000508DA
:1026B8006C1B0508000000000D630308A0860100DC
:1026C80004000000000000000000000000000000FE
:1026D80000000000000000000000000000000000F2
:1026E800300005088C1C0508000000004175010831
:1026F800E8030000040000000000000000000000E3
:1027080000000000000000000000000000000000C1
:10271800000000001C12050880E204080000000008
:10272800D1F300087D000000060000000000000052
:102738000000000000000000000000000000000091
:10274800000000000000000088FF040800000000EE
:102758000000000031E70108E80300000300000062
:102768000000000000000000000000000000000061
:10277800000000000000000000000000941C050894
:102788000000000000000000A9F80308102700005E
:10279800030000000000000000000000000000002E
:1027A8000000000000000000000000000000000021
:1027B800B818050800000000550B020875D101087B
:1027C8005F76000005000000000000000000000027
:1027D80000000000000000000000000000000000F1
:1027E80000000000F00105080000000000000000E3
:1027F800F9EB0108102700000100000000000000AC
:1028080000000000000000000000000000000000C0
:102818000000000000000000A01C050800000000E7
:102828000000000045750108E803000005000000ED
:102838000000000000000000000000000000000090
:10284800000000000000000000000000AC1C0508AB
:10285800000000000000000085660108204E00000E
:10286800030000000000000000000000000000005D
:102878000000000000000000000000000000000050
:10288800BC1C05080000000000000000716401087D
:10289800204E0000030000000000000000000000BF
:1028A8000000000000000000000000000000000020
:1028B80000000000CC1C050800000000000000001B
:1028C800717A0108400D03000300000000000000B9
:1028D80000000000000000000000000000000000F0
:1028E8000000000000000000F400050800000000DF
:1028F800000000002D6F03081027000001000000F1
:1029080000000000000000000000000000000000BF
:10291800000000000000000000000000A0FF040804
:10292800000000000000000055D502081027000034
:10293800030000000000000000000000000000008C
:10294800000000000000000000000000000000007F
:102958008CFF040800000000000000009D790108B9
:1029680050C300000100000000000000000000004B
:10297800000000000000000000000000000000004F
:10298800000000001C0F0508000000000000000007
:102998002D770108A8610000010000000000000078
:1029A800000000000000000000000000000000001F
:1029B8000000000000000000DC1C0508000000000A
:1029C8000000000009F10208A086010001000000D3
:1029D80000000000000000000000000000000000EF
:1029E800000000000000000000000000F8010508D9
:1029F800000000000000000025A10108A00F000051
:102A080001000000000000000000000000000000BD
:102A180000000000000000000000000000000000AE
:102A2800E81C05080000000000000000619A020888
:102A38001027000001000000000000000000000056
:102A4800000000000000000000000000000000007E
:102A580000000000FC000508000000000000000065
:102A6800E94203081A4100000100000000000000CC
:102A7800000000000000000000000000000000004E
:102A880000000000000000005802050800000000D7
:102A980000000000A90E0308102700000100000034
:102AA800000000000000000000000000000000001E
:102AB800000000000000000000000000801B050866
:102AC800000000000000000079C102081A4100005F
:102AD80001000000000000000000000000000000ED
:102AE80000000000000000000000000000000000DE
:102AF800F41C05080000000000000000613E030807
:102B0800400D03000000000000000000000000006D
:102B180000000000000000000000000000000000AD
:102B280000000000FC1C0508000000000000000078
:102B380049630308400D0300000000000000000086
:102B4800000000000000000000000000000000007D
:102B58000000000000000000041D0508000000003F
:102B680000000000CDE2020850C30000030000008E
:102B7800000000000000000000000000000000004D
:102B8800000000000000000000000000101D050803
:102B98000000000000000000E563010840420F004B
:102BA800000000000000000000000000000000001D
:102BB800000000000000000000000000000000000D
:102BC8001C1D0508000000000000000065640308E3
:102BD80050C30000000000000000000000000000DA
:102BE80000000000000000000000000000000000DD
:102BF80000000000000200051002700BF10B030832
:102C080095090308692403080000000091060308D9
:102C1800392103085D0B0308B120030800000000F8
:102C2800000000004D060308610B0308550903085E
:102C3800A92303080000000065060308B52003085F
:102C4800310B0308112003080000000000000000F9
:102C58005906030808000000B1050308AD0503087C
:102C6800A90503089D05030899050308A505030898
:102C7800A10503082506030819060308F10503083A
:102C880005060308DD050308C9050308B50503089B
:102C980001000000006002401060024000000000D7
:102CA80000000000000B0000000000000000000011
:102CB800000000000060024028600240010000009F
:102CC80000000000060C00000000000000000000EA
:102CD8000000000000600240406002400200000066
:102CE80000000000100D00000000000000000000BF
:102CF800000000000060024058600240030000002D
:102D080000000000160E0000000000000000000097
:102D180000000000006002407060024004000000F3
:102D280000000000200F000000000000000000006C
:102D380000000000006002408860024005000000BA
:102D48000000000026100000000000000000000045
:102D58000000000000600240A06002400600000081
:102D6800000000003011000000000000000000001A
:102D78000000000000600240B86002400700000048
:102D880000000000362F00000000000000000000D6
:102D980000000000006402401064024000000000CF
:102DA80000000000003800000000000000000000E3
:102DB8000000000000640240286402400100000096
:102DC80000000000063900000000000000000000BC
:102DD800000000000064024040640240020000005D
:102DE80000000000103A0000000000000000000091
:102DF8000000000000640240586402400300000024
:102E080000000000163B0000000000000000000069
:102E180000000000006402407064024004000000EA
:102E280000000000203C000000000000000000003E
:102E380000000000006402408864024005000000B1
:102E48000000000026440000000000000000000010
:102E58000000000000640240A06402400600000078
:102E680000000000304500000000000000000000E5
:102E78000000000000640240B8640240070000003F
:102E880000000000364600000000000000000000BE
:102E9800000000000000803F00000000000000006B
:102EA800000000000000803F00000000000000005B
:102EB800000000000000000000000000000000000A
:102EC80000000000000000000000000001000000F9
:102ED8000000803F0000000000000000000000002B
:102EE8000000803FB826002000000000000000001D
:102EF80000000000000000000000000000000000CA
:102F080000000000000000000000000000000000B9
:102F180000000000000000000000000000000000A9
:102F28000000000000000000000000000000000099
:102F38000000000000000000000000000000000089
:0C2F48000000000000000000010000007C
:1080000003685A1C02601970704700BF2DE9F047E1
:10801000089C2578002B804689460CBF4FF0200A2B
:108020004FF0300A661C25B3002A26DD334601E0F6
:10803000024698B113F8011B501E0029F8D1971E73
:1080400060B13D46013D51464046C8476B1C002B80
:10805000F8DC257827EAE770013045B1041B294692
:108060004046C847301916F8015B002DF7D1BDE82E
:10807000F087002A03DC2846F9E70020EEE7571EC8
:10808000DFE700BF2DE9F04714461D4606464FF4D2
:108090007A720023204629463FF050F94D4BDFF815
:1080A00048814D4A4D4F034488FB03101844D917AB
:1080B00082FB032CC1EB601088FB002887FB0327A1
:1080C0009C44474AC1EBEC2CC0EB001E82FB0C2900
:1080D000A3EB8E0E1F44434A86F806E0C1EB274708
:1080E0004FEAEC7E08EB000ACEEBA90E82FB07827A
:1080F0004FEAE0780EEB4E0EC8EB6A18ACEBCE0CF4
:10810000C8EB0818DFF8E4E086F804C0A0EB8800AC
:1081100070718EFB0303F817C0EBE21240F2B5500A
:1081200000FB1272C1EBE353B2F5896F4FEA83078C
:108130003CDA40F2DA239A4242DCB2F5B77FB4BFB0
:108140004FF0000E4FF0010E4FEA4E09DFF8A0800D
:1081500009EB0E0308EBC3031FFA8EFCD88A09EB68
:108160000E0108EBC10116310B2301E031F8020DBD
:10817000904218DD013BF9D1CE44012338F83E008E
:10818000B37007F5FA670132121ABC44F270A6F810
:1081900000C0204629464FF47A7200233FF0CEF803
:1081A0003281BDE8F0870133DBB2E9E74FF0030C21
:1081B000E64640F29650DFF838804FF00609CEE7E9
:1081C0004FF0020CDFF82880E64640F229404FF0DD
:1081D0000409C4E780BC92C7C5B3A29107452EC26B
:1081E000ABAAAA2A73B06D1689888888792D0311E5
:1081F0007890040830B403888278C478154DA3F5CC
:10820000FA6303F0030101EB4101013A02EB810241
:108210009B0835F812500279611E40F2B55404FBF8
:1082200003132B4403EB430302EBC303427984792A
:1082300009490089C3EB031302EB83032144C3EB19
:10824000031301EB83034FF47A720021C2FB030195
:1082500030BC70477890040880436D380028F0B433
:1082600003DA2D230B7040420131092804464FF0F8
:10827000010307DD03EB83035B00B0FBF3F2092A84
:10828000F8D883B10F48A0FB0326B4FBF3F2092A08
:1082900002F1570C02F1300709DD03FB1244F30829
:1082A00001F801CBEFD100230B70F0BC704703FB4A
:1082B0001244F30801F8017BE5D100230B70F0BCF8
:1082C000704700BFCDCCCCCC884270B44FF00104D5
:1082D00042D301FB04F4B0FBF4F58D42F9D2ECB1CA
:1082E00042BB092D04FB150005F1570605F13002CC
:1082F0000EDDB4FBF1F403F8016B7CB1B0FBF4F5D7
:10830000092D04FB150005F1570605F13002F0DCDC
:10831000B4FBF1F403F8012B002CEFD100221A700A
:1083200070BC704703F8016BB4FBF1F4002CF5D07E
:10833000B0FBF4F5092D04FB150005F1370605F136
:108340003002EFDCB4FBF1F403F8012B002CEFD189
:1083500000221A7070BC70470546002AEAD1C0E7B7
:1083600090ED057A90ED004AD0ED066AD0ED014A15
:10837000D0ED047A90ED035AD0ED025AA4EE007AC3
:10838000B0EE406AB0EE470AB0EE667AA4EE867AA6
:1083900067EEC07AA5EE407AE5EE867A80ED057A42
:1083A000C0ED067A704700BFD0ED057A90ED013A36
:1083B000D0ED003AD0ED064A90ED024A90ED077AF2
:1083C00090ED035A90ED086AD0ED045AC0ED067A9C
:1083D000F0EE406A27EE830AC0ED056AA3EEA60A16
:1083E00080ED087AA4EE240AA5EE470AA5EEC60A97
:1083F00080ED070A704700BFD0ED007A90ED017A5A
:1084000030EE670AE7EE007AB0EE670AC0ED007A58
:10841000704700BF704700BF06224FF47A730270A6
:1084200043607047F0B400250E4E00F1FF3C2F462C
:10843000142165B103788B420BD003460CEB050485
:1084400003E013F8012F8A4203D0A342F9D1C155AA
:10845000013701350B2D02D016F8011FE9E7F0BCFA
:10846000704700BFD890040830B415231625172490
:108470002D212E2203702F2345708470C17002714C
:10848000437130BC704700BF01212C2202230170D0
:1084900042708370704700BF012320212122417068
:1084A000427103720370037170476D4B2DE9F04FF9
:1084B0001C686C4BB3F80AE0B3F804809A894FEA61
:1084C0000E2AB4EB0A044FEA1E6B4FF0000587B08A
:1084D00065EB0B05CDE900450746009C1889019E18
:1084E000A0FB044500FB0655E00940EA45604FEA61
:1084F00008448C46E9114FEA184510EB0408D88867
:10850000009C41EB0509CDE90489A0FB0445B3F8C3
:10851000028000FB0655200A40EA05604FEAC83495
:1085200029124FEA584510EB040841EB0509009960
:10853000A2FB010102FB06114FEAD05A4AEA412A86
:108540001AF5FA634FEAE15B4BF10004B3F5FA6FF9
:10855000CDE9023474F10003414E64DA0524AAFB2C
:10856000040104FB0B1100FB0BF40AFB0144DDE9E1
:108570000423A0FB0A0121444D104FEA3004121BD2
:108580004FEA900463EB050344EA8174B8EB0408F6
:10859000CDE90423DDE9023433484FEAA10569EB54
:1085A00005094FF0FF31834274EB010326DA40F6F0
:1085B000AC501AEB00024FF000014BEB010302FB41
:1085C00003F1A2FB022303EB4103D400DD00101BE7
:1085D00045EA527563EB0501DDE9044524184D4178
:1085E000CDE904450B24A2FB040104FB031149104F
:1085F0004FEA3000B8EB000869EB0109DDE9003211
:108600005343009ADDE90201A2FB02AB0BEB430BE3
:108610004FEADA7242EA4B02801A4FEAEB7361EBDF
:108620000301CDE9020197B17168A1FB082301FBA9
:108630000933540D5D1544EAC324DDE90423A21A6D
:1086400065EB03031D46D30B43EA45433B60BCF196
:10865000000F02D0029BCCF8003007B0BDE8F08FCD
:10866000202700205446002024FAFFFF2DE9F04F78
:10867000DFF8DCC1754CDCF808502288B4F90AA098
:10868000C2EB25135200C2EBE502B4F902505B4382
:108690006A43B4F904501B135D43AD1305EBE225A7
:1086A000B5F5FA324FEAE57B85B04BF1FF33CDE902
:1086B0000023DDE900325343009AA561A2FB028941
:1086C000CDE90201B4F908200199009809EB4309AA
:1086D0005143D31700FB0311A2FB00230B444FEAC5
:1086E000EA7B0AFB09F11F0308FB0B13AAFB080135
:1086F00019444FEA102A4AEA016A16034FEA212B6D
:1087000047EA12571AEB0602E6884BEB070312F111
:10871000000A43F5004BAAFB060106FB0B114A10A9
:10872000CB1752EA030100F08E80B4F91060009874
:1087300006FB09F1F71708FB0711A6FB0867394488
:10874000B4F90E808B4601994FEAE87908FB01F1F4
:1087500000FB0911A8FB00898944DCF80C104FEAE2
:108760004947C1F5801C47EAD837B2464FEA484628
:10877000B4F90C801AEB060A66464BEB070BF717A9
:108780004FEAC806019600260096F907DDE9006762
:108790004FEACC7016EB0A0647EB0B0741EA5C0187
:1087A000801B61EB070140F6354C8946A0FB0C01AC
:1087B0000CFB09113EF0C2FDB4F91620B4F914A067
:1087C0004E13470B47EAC14702FB06FCD31707FBD2
:1087D00003CCA2FB07236344564307FB0366A2FBBB
:1087E00007233344560E46EAC31632184FEA63672E
:1087F00047EB010380460AFB01F14FEAEA7B08FBE5
:108800000B17AAFB08013944C60C46EA413612EBA5
:1088100006084FEAE147B4F9122043EB07094FEA93
:10882000182141EA096113010B44029A0AB11B0A9B
:108830001360039B23B105EB850580352D121D6068
:1088400005B0BDE8F08F0023EFE700BF68460020C9
:1088500020270020704770472DE9F041334B344EFC
:108860001A8A7489B6F91450B6F90480B6F90E70F4
:10887000B6F920C05B69121B34895443E213B6F980
:1088800012401544E40294FBF5F4B6F90250144486
:10889000A4F57A6E0EFB0EF20EFB05F50EFB08FE3C
:1088A000B6F90C80F4611213574302FB08F212145C
:1088B00002EB6E32ED1205EBE7270232B6F90050FB
:1088C000B6F806E0921002F5004207EB85070EFBB2
:1088D00002F207FA0CF74FEAD23E02374CF250325E
:1088E000A3EBA70742FA0CF37B4355BF5B00B3FB36
:1088F000FEF3B3FBFEF35B0078B11A1202FB02F544
:1089000040F6DE326A430B4D12145D4302EB254202
:1089100002F6CF6203EB2213036021B10A235C430A
:10892000083424110C60BDE8F08100BF202700202E
:108930003046002043E3FFFF4FF40063838270471B
:108940004FF4006383827047012380F854307047EE
:108950004FF4006383827047F0B4037C456902687A
:108960001F2B37D9203B2021546899400C4223D03B
:1089700010249C40D160D4605168D940CE074ED4B9
:10898000EFF31183502282F31288EA6B1168C90752
:1089900009D45468002C52D1D5E909618E4243D1E3
:1089A000012285F86020DBB283F31188037C026822
:1089B0001F2B194614D9203B0821506899400842C2
:1089C00000D0D1600421506801FA03F3184223D18A
:1089D000F0BC7047202416689C4026420FD11946EF
:1089E000082310688B40184200D09360042310685D
:1089F00003FA01F10842EBD09160F0BC70471021FE
:108A00009940946091601168D940CC07B8D5012194
:108A100001FA03F39360B3E7D360F0BC7047012120
:108A200001FA03F3D360ABE7AF690F44D7600ED808
:108A30002E69711A5160AC62002185F860101168CE
:108A400041F00101DBB2116083F31188AEE7711AC6
:108A50005160AE62F0E700BF70B4037C01681F2B69
:108A600026D9A3F1200520224C68AA40224214BF37
:108A700001220022D2B142691B481C4C02EB420287
:108A800000EB4212257854682068CDB9E568568914
:108A90002C6824F001042C6082891F2B22EA060234
:108AA00082811AD8202202FA03F38B6070BC7047CF
:108AB00020220C689A40224214BF01220022D9E7EA
:108AC000A469226822F001022260828922F4807265
:108AD0001204120C1F2B8281E4D9A3F1200220235F
:108AE0009340CB6070BC7047E0A20020DCA2002065
:108AF00070B59D4C2368002B40F005819B4B1A7884
:108B0000002A68D09A4B19789A4B002964D11868CA
:108B1000B3F82C5141628489012A44EA0504848116
:108B2000A3F82C1157D0D3F83001B3F85C5241624E
:108B30008489022A44EA05048481A3F85C124AD09D
:108B4000D3F86002B3F88C5341628489032A44EA63
:108B500005048481A3F88C133DD0D3F89003B3F8B7
:108B6000BC5441628489042A44EA05048481A3F840
:108B7000BC1430D0D3F8C004B3F8EC5541628489FA
:108B8000052A44EA05048481A3F8EC1523D0D3F820
:108B9000F005B3F81C5741628489062A44EA0504AB
:108BA0008481A3F81C1716D0D3F82007B3F84C58CB
:108BB00041628489072A44EA05048481A3F84C1899
:108BC00009D0D3F85028B3F87C49516290892043EA
:108BD0009081A3F87C1970BD5C6819896160256873
:108BE000186845F0010540F20D312560A0F84810E5
:108BF0008489012A44F480748481ECD0D3F8344110
:108C0000B3F83851D3F830016560256845F00105A7
:108C10002560A0F848108489022A44F48074848175
:108C2000D9D0D3F86442B3F86852D3F860026560D3
:108C3000256845F001052560A0F848108489032ABD
:108C400044F480748481C6D0D3F89443B3F8985325
:108C5000D3F890036560256845F001052560A0F80C
:108C600048108489042A44F480748481B3D0D3F8F2
:108C7000C444B3F8C854D3F8C0046560256845F00F
:108C800001052560A0F848108489052A44F4807401
:108C90008481A0D0D3F8F445B3F8F855D3F8F005A3
:108CA0006560256845F001052560A0F848108489B5
:108CB000062A44F4807484818DD0D3F82447B3F815
:108CC0002857D3F820076560256845F00105256021
:108CD000A0F848108489072A44F4807484813FF402
:108CE0007AAFD3F85428B3F85808D3F85038506006
:108CF000106840F001001060A3F848109A8942F40F
:108D000080729A8170BD054610F0A2FF217AA9B148
:108D10006DB1194A002316890133002E18BF0021B6
:108D2000AB4202F16002F6D100293FF4E7AE00F554
:108D30001C501030002320602372DFE62368C31A22
:108D4000002BFFF648AF637A3BB1013BDBB26372A5
:108D50002BB100F57A702060D0E62360CEE6636820
:108D600003442360CAE600BF902B0020E0A500204A
:108D7000DCA20020E4A50020E0A2002010B5027CC7
:108D800001681F2A4FF020030ED94C68203A934007
:108D90001C4208D00B4A406800241470026822F07C
:108DA00001020260CB6010BD0C6893401C42FAD0F7
:108DB000044A406800241470026822F00102026034
:108DC0008B60F0E7585000202DE9F041C4002318D3
:108DD0009B00B749CA585268958AADB2EFB2FE07F8
:108DE0000B4461D4BE0737D5BFF35F8F1D7EEDB254
:108DF000012D00F0BB80AF4E138BBFF35F8F2318A4
:108E000001EB83031D7E022D00F0CE80231801EBC1
:108E100083031D7E032D05D19B7E1BB1737E002B2A
:108E200040F01A81938896F918C043F480639380C8
:108E3000231801EB83031B7E013363450AD1B37E04
:108E400000257576002B40F08A80204401EB8000DD
:108E500000234375BDE8F081964E17F0040F96F994
:108E600018C04DD117F0400700F0B280178A1D6A74
:108E7000FFB205F80C705FFA8CF56F1C93F818E0E0
:108E80007BB2DF1CBE4533769C4600F00981271873
:108E900001EB87073F7EBB42CAD105F1020C4FFAB6
:108EA0008CFC86F818C0C3E71588824E25F400654F
:108EB0002D042D0C1580158845F4806515809D7E48
:108EC00000273776002D3DD0757E002D37D0231832
:108ED00001EB830301251B7E7576022B03D11388DA
:108EE00043F400631380231801EB83039B7D43F05D
:108EF00001031382204401EB8000037EBDE8F08172
:108F00009F7E757E4FF0010E86F81AE0002F5CD030
:108F1000002D78D1231801EB83035B7E002B00F03A
:108F2000A48013880CF1010C4FFA8CFC43F40073FD
:108F300086F818C013801388DF05FCD478E7DB7D42
:108F4000FF2BC4D0231801EB83039D7D05F0FE05A4
:108F50001582DB7DFF2BCDD0FF233376CAE79388C4
:108F600023F440731B041B0C93806EE79B7E514ED1
:108F7000002B3FF441AF737E002B3FF43DAF1388CD
:108F800023F480631B041B0C1380BFF35F8F138BD0
:108F90001388B57643F400731380938896F918C04C
:108FA00043F48063938043E79B7E002B3FF42EAF16
:108FB000737E002B3FF42AAF138896F918C023F470
:108FC00080631B041B0C138016E0002DA2D0A8E7C1
:108FD0002D067FF52DAFBCF1FF3F6DD0DD6915F893
:108FE0000C5015820CF1010C1D7E4FFA8CF39D4242
:108FF0009C4633767FF41CAF938823F480631B0474
:109000001B0C938014E71F7ED3F820805FFA8CF549
:10901000AE44022F4FFA8EFE17882DD927F48067B1
:109020003F043F0C1780178AFFB208F80C701788AE
:10903000D3F820C047F400731380138ADBB20CF816
:109040000E30938805F1020C4FFA8CFC43F48063D8
:1090500086F818C093806EE7938896F918C023F4B9
:1090600080631B041B0C9380E2E61388012543F404
:109070008073138075765EE747F400771780178A50
:10908000FFB208F80C70178AD3F8208005F1030CA2
:109090004FFA8CFCFBB286F818C008F80E304AE78D
:1090A000978827F480673F043F0C9780EFE600BF66
:1090B000D436002020270020DD7D15829D7E377666
:1090C0001DB91B7E002B7FF415AF938823F48063BA
:1090D0001B041B0C93800DE7014B186811F01EB8A0
:1090E000B43C002038B51D4B1B78044600F1250523
:1090F00093B104221A4920303EF000FC2846142285
:1091000018493EF0FBFB012384F83A30164B1B78DC
:1091100073B984F83B3038BD2846142213493EF019
:10912000EDFB012384F83A300F4B1B78002BF0D075
:109130000F4B186859689A68DD68E56020606160C7
:10914000A260DD69186959699A69A2610123E56124
:109150002061616184F83B3038BD00BFE5430020E9
:10916000E6430020EB430020C443002028CE04083F
:10917000C543002010B429212824012200230470B3
:1091800041708270C3705DF8044B704738B52C2273
:1091900000213EF075FB0346642140F2DC5240F2B0
:1091A000022019745A821321202240F21A4540F2FB
:1091B0006C74188399760E2002211A7701229D8201
:1091C000DC8240F2753540F6430483F822001972C0
:1091D00083F82A109A7383F82920DD831C841946AA
:1091E0000248BDE838401DF04FB800BF38CE040833
:1091F00010B50021044601200FF0F4FF207010BDCF
:1092000038B500240472451EE1B202200FF0EAFFD7
:109210000134082C05F8010FF6D138BDF0B5876987
:1092200083B0064617B13B68BA885A837069DFF885
:10923000A8E08389C3244FF47A734FF0060C6D467F
:109240004FF6FF710EF1010E03E0013B9BB28B4222
:1092500020D002899207F8D5A3B283814FF47A73A4
:1092600002E0A3B28B4215D00289D20703F1FF348A
:10927000F7D5828992B20DB12A700135BCF1000F89
:109280000BD00CF1FF3CFF24BEF1000FE1D09EF8A3
:109290000040D7E714F01CFFB76917B13B68BA88E4
:1092A0001A839DF805009DF801509DF802109DF865
:1092B00003409DF804209DF8063041EA052143EA69
:1092C000002342EA04220120A6F85010A6F85220FA
:1092D000A6F8543003B0F0BDE49004080122482100
:1092E00015F026B80122582115F022B83122F421B8
:1092F00015F01EB8044B93F820209201343202F08E
:10930000FC02F42115F014B8304600202E22F4217E
:1093100015F00EB807B5032301AA002114F03AFF97
:109320009DF805309DF804001B0243EA00439DF8B8
:109330000600184303B05DF804FB08B5FFF7EAFF29
:10934000014B586008BD00BF2027002008B5FFF77B
:10935000E1FF014B186008BD2027002007B5062358
:109360006A46F72114F016FF9DF801309DF80010B1
:109370000B4A1B0143EA01339DF8021043EA111323
:10938000D3609DF804309DF803101B0143EA0133BC
:109390009DF8051043EA1113936003B05DF804FBD8
:1093A0002027002007B5032301AAF62114F0F2FEBE
:1093B0009DF805309DF804201B0243EA02439DF806
:1093C00006201343054AB2F92020C2F10802D34017
:1093D000034A536103B05DF804FB00BF3046002030
:1093E0002027002007B5022301AAF62114F0D2FE9F
:1093F0009DF804209DF8053043EA0223024A1382B7
:1094000003B05DF804FB00BF2027002070B582B0D8
:109410000446062310306A46432114F0BBFEC0B157
:109420009DF804009DF800609DF801109DF8025021
:109430009DF803209DF8053041EA062143EA002308
:1094400042EA0522A4F85010A4F85220A4F854309F
:10945000012002B070BD00BF70B582B00446062383
:1094600008306A463B2114F095FEA8B19DF804002F
:109470009DF800609DF801109DF802509DF80320B2
:109480009DF8053041EA062143EA002342EA05221D
:10949000E18222836383012002B070BD2DE9F04F89
:1094A00089B0039090F86500002840F03786039B50
:1094B00093F85C30072B00F027861823CDE904339E
:1094C000039BC64CC64EDFF82483C64F10331846A4
:1094D00080226B21029314F02BFF6423DFF810E34A
:1094E000C14801934FF01009DEF80430C3F30803BC
:1094F000002B40F06284EFF31183002B40F05D8479
:109500002568826823689D42FAD13B689A42F7D861
:10951000D6F800C04FF47A7101FB0CF39B1AB3FB31
:10952000FCF301FB05354FF47A7C4FF0010ADEF8BD
:109530000430C3F30803002B40F0FF83EFF31183E3
:10954000002B40F0FA832368816822689342FAD1A5
:109550003A689142F7D832680CFB02FBABEB010191
:10956000B1FBF2F10CFB03135B1BB3F57A7FDED387
:10957000019B013B0193B7D1072268210298DFF8D4
:109580006C82984F14F0D4FE6423DFF864E29648AE
:1095900001934FF01009DEF80430C3F30803002BE9
:1095A00040F0EA83EFF31183002B40F0E583256858
:1095B000826823689D42FAD13B689A42F7D8D6F870
:1095C00000C04FF47A7101FB0CF39B1AB3FBFCF360
:1095D00001FB05354FF47A7C4FF0010ADEF80430C8
:1095E000C3F30803002B40F08A83EFF31183002BB1
:1095F00040F085832368816822689342FAD13A68F3
:109600009142F7D832680CFB02FBABEB0101B1FBD6
:10961000F2F10CFB03135B1BB3F57A7FDED3019BE6
:10962000013B0193B7D11A466B210298DFF8BC8148
:109630006C4F14F07DFE6423DFF8B4E16A480193B7
:109640004FF01009DEF80430C3F30803002B40F09C
:10965000F783EFF31183002B40F0F28325688268D3
:1096600023689D42FAD13B689A42F7D8D6F800C0E9
:109670004FF47A7101FB0CF39B1AB3FBFCF301FB73
:1096800005354FF47A7C4FF0010ADEF80430C3F35D
:109690000803002B40F01583EFF31183002B40F0FB
:1096A00010832368816822689342FAD13A68914214
:1096B000F7D832680CFB02FBABEB0101B1FBF2F116
:1096C0000CFB03135B1BB3F57A7FDED3019B013BDD
:1096D0000193B7D101226B210298DFF81081414F2D
:1096E00014F026FE0F23DFF808E13F4801934FF006
:1096F0001009DEF80430C3F30803002B40F07F8329
:10970000EFF31183002B40F07A8325688268236889
:109710009D42FAD13B689A42F7D8D6F800C04FF480
:109720007A7101FB0CF39B1AB3FBFCF301FB0535CB
:109730004FF47A7C4FF0010ADEF80430C3F30803DB
:10974000002B40F0A082EFF31183002B40F09B82AE
:109750002368816822689342FAD13A689142F7D827
:1097600032680CFB02FBABEB0101B1FBF2F10CFB2D
:1097700003135B1BB3F57A7FDED3019B013B01939F
:10978000B7D1039A92F85F30032B09D992F863306E
:10979000012B049B0CBF43F0010343F0020304932D
:1097A0009DF810200298DFF844800E4F1B2114F022
:1097B000BFFD0F23DFF838E00B4801934FF010098D
:1097C000DEF80430C3F30803002B40F07C83EFF392
:1097D0001183002B40F077830CE000BF4085002010
:1097E000448500204885002010E000E03C850020F2
:1097F00000ED00E02568826823689D42FAD13B684D
:109800009A42F7D8D6F800C04FF47A7101FB0CF3F6
:109810009B1AB3FBFCF301FB05354FF47A7C4FF048
:10982000010ADEF80430C3F30803002B40F00D8278
:10983000EFF31183002B40F00882236881682268CF
:109840009342FAD13A689142F7D832680CFB02FB96
:10985000ABEB0101B1FBF2F10CFB03135B1BB3F5A6
:109860007A7FDED3019B013B0193A9D1059A02982F
:10987000DFF81483C24F1C2114F05AFD0F23DFF8C8
:109880000CE3C04801934FF01009DEF80430C3F335
:109890000803002B40F0F682EFF31183002B40F019
:1098A000F1822568826823689D42FAD13B689A421A
:1098B000F7D8D6F800C04FF47A7101FB0CF39B1A6D
:1098C000B3FBFCF301FB05354FF47A7C4FF0010A42
:1098D000DEF80430C3F30803002B40F09881EFF367
:1098E0001183002B40F093812368816822689342A2
:1098F000FAD13A689142F7D832680CFB02FBABEB25
:109900000101B1FBF2F10CFB03135B1BB3F57A7F92
:10991000DED3019B013B0193B7D1039A92F85F30EC
:10992000032B00F2EF8392F86220012A00F0EC8210
:10993000A2F10202B2FA82F252091A210298DFF869
:1099400048828F4F14F0F4FC0F23DFF840E28D487B
:1099500001934FF01009DEF80430C3F30803002B25
:1099600040F04C83EFF31183002B40F047832568D0
:10997000826823689D42FAD13B689A42F7D8D6F8AC
:1099800000C04FF47A7101FB0CF39B1AB3FBFCF39C
:1099900001FB05354FF47A7C4FF0010ADEF8043004
:1099A000C3F30803002B40F00B83EFF31183002B6C
:1099B00040F006832368816822689342FAD13A68AE
:1099C0009142F7D832680CFB02FBABEB0101B1FB13
:1099D000F2F10CFB03135B1BB3F57A7FDED3019B23
:1099E000013B0193B7D1039B029893F86420DFF801
:1099F0009881634F192114F09BFC6423DFF88CE1FC
:109A0000604801934FF01009DEF80430C3F30803F7
:109A1000002B40F03583EFF31183002B40F03083AF
:109A20002568826823689D42FAD13B689A42F7D83C
:109A3000D6F800C04FF47A7101FB0CF39B1AB3FB0C
:109A4000FCF301FB05354FF47A7C4FF0010ADEF898
:109A50000430C3F30803002B40F09482EFF311832A
:109A6000002B40F08F822368816822689342FAD1EC
:109A70003A689142F7D832680CFB02FBABEB01016C
:109A8000B1FBF2F10CFB03135B1BB3F57A7FDED362
:109A9000019B013B0193B7D1102237210298DFF8D7
:109AA000E880374F14F044FC0F23DFF8E0E035483E
:109AB00001934FF01009DEF80430C3F30803002BC4
:109AC00040F0BD82EFF31183002B40F0B88225688F
:109AD000826823689D42FAD13B689A42F7D8D6F84B
:109AE00000C04FF47A7101FB0CF39B1AB3FBFCF33B
:109AF00001FB05354FF47A7C4FF0010ADEF80430A3
:109B0000C3F30803002B40F01F82EFF31183002BF7
:109B100040F01A822368816822689342FAD13A6839
:109B20009142F7D832680CFB02FBABEB0101B1FBB1
:109B3000F2F10CFB03135B1BB3F57A7FDED3019BC1
:109B4000013B0193B7D10298DFF83C800C4F012212
:109B5000382114F0EDFB0F23DFF830E009480193C2
:109B60004FF01009DEF80430C3F30803002B40F077
:109B7000A882EFF31183002B40F0A38208E000BF1E
:109B80004885002010E000E03C85002000ED00E06A
:109B90002568826823689D42FAD13B689A42F7D8CB
:109BA000D6F800C04FF47A7101FB0CF39B1AB3FB9B
:109BB000FCF301FB05354FF47A7C4FF0010ADEF827
:109BC0000430C3F30803002B40F0A081EFF31183AE
:109BD000002B40F09B812368816822689342FAD170
:109BE0003A689142F7D832680CFB02FBABEB0101FB
:109BF000B1FBF2F10CFB03135B1BB3F57A7FDED3F1
:109C0000019B013B0193ADD109B0BDE8F08FEFF3AB
:109C1000118189F31288D0F808B00368DB0344BFD0
:109C2000C8F800A0D0F808B02368D8F80020C9B25E
:109C300081F31188316813440CFB01F2A2EB0B0293
:109C4000B2FBF1F20CFB03235FE6EFF3118189F322
:109C50001288D0F808B00368DB0344BFC8F800A03E
:109C6000D0F808B02368D8F80020C9B281F3118871
:109C7000316813440CFB01F2A2EB0B02B2FBF1F2D0
:109C80000CFB0323EAE5EFF3118189F31288D0F886
:109C900008B00368DB0344BFC8F800A0D0F808B0E0
:109CA0002368D8F80020C9B281F3118831681344C1
:109CB0000CFB01F2A2EB0B02B2FBF1F20CFB032353
:109CC00057E5EFF3118189F31288D0F808B00368E3
:109CD000DB0344BFC8F800A0D0F808B02368D8F868
:109CE0000020C9B281F31188316813440CFB01F2E2
:109CF000A2EB0B02B2FBF1F20CFB0323E2E4EFF365
:109D0000118189F31288D0F808B00368DB0344BFDF
:109D1000C8F800A0D0F808B02368D8F80020C9B26D
:109D200081F31188316813440CFB01F2A2EB0B02A2
:109D3000B2FBF1F20CFB03236DE4EFF3118189F325
:109D40001288D0F808B00368DB0344BFC8F800A04D
:109D5000D0F808B02368D8F80020C9B281F3118880
:109D6000316813440CFB01F2A2EB0B02B2FBF1F2DF
:109D70000CFB0323FFF7F8BBEFF3118389F3128881
:109D8000D0F808C00268D20304D50122C8F8002028
:109D9000D0F808C02568D8F800A0DBB283F311889A
:109DA00031684FF47A72554402FB01F3A3EB0C03C4
:109DB000B3FBF1F302FB05350CE4EFF3118389F3F8
:109DC0001288D0F808C00268D20304D50122C8F86E
:109DD0000020D0F808C02568D8F800A0DBB283F3D3
:109DE000118831684FF47A72554402FB01F3A3EBFA
:109DF0000C03B3FBF1F302FB0535FFF794BBEFF364
:109E0000118389F31288D0F808C00268D20304D500
:109E10000122C8F80020D0F808C02568D8F800A0B2
:109E2000DBB283F3118831684FF47A72554402FB38
:109E300001F3A3EB0C03B3FBF1F302FB053577E46D
:109E4000EFF3118389F31288D0F808C00268D203B7
:109E500004D50122C8F80020D0F808C02568D8F839
:109E600000A0DBB283F3118831684FF47A72554455
:109E700002FB01F3A3EB0C03B3FBF1F302FB05358B
:109E8000FFF7FFBBEFF3118389F31288D0F808C006
:109E90000268D20304D50122C8F80020D0F808C017
:109EA0002568D8F800A0DBB283F3118831684FF43D
:109EB0007A72554402FB01F3A3EB0C03B3FBF1F3FD
:109EC00002FB053500E5EFF3118389F31288D0F822
:109ED00008C00268D20304D50122C8F80020D0F8D7
:109EE00008C02568D8F800A0DBB283F31188316878
:109EF0004FF47A72554402FB01F3A3EB0C03B3FB5E
:109F0000F1F302FB053588E4072216E5EFF3118132
:109F100089F31288D0F808B00368DB0344BFC8F89F
:109F200000A0D0F808B02368D8F80020C9B281F3A7
:109F30001188316813440CFB01F2A2EB0B02B2FB57
:109F4000F1F20CFB032357E6EFF3118189F312883A
:109F5000D0F808B00368DB0344BFC8F800A0D0F80D
:109F600008B02368D8F80020C9B281F3118831689D
:109F700013440CFB01F2A2EB0B02B2FBF1F20CFB5F
:109F80000323D8E5EFF3118189F31288D0F808B0E4
:109F90000368DB0344BFC8F800A0D0F808B023680A
:109FA000D8F80020C9B281F31188316813440CFB42
:109FB00001F2A2EB0B02B2FBF1F20CFB032363E50F
:109FC000EFF3118189F31288D0F808B00368DB033E
:109FD00044BFC8F800A0D0F808B02368D8F8002023
:109FE000C9B281F31188316813440CFB01F2A2EB72
:109FF0000B02B2FBF1F20CFB0323ECE4EFF3118351
:10A0000089F31288D0F808C00268D20304D501226F
:10A01000C8F80020D0F808C02568D8F800A0DBB246
:10A0200083F3118831684FF47A72554402FB01F3CF
:10A03000A3EB0C03B3FBF1F302FB0535AAE4EFF34A
:10A04000118389F31288D0F808C00268D20304D5BE
:10A050000122C8F80020D0F808C02568D8F800A070
:10A06000DBB283F3118831684FF47A72554402FBF6
:10A0700001F3A3EB0C03B3FBF1F302FB053539E568
:10A08000EFF3118389F31288D0F808C00268D20375
:10A0900004D50122C8F80020D0F808C02568D8F8F7
:10A0A00000A0DBB283F3118831684FF47A72554413
:10A0B00002FB01F3A3EB0C03B3FBF1F302FB053549
:10A0C000C1E4EFF3118389F31288D0F808C0026865
:10A0D000D20304D50122C8F80020D0F808C02568B2
:10A0E000D8F800A0DBB283F3118831684FF47A729C
:10A0F000554402FB01F3A3EB0C03B3FBF1F302FBAA
:10A10000053558E5019A18E4039B93F86130002B5C
:10A1100046D11023CDE90433FFF7D2B90EF0E8FBA6
:10A12000039B044603F10C0500283FD00068284932
:10A1300000F13F4303F57E039A0A01238A5C02F093
:10A140001F01520920268B40032A4FF00001A671FF
:10A15000E17138D0042A31D0022A03D11D4A516C52
:10A160000B435364A388069306A90023079328F0A2
:10A17000B5FC039A184BD3602946204630F060FFA7
:10A18000A388B3FA83F3C3F11F03012212FA03F386
:10A190003FF48DA911490A6813430B60FFF787B993
:10A1A00018231021CDE90431FFF78AB91A460A4B6A
:10A1B000D360294630F044FFFFF779B9054A116BA7
:10A1C0000B431363CEE7034A116C0B431364C9E7D7
:10A1D00074C304080038024049890008003C01406B
:10A1E0002DE9F04F804B426983B09A42019000F014
:10A1F000D88003F580639A4200F0D380138823F05F
:10A2000040031B041B0C1380138823F038031B042A
:10A210001B0C30210B431380138843F04003138041
:10A2200001200FF067FD019C2046FFF737F9A36975
:10A2300013B11A689B885383019B586940F2E93334
:10A2400002E0002B00F0C7800289013B12F0020FF0
:10A250009BB2F6D06A23838140F2E93302E0002BFF
:10A2600000F0B9800289013B12F0010F9BB2F6D0D9
:10A27000838940F2E93302E0002B00F0B1800289CB
:10A28000013B12F0020F9BB2F6D01023838140F203
:10A29000E93302E0002B00F0A3800289013B12F0B9
:10A2A000010F9BB2F6D08389019B9B6913B11A6899
:10A2B0009B88138364234D4CDFF83C91DFF83C818D
:10A2C0004B4DDFF83CA14B4E00930FF0C1FC4FF417
:10A2D0007A774FF0100C4FF0010ED8F80430C3F32A
:10A2E0000803002B3ED1EFF31183002B3AD12368F2
:10A2F000A96822689342FAD132689142F7D8D9F816
:10A30000002007FB02FBABEB0101B1FBF2F107FB05
:10A3100003131B1AB3F57A7FDFD3009B013B009335
:10A32000D3D1019B5A69304B9A4247D003F58063E1
:10A330009A4243D0138823F040031B041B0C138064
:10A34000138823F038031B041B0C08210B431380D4
:10A350001388012043F04003138003B0BDE8F04FA1
:10A360000FF0C8BCEFF311818CF31288D5F808B058
:10A370002B68DB0344BFCAF800E0D5F808B02368B7
:10A38000DAF80020C9B281F31188D9F8001013441B
:10A3900007FB01F2A2EB0B02B2FBF1F207FB032376
:10A3A000B7E7138823F040031B041B0C13801388AA
:10A3B00023F038031B041B0C28212BE7138823F000
:10A3C00040031B041B0C1380138823F038031B0469
:10A3D0001B0C0021BAE713F07BFE019B586948E78C
:10A3E00013F076FE60E700BF003800404085002093
:10A3F00010E000E0488500204485002000ED00E0EA
:10A400003C850020F8B50468C4F30D0405460E46EB
:10A4100004B32F6828F050FB092840F08880454C91
:10A42000236923F440732361236943F40073236198
:10A43000236943F0010323613E6028F03DFB23695B
:10A44000092823F00103236171D12B6804332B60A9
:10A45000002035E0384B394A93422BD902F580422F
:10A46000934226D902F5804293422AD902F58042CE
:10A47000934228D902F58032934226D902F5003260
:10A48000934224D902F50032934222D902F50032D8
:10A49000934220D902F5003293421ED902F5802260
:10A4A00093421CD9B3F1016F1BD305200FF04AF979
:10A4B000FBE7082428F000FB092814D04FF0FF30F8
:10A4C000F8BD1024F6E71824F4E72024F2E7282446
:10A4D000F0E73024EEE73824ECE74024EAE74824AC
:10A4E000E8E75824E6E7134F3B6923F440733B61E8
:10A4F0003B6943F400733B613B6923F0F8033B6124
:10A500003B6943F002031C433C613B6943F48033E5
:10A510003B6128F0D1FA3B6923F002033B613B69C0
:10A52000092823F0F8033B613FF473AFC6E76FF0EF
:10A530000100C5E7003C024000400008FF3F000862
:10A54000F8B504460D468E180027B542206900D1A3
:10A55000F8BDE368591CE160234415F8012B1A7219
:10A560000429F2D118B9A1682046FFF74BFFC4E9CE
:10A570000370EAE7024A136823EA0000106070479C
:10A58000BC620020DFED2E7AB4EEE70AF1EE10FA9D
:10A590004ADDDFED2C6A9FED2C7A01E0B0EE670A10
:10A5A000B4EEC70AF1EE10FA70EE667AF6DC9FEDB3
:10A5B000277AF4EEC77AF1EE10FA3ED5DFED216A84
:10A5C0009FED237A01E0F0EE407AF4EEC77AF1EEE7
:10A5D00010FA37EEA60AF6D4DFED1E7AB4EEE70ADB
:10A5E000F1EE10FA14DDDFED167A37EEC00A60EEF8
:10A5F000006A9FED196A9FED197ADFED197AA6EED0
:10A60000867A20EE266AE6EE877AA6EE270A70475B
:10A61000DFED147AB4EEE70AF1EE10FA44BFDFED95
:10A620000B7A37EEC00AE2E79FED087AF0EE407A47
:10A63000F4EEC77AF1EE10FAC0D4B0EE670ACBE7B9
:10A64000DB0F4940DB0FC940E4CB1641DB0F49C0AB
:10A65000E4CB16C1DB0FC93F92E741B99730083C04
:10A6600015A82ABEDB0FC9BFF0EEC07AB0EEE07AC3
:10A67000B4EEE77AF1EE10FAB4BFB0EE676AB0EE6E
:10A68000476AB5EE406AF1EE10FA46D0B4EEE77ACA
:10A69000F1EE10FA8CBFF0EE675AF0EE475AC5EEB5
:10A6A000866A9FED1F3A9FED1F6A9FED1F4A9FED3F
:10A6B0001F5ADFED1F3ADFED1F4ADFED1F5AA6EEEE
:10A6C000C36AE6EEA34AA6EE864AB7EE006AA6EE95
:10A6D000845AA6EEA46AE6EE855AC5EE866AB4EE02
:10A6E000E77AF1EE10FA48BFDFED147AF5EEC00A12
:10A6F00048BF77EEE66AF1EE10FA48BFDFED107A58
:10A70000B5EEC00A48BF77EEE66AF1EE10FA48BF30
:10A71000F1EE666AB0EE660A7047DFED076ADEE7C3
:10A7200039094E3DE3B59E3E88FA163E45FE7F3F11
:10A7300099FB243F69A2163EA7DFA834DB0FC93F6F
:10A74000DB0F4940DFED317A30EE277AFDEEC76A44
:10A7500016EE903A2033402B02D99FED2D0A704718
:10A76000B4EEE70AF1EE10FA4DDD9FED2A6ADFED57
:10A770002A6A01E0B0EE677AB4EEE67AF1EE10FAFA
:10A7800077EE467AF6DC9FED257AF4EEC77AF1EEA5
:10A7900010FA35D5DFED1F6A9FED217A01E0F0EE6A
:10A7A000407AF4EEC77AF1EE10FA37EEA60AF6D444
:10A7B000DFED167AB4EEE70AF1EE10FA1BDCDFEDFE
:10A7C000197AB4EEE70AF1EE10FA44BFDFED137A1E
:10A7D00037EEC00A60EE006A9FED136A9FED137AB0
:10A7E000DFED137AA6EE867A20EE266AE6EE877A09
:10A7F000A6EE270A7047DFED0F7A37EEC00AE9E7C9
:10A80000B0EE670AD4E7F0EE477ABCE7DB0FC93F4A
:10A8100000000000DB0FC940E4CB1641DB0F49C04C
:10A82000E4CB16C1DB0FC9BF92E741B99730083CB2
:10A8300015A82ABEDB0F4940FDEEC07A17EE903A0C
:10A840002033402B45D8DFED2D7AB4EEE70AF1EE48
:10A8500010FA4DDDDFED2A6A9FED2A7A01E0B0EEB5
:10A86000670AB4EEC70AF1EE10FA70EE667AF6DC0B
:10A870009FED257AF4EEC77AF1EE10FA3BD5DFEDC5
:10A88000206A9FED227A01E0F0EE407AF4EEC77A7A
:10A89000F1EE10FA37EEA60AF6D4DFED1D7AB4EE2B
:10A8A000E70AF1EE10FA17DDDFED147A37EEC00A91
:10A8B00060EE006A9FED176A9FED177ADFED177A59
:10A8C000A6EE867A20EE266AE6EE877AA6EE270ABC
:10A8D00070479FED130A7047DFED127AB4EEE70A76
:10A8E000F1EE10FA44BFDFED087A37EEC00ADFE779
:10A8F000F0EE407ABCE7B0EE670ACEE7DB0F4940E6
:10A90000DB0FC940E4CB1641DB0F49C0E4CB16C1D5
:10A91000DB0FC93F92E741B99730083C15A82ABE22
:10A9200000000000DB0FC9BF10B44C09012250F831
:10A93000243001F01F0102FA01F10B4340F82430EA
:10A940005DF8044B704700BF4B0901F01F0150F840
:10A950002320012303FA01F1114214BF18460020FD
:10A96000704700BF2DE9F043002489B006460D462C
:10A970001F46A04605E025290CD030460134A847E3
:10A98000039A531C039311780029F4D1204609B08F
:10A99000BDE8F083931CCDE903385078302842D0CD
:10A9A000A0F13003DBB2092B4FF0000945D96C2828
:10A9B0002AD0642873D019D9732858D063D9752840
:10A9C00040F0828007F1040C386805AB00220A21B0
:10A9D0006746FDF779FC05AB049A009329464B4680
:10A9E0003046FDF713FB039A0444CAE725283CD000
:10A9F00051D958286BD06328C2D139783046A8473E
:10AA000004370134039ABCE7039B5A1C03921B785A
:10AA1000642B52D016D8252B27D064D9582B18D0A8
:10AA2000632BEAD0ADE7D31C03939078A0F13003F9
:10AA3000DBB2092B4FF00109B9D804AA03A931F000
:10AA4000A9FCB4E7732B12D051D9752B2DD0782BDC
:10AA500097D1A3F15802B2FA82F23868520905ABD5
:10AA600010210437FDF730FCB5E7252185E73B6869
:10AA7000049A0093294600233046FDF7C7FA0437AD
:10AA80000444039A7DE76E287FF47AAF039A3B680B
:10AA900004371C6075E700283FF478AF70E738682A
:10AAA00005A9FDF7DBFB043795E7386805AB002205
:10AAB0000A21FDF709FC04378DE73B1D386805A91D
:10AAC0001F46FDF7CBFB86E778287FF459AFA0F14E
:10AAD0005802B2FA82F23868520905AB1021FDF72C
:10AAE000F3FB043777E7002B3FF450AF49E76E2BB9
:10AAF000CDD046E70EB400B584B005AB019053F855
:10AB0000042B0649039301A8FFF72CFF019B0022A9
:10AB10001A7004B05DF804EB03B0704701800008C0
:10AB200070B406688E4217D90139751E002311F8DA
:10AB3000014F0822634013F0800F4FEA430318BF10
:10AB400083F0D503013ADBB2F5D18D42EFD1721C0F
:10AB50000260337070BC7047721C00230260337057
:10AB600070BC70470A44914215D010B40139541E8C
:10AB700011F8012F0823504010F0800F4FEA4000D9
:10AB800018BF80F0D500013BC0B2F5D1A142EFD192
:10AB90005DF8044B704770474840082310F0800F61
:10ABA0004FEA400018BF80F0D500013BC0B2F5D19C
:10ABB000704700BF0A44914215D030B40139551E88
:10ABC00041F2210211F8014F082380EA0420040415
:10ABD0004CBF82EA40004000013B80B2F7D18D4279
:10ABE000F0D130BC704770472DE90048FDF702FBFB
:10ABF000054A064B1268B0EB020B61F1000CC3E989
:10AC000000BC0120BDE8008840850020A060002035
:10AC10000F4B2DE93048D3E9004554EA05020AD12B
:10AC2000034640F2011200201880988098715A80E3
:10AC30001881BDE83088074B1A6814EB020B45F108
:10AC4000000C5A466346FDF71DFA0120BDE8308826
:10AC5000A0600020408500202DE9F04707468CB019
:10AC60001E469246002A5CD1154614460A88B2F563
:10AC7000FA6F36D38B78581E0B2832D891F803C060
:10AC80000CF1FF301E282CD891F804E0BEF1170F0C
:10AC900027D891F80590B9F13B0F22D888793B2845
:10ACA0001FD8B1F80880B8F57A7F1AD24FF00108A2
:10ACB0005EBB09890491002CB4BF2D212B21002CEF
:10ACC000B8BF6442CDE90290CDE905140795CDE9FE
:10ACD00000CE38462A49FFF70DFF40460CB0BDE8CC
:10ACE000F08700232749ADF828304FF0010C1846B3
:10ACF0008DF82A30ADF82C3099469E461A46984673
:10AD00000991634609A9002ED3D0CDE90290CDE97F
:10AD100000CE38461C49FFF7EDFE40460CB0BDE8BA
:10AD2000F0871A4C84FB0234A318D417C4EB6314C5
:10AD3000C4EB0415A2EB85052DB2002D0846B8BF63
:10AD40006D42FDF757FA4FF47A7200238046894628
:10AD50003CF0F4FA3C230AFB030A4FF47A72002316
:10AD6000404649463CF0EAFA4FF47A7192B2002329
:10AD7000C1FB0A2309A8FDF785F924B209A975E7E3
:10AD800064CE04080000010144CE04088988888844
:10AD90000378202B024600F10100F9D0092BF7D0EF
:10ADA0002D2B00F0A4802B2B03BF5378B7EE000AA5
:10ADB0000246B7EE000AA3F13001C8B209289FEDA0
:10ADC000577A10D8F2EE046A07EE901AF8EEE77A96
:10ADD00012F8013FE7EE267AA3F13001C8B2092844
:10ADE000B0EE677AF0D92E2B63D003F0DF03452B4A
:10ADF00002D020EE070A704710B451782D294FD0A9
:10AE00002B2979D0A1F13003092B02F101027AD864
:10AE10000024002303EB830301EB430312F8011F1B
:10AE2000A1F130000928A3F13003F3D9B3F59A7FDB
:10AE30001A4628BF4FF49A72072B6CD9DFED386A97
:10AE40001346F7EE007A083B072B67EEA67AFAD88E
:10AE500002F00702DAB1F2EE046A012A67EEA67A7E
:10AE600015D0022A67EEA67A11D0032A67EEA67AD9
:10AE70000DD0042A67EEA67A09D0052A67EEA67AD5
:10AE800005D067EEA67A062A18BF67EEA67A002CD0
:10AE90003BD087EE277A5DF8044B20EE070A704717
:10AEA0009178A1F13003092B02F1020230D801247C
:10AEB000AFE75378A3F13001C8B2092802F10102CB
:10AEC00093D8F2EE046AF0EE665A07EE901AF8EEA6
:10AED000E77A12F8013F87EEA66AA3F13001C8B203
:10AEE000092866EEA56A37EE067AEED97DE7537833
:10AEF000BFEE000A02465EE79178A1F13003092B0C
:10AF000002F1020284D9F7EE007A27EE277AC2E72F
:10AF1000F7EE007ABDE7F7EE007A9BE7000000004D
:10AF200020BCBE4CB5EEC00ADFED317AF1EE10FA6E
:10AF3000CCBF30EE270A30EE670ADFED2E7A20EE26
:10AF4000270A30B5FDEEC07A87B017EE904A054665
:10AF500084EAE470002303A9A0EBE470CDE9003398
:10AF6000029333F0ADFB002CACBF20232D2303A8AC
:10AF70008DF800303BF0F6FC012803A924D002280C
:10AF80002DD0032805BF3023684668468DF8013070
:10AF90003CF07EFC68463BF0E5FC0338C4B2224638
:10AFA000694628463CF0AAFC00232B5528463BF076
:10AFB000D9FC2E22431C2A540DEB0401E8183CF066
:10AFC00083FC284607B030BD302368468DF8013039
:10AFD0008DF802308DF803303CF05AFCDAE730236C
:10AFE00068468DF801308DF802303CF051FCD1E715
:10AFF0006F12033A00007A44F8B506461546084633
:10B00000B6FBF2F434B905FB14640C4B1B5D00F87D
:10B01000013BF8BDB4FBF2F75FB905FB1747074BDF
:10B0200005FB1464DA5D00F8012B1B5D00F8013BA1
:10B03000F8BD3846FFF7E0FFEFE700BF94CE040805
:10B0400002B370B48E1803E0121B14D1B14215D0B4
:10B0500010F8012BA2F14103192B11F8013BA3F1C8
:10B06000410598BF2032192D03F12004ECD9D21AE2
:10B0700001D1002BEAD1104670BC70470022104667
:10B0800070BC70471046704770B5044608460D46C0
:10B090003BF068FC064602E014F8013F43B132463B
:10B0A00029462046FFF7CCFF0028F5D1204670BD89
:10B0B0001C46204670BD00BF4FF0FF32FFF7C0BFF7
:10B0C000A0F16103192B98BF20387047A0F141030C
:10B0D000192B98BF20307047202805D00938042844
:10B0E0008CBF002001207047012070472DE9F041FE
:10B0F0001F46064603461C782046FFF7EDFF1D4617
:10B1000001330028F7D12B2C51D02D2C24D0102A1C
:10B11000804628D04FF0FF33B3FBF2F302FB03FC71
:10B120006FEA0C0C5FFA8CFC013500200BE0303C20
:10B13000E4B2944225DA98422E461DD81AD002FB7A
:10B14000004015F8014B392CF1D944F02004602C53
:10B1500017D9573CE4B2ECE74FF00108102A6C789D
:10B1600005F10105D6D1302C23D06FF070434FF09C
:10B170000F0CD9E76445E2D907EA08084FF0FF3021
:10B18000DFE701B10E60B8F1000F08D027B1B0F1D0
:10B19000004F28BF4FF000404042BDE8F081002F33
:10B1A000FBD06FF00043984228BF1846F5E7804671
:10B1B000D4E76C782046FFF789FF782805F101066F
:10B1C00005D035466FF070434FF00F0CACE7AC780C
:10B1D0006FF0704302354FF00F0CA5E701230A22F0
:10B1E000002183E7613819288CBF002001207047B7
:10B1F000413819288CBF00200120704730380928B9
:10B200008CBF002001207047A0F13003092B07D923
:10B2100020F02000413819288CBF00200120704701
:10B220000120704707EE901AF8EE677A9FED837A57
:10B2300027EE800A20EE070AFDEEC07A17EE903A5C
:10B240002033402B00F28180DFED7D7AB4EEE70AF7
:10B25000F1EE10FA40F3E680B0EE407A9FED796AA5
:10B26000DFED796A01E0B0EE677AB4EEE67AF1EEEE
:10B2700010FA77EE467AF6DC9FED747AF4EEC77A30
:10B28000F1EE10FA40F1D1809FED6E6ADFED706A49
:10B2900001E0F0EE477AF4EEE67AF1EE10FA37EEDE
:10B2A000867AF6D4DFED6B7AB4EEE77AF1EE10FA37
:10B2B00040F3A780DFED627A37EEC77A27EE076AA0
:10B2C000DFED655ADFED657ADFED656A9FED655A62
:10B2D000E6EE257A67EE065AE6EE276AF7EE007A82
:10B2E000A5EEA67AF0EE675AE7EE055AE7EE457A44
:10B2F00087EEA55ADFED577A30EE277AFDEEC76A62
:10B3000016EE903A2033402B24D99FED577AF6EE73
:10B31000006AB7EE006AF7EE004AC4EEA57A002391
:10B32000836143610362C36180ED045A67EEA66ADC
:10B3300027EE866A27EE877AC0ED006AC0ED026AC2
:10B3400080ED016A80ED037A7047B7EE005AF0EEA7
:10B35000455ACFE7B4EEE70AF1EE10FA6BDD9FED48
:10B36000396ADFED396A01E0B0EE677AB4EEE67A69
:10B37000F1EE10FA77EE467AF6DC9FED347AF4EED1
:10B38000C77AF1EE10FA53D59FED2E6ADFED306AE1
:10B3900001E0F0EE477AF4EEE67AF1EE10FA37EEDD
:10B3A000867AF6D4DFED2B7AB4EEE77AF1EE10FA76
:10B3B00033DCDFED2E7AB4EEE77AF1EE10FA44BF1B
:10B3C000DFED227A37EEC77A27EE076ADFED224AF1
:10B3D000DFED226ADFED227AE6EE246A67EE064AA6
:10B3E000E6EE267AB7EE006AA4EEA77AF6EE006AD9
:10B3F00036EE476AF8EE007A27EE277A66EE266A7E
:10B4000089E7DFED1A7AB4EEE77AF1EE10FA44BF7D
:10B41000DFED0E7A37EEC77A50E7DFED097A37EEC7
:10B42000C77AD1E7F0EE407A26E7B0EE677A39E7DF
:10B43000B0EE677AB6E7F0EE477A9EE727D4D236C9
:10B44000DB0F4940DB0FC940E4CB1641DB0F49C09D
:10B45000E4CB16C1DB0FC93F92E741B99730083CF6
:10B4600015A82ABEF304353F00000000DB0FC9BF5A
:10B4700010EE103AC3F3160242F07E5207EE102A85
:10B48000DFED167ADFED164A9FED165ADFED165AFC
:10B490009FED166ADFED163ADFED166A9FED164A4C
:10B4A000E7EE274ADB1507EE903AA4EE875AF8EE4E
:10B4B000E77AE5EE075A67EEA37AA5EE876AB5EE5E
:10B4C000C00AE6EE077AF1EE10FAD4BFB0EE440AF5
:10B4D000B0EE660A37EE800A704700BFDACDFE3C58
:10B4E000B9D593BE5CB8903FAA841DC022E06140EC
:10B4F0001872313F07F1B3C2000080FFDFED1D3A43
:10B50000DFED1D7A9FED1D7A9FED1D4ADFED1D4A8F
:10B510009FED1D5ADFED1D5A9FED1D6ADFED1D6A7F
:10B52000E0EE237AF4EEC77AF1EE10FA88BFF0EE7F
:10B53000477AF4EEC47AF1EE10FAB8BFF0EE447A2E
:10B54000FDEEE77A17EE903AC3F3160242F07E5210
:10B5500007EE102AA7EE245A03F0FF4300EE103A3C
:10B56000E5EE075AA5EE876AE6EE076A26EE800A40
:10B57000704700BF3BAA384B00007E4E0000FF4ED4
:10B5800000000000ED185E3C81900FBBAF9D2A3E8D
:10B59000B2D19F3EE886023F30B402681146531C88
:10B5A000036011F8024B0160D31C5178036093785B
:10B5B000151D05601B0443EA0123D078234343EAA9
:10B5C000006030BC704700BF0368591C1A46016018
:10B5D00012F8021B0260587841EA0020704700BF51
:10B5E00003685A1C02601878704700BF70B50446A3
:10B5F00008460E463BF0B6F931460546024620683D
:10B600003CF0D8F820682844206070BD38B5044666
:10B61000006815463CF0CEF822682A44226038BD06
:10B62000036810B40A0E5C1C04601A7003680A0CEC
:10B630005C1C04601A7003680A0A5C1C04601A70BF
:10B6400003685A1C026019705DF8044B704700BF14
:10B65000036810B40A0A5C1C04601A7003685A1C60
:10B66000026019705DF8044B704700BF03685A1CF4
:10B67000026010B4197003680A0A5C1C04601A7036
:10B6800003680A0C5C1C04601A700368090E5A1CDB
:10B69000026019705DF8044B704700BF03685A1CC4
:10B6A000026019700368090A5A1C02601970704719
:10B6B00070B544880546C4F30B04224608460E467E
:10B6C00000213CF0DDF82B69094A934202D3094A74
:10B6D000934205D35BB121463046BDE87040184720
:10B6E000224630461946BDE870403CF063B870BD54
:10B6F000F00600083808000838B5064C064DAC4284
:10B7000006D2616820461434FFF7D2FFAC42F8D36A
:10B7100038BD00BFA0010008F0060008084B094929
:10B720008B4203D309E014338B4206D21A88C2F34A
:10B730000B029042F7D11846704700231846704715
:10B74000A0010008F00600082DE9F84FDFF8B082EC
:10B7500098F8003003B1FEE7A64EB368012288F8DE
:10B76000002013B11A689B885383A34B012204461F
:10B770001A708B46706840F2E93302E0002B00F04B
:10B780007C810289013B12F0020F9BB2F6D00023AC
:10B79000838140F2E93302E0002B00F06E810289E0
:10B7A000013B12F0010F9BB2F6D0838940F2E933DE
:10B7B00002E0002B00F075810289013B12F0020FBC
:10B7C0009BB2F6D00023838140F2E93302E0002BE4
:10B7D00000F067810289013B12F0010F9BB2F6D0A5
:10B7E000838940F2E93302E0002B00F056810289A0
:10B7F000013B12F0020F9BB2F6D00923838140F285
:10B80000E93302E0002B00F048810289013B12F08D
:10B81000010F9BB2F6D0838940F2E93302E0002B9E
:10B8200000F037810289013B12F0020F9BB2F6D083
:10B83000A4B2848140F2E93302E0002B00F02981B8
:10B840000289013B12F0010F9BB2F6D083896B4F46
:10B850000BF1FF3B00254FF00A0A4FF00B0940F2B5
:10B86000E93302E0002B00F0E5800289013B12F091
:10B87000020F9BB2F6D0A0F80CA040F2E93302E030
:10B88000002B00F0D7800289013B12F0010F9BB220
:10B89000F6D0838940F2E93302E0002B00F0D68035
:10B8A0000289013B12F0020F9BB2F6D0ABB283814A
:10B8B00040F2E93302E0002B00F0C8800289013B2E
:10B8C00012F0010F9BB2F6D083891BF8014F40F2B2
:10B8D000E93302E0002B00F0B1800289013B12F055
:10B8E000020F9BB2F6D0A0F80C9040F2E93302E0D0
:10B8F000002B00F0A3800289013B12F0010F9BB2E4
:10B90000F6D0838940F2E93302E0002B00F09A8000
:10B910000289013B12F0020F9BB2F6D0A4B28481DF
:10B9200040F2E93302E0002B00F08C800289013BF9
:10B9300012F0010F9BB2F6D083893B6833B11A68CD
:10B940009B8851690B4214BF538313830135362DF5
:10B9500085D140F2E93302E0002B00F096800289A5
:10B96000013B12F0020F9BB2F6D00823838140F214
:10B97000E93302E0002B00F088800289013B12F0DD
:10B98000010F9BB2F6D0838940F2E93301E0002B2E
:10B9900077D00289013B12F0020F9BB2F7D0A023AF
:10B9A000838140F2E93301E0002B6AD00289013B38
:10B9B00012F0010F9BB2F7D08389A025002440F23A
:10B9C000E93301E0002B45D00289013B12F0020F60
:10B9D0009BB2F7D0858140F2E93301E0002B39D0EA
:10B9E0000289013B12F0010F9BB2F7D0838940F22C
:10B9F000E93308E0B4840020566200200C85002062
:10BA00005562002053B30289013B12F0020F9BB232
:10BA1000F8D0848140F2E93300E0FBB10289013BB8
:10BA200012F0010F9BB2F8D08089C0B283061AD5FC
:10BA30007068C4E712F04CFB70682BE712F048FB0B
:10BA400070685FE712F044FB706876E712F040FB25
:10BA500070683AE712F03CFB7068C8E712F038FBF8
:10BA6000C0B28306E4D4B36813B11A689B88138309
:10BA7000002388F80030BDE8F88F12F029FB7068C9
:10BA800094E612F025FB706897E712F021FB7068CE
:10BA90007AE712F01DFB7068D9E612F019FB7068A6
:10BAA000BAE612F015FB70689BE600BF30B5204D7A
:10BAB00083B06B6840F2E93200E062B31C89013A5E
:10BAC00014F0020F92B2F8D080B2988140F2E932BD
:10BAD00000E002B31889013A10F0010F92B2F8D0D9
:10BAE0009A8940F2E93200E0E2B11889013A10F097
:10BAF000020F92B2F8D089B2998140F2E93200E0A7
:10BB000082B11989013A11F0010F92B2F8D09889E7
:10BB1000C0B203B030BD1846019112F0D9FA6B687B
:10BB20000199DEE7184612F0D3FAC0B2F1E700BF80
:10BB3000B484002008B540F2E93300E0A3B10289E3
:10BB4000013B12F0020F9BB2F8D089B2818140F222
:10BB5000E93300E043B10289013B12F0010F9BB2CF
:10BB6000F8D08089C0B208BD12F0B2FAC0B208BDE8
:10BB70002DE9F84FDFF8BCB3DBF8083013B11A68D1
:10BB80009B885383DBF8040040F2E93302E0002B8A
:10BB900000F089820289013B12F0020F9BB2F6D0BD
:10BBA0000523838140F2E93302E0002B00F07B8221
:10BBB0000289013B12F0010F9BB2F6D0838940F25B
:10BBC000E93302E0002B00F069820289013B12F0A8
:10BBD000020F9BB2F6D00023838140F2E93302E0EA
:10BBE000002B00F05B820289013B12F0010F9BB237
:10BBF000F6D0838940F2E93302E0002B00F067823F
:10BC00000289013B12F0020F9BB2F6D0062383811A
:10BC100040F2E93302E0002B00F059820289013B37
:10BC200012F0010F9BB2F6D0838940F2E93302E0B3
:10BC3000002B00F047820289013B12F0020F9BB2F9
:10BC4000F6D00023838140F2E93302E0002B00F0BC
:10BC500039820289013B12F0010F9BB2F6D0838931
:10BC6000B14BDC7E40F2E93344F0010402E0002BEA
:10BC700000F023820289013B12F0020F9BB2F6D042
:10BC80000423838140F2E93302E0002B00F01582A7
:10BC90000289013B12F0010F9BB2F6D0838940F27A
:10BCA000E93302E0002B00F003820289013B12F02D
:10BCB000020F9BB2F6D0A4B2848140F2E93302E0D5
:10BCC000002B00F0F5810289013B12F0010F9BB2BD
:10BCD000F6D08389954E3388002B49D0DFF85892EF
:10BCE000DFF858824F464FF0200A072518F8014F19
:10BCF000FF2C40F2E93303D17BE1002B00F0A78158
:10BD00000189013B11F0020F9BB2F6D0858140F210
:10BD1000E93302E0002B00F09A810189013B11F028
:10BD2000010F9BB2F6D0838940F2E93302E0002B89
:10BD300000F088810189013B11F0020F9BB2F6D01F
:10BD4000A4B2848140F2E93302E0002B00F07A8152
:10BD50000189013B11F0010F9BB2F6D0838998F85D
:10BD6000003007F8013B3188A7EB09039942BDDC9D
:10BD700040F2E93302E0002B00F0BB810289013B75
:10BD800012F0020F9BB2F6D00723838140F2E93311
:10BD900002E0002B00F0AD810289013B12F0010F9F
:10BDA0009BB2F6D0838940F2E93302E0002B00F029
:10BDB0009B810289013B12F0020F9BB2F6D0FF2358
:10BDC000838140F2E93302E0002B00F08D8102898B
:10BDD000013B12F0010F9BB2F6D08389524BDC7EFF
:10BDE00040F2E93302E0002B00F079810289013B47
:10BDF00012F0020F9BB2F6D00423838140F2E933A4
:10BE000002E0002B00F06B810289013B12F0010F70
:10BE10009BB2F6D0838940F2E93302E0002B00F0B8
:10BE20005B810289013B12F0020F9BB2F6D0A4B2F3
:10BE3000848140F2E93302E0002B00F04D81028959
:10BE4000013B12F0010F9BB2F6D083893388002B9F
:10BE500000F0C680364D00244FF0FF08072703E0AE
:10BE60000134A34240F3BC8015F8012BFF2AF7D11F
:10BE70004FEA2429DBF8040040F2E93302E0002B0A
:10BE800000F007810289013B12F0020F9BB2F6D04D
:10BE90000523838140F2E93302E0002B00F0F980B2
:10BEA0000289013B12F0010F9BB2F6D0838940F268
:10BEB000E93302E0002B00F0E7800289013B12F039
:10BEC000020F9BB2F6D01FFA89F9A0F80C9040F24D
:10BED000E93302E0002B00F0D7800289013B12F029
:10BEE000010F9BB2F6D083895FFA84F940F2E933FF
:10BEF00002E0002B00F0C3800289013B12F0020F28
:10BF00009BB2F6D00623838140F2E93302E0002B96
:10BF100000F0B5800289013B12F0010F9BB2F6D010
:10BF2000838940F2E9330EE020270020B40000208E
:10BF3000504E0020B48400203C2700204F4E0020AB
:10BF4000002B00F097800289013B12F0020F9BB298
:10BF5000F6D01FFA89F9A0F80C9040F2E93302E01C
:10BF6000002B00F087800289013B12F0010F9BB289
:10BF7000F6D0838940F2E93301E0002B75D00289C5
:10BF8000013B12F0020F9BB2F7D0878140F2E933F8
:10BF900001E0002B69D00289013B12F0010F9BB236
:10BFA000F7D0838940F2E93301E0002B59D00289B0
:10BFB000013B12F0020F9BB2F7D0A0F80C8040F2C8
:10BFC000E93301E0002B4CD00289013B12F0010F54
:10BFD0009BB2F7D0838933880134A3423FF744AF43
:10BFE000DBF8083013B11A689B881383BDE8F88F1B
:10BFF00093B30189013B11F0020F9BB2F8D0858108
:10C0000040F2E93300E03BB30189013B11F0010F3D
:10C010009BB2F8D0838940F2E93300E093B1018903
:10C02000013B11F0020F9BB2F8D0A0F80CA040F237
:10C03000E93300E033B10189013B11F0010F9BB2FC
:10C04000F8D08BE612F044F8DBF8040087E612F033
:10C050003FF8DBF8040067E612F03AF8DBF804007A
:10C06000D9E712F035F83388FAE612F031F8DBF848
:10C07000040097E712F02CF8DBF804007AE712F0DE
:10C0800027F8DBF804004CE712F022F8DBF8040094
:10C090002AE712F01DF8DBF8040008E712F018F8A0
:10C0A000DBF80400A6E512F013F8DBF8040086E5DF
:10C0B00012F00EF8DBF804000CE612F009F8DBF8D9
:10C0C0000400ECE512F004F8DBF80400C8E511F018
:10C0D000FFFFDBF80400A8E511F0FAFFB6E611F067
:10C0E000F7FFDBF8040096E611F0F2FFDBF804003E
:10C0F00074E611F0EDFFDBF8040054E62DE9F041A1
:10C100009C4CA36813B11A68998851839A4A606855
:10C110001278012A00F0AC81C0F06481022A00F09C
:10C120005381964D2A7812F0400F0CBF4FF4C37222
:10C130004FF4F072924E328013B11A689B88538389
:10C1400010274FF0010840F2E93302E0002B00F025
:10C1500041810289013B12F0020F9BB2F6D0BBB2C3
:10C16000838140F2E93302E0002B00F03381028941
:10C17000013B12F0010F9BB2F6D0838940F2E93304
:10C1800002E0002B00F02A810289013B12F0020F2D
:10C190009BB2F6D0A0F80C8040F2E93302E0002B0D
:10C1A00000F01C810289013B12F0010F9BB2F6D016
:10C1B00083890137202FC6D1A3681BB11A689B88D9
:10C1C000138353832D7840F2E93302E0002B00F013
:10C1D00058810289013B12F0020F9BB2F6D0002376
:10C1E000838140F2E93302E0002B00F04A810289AA
:10C1F000013B12F0010F9BB2F6D0838940F2E93384
:10C2000002E0002B00F041810289013B12F0020F95
:10C210009BB2F6D0ADB2858140F2E93302E0002B4B
:10C2200000F033810289013B12F0010F9BB2F6D07E
:10C230008389544A40F2E933157802E0002B00F07C
:10C2400028810289013B12F0020F9BB2F6D0022333
:10C25000838140F2E93302E0002B00F01A81028969
:10C26000013B12F0010F9BB2F6D0838940F2E93313
:10C2700002E0002B00F011810289013B12F0020F55
:10C280009BB2F6D0ADB2858140F2E93302E0002BDB
:10C2900000F003810289013B12F0010F9BB2F6D03E
:10C2A0008389394A40F2E933157802E0002B00F027
:10C2B000F8800289013B12F0020F9BB2F6D00323F3
:10C2C000838140F2E93302E0002B00F0EA8002892A
:10C2D000013B12F0010F9BB2F6D0838940F2E933A3
:10C2E00002E0002B00F0E1800289013B12F0020F16
:10C2F0009BB2F6D0ADB2858140F2E93302E0002B6B
:10C3000000F0D3800289013B12F0010F9BB2F6D0FE
:10C3100083891E4BDD7E40F2E93345F0040502E0DF
:10C32000002B00F0C6800289013B12F0020F9BB285
:10C33000F6D00423838140F2E93302E0002B00F0C1
:10C34000B8800289013B12F0010F9BB2F6D08389BD
:10C3500040F2E93302E0002B00F090800289013BBB
:10C3600012F0020F9BB2F6D0ADB2858140F2E933F4
:10C3700010E000BFB484002000850020A802002047
:10C38000B400002007850020088500202027002019
:10C39000002B73D00289013B12F0010F9BB2F7D042
:10C3A0008389A36813B11A689B881383474C32882A
:10C3B000474800213BF064FA23781BB1FFF7D8FB14
:10C3C00000232370BDE8F081424D08222A704FF40B
:10C3D000C372AFE611F07CFE6068CFE611F078FE24
:10C3E0006068E6E640F2E93301E0002B69D002899B
:10C3F000013B12F0020F9BB2F7D0A023838140F2E1
:10C40000E93301E0002B5CD00289013B12F0010FFF
:10C410009BB2F7D0838940F2E93301E0002B4CD086
:10C420000289013B12F0020F9BB2F7D000238381F7
:10C4300040F2E93301E0002B3FD00289013B12F0CA
:10C44000010F9BB2F7D08389D8B200F00603022B0C
:10C45000204D08D000F00503012B04D14822D4E977
:10C4600001032A7007E00822D4E901032A70AEE72D
:10C47000184D48222A704FF4F0725BE611F028FE46
:10C480008FE711F025FE6068B8E611F021FE6068C4
:10C49000CFE611F01DFE6068E8E611F019FE606855
:10C4A000FFE611F015FE606818E711F011FE6068F4
:10C4B0002FE711F00DFE60684AE711F009FEC0B2E7
:10C4C000C3E711F005FE6068A5E700BF000000208B
:10C4D0003C270020A80200202DE9F041574CA3681A
:10C4E00013B11A689B885383606840F2E93301E016
:10C4F000002B4BD00289013B12F0020F9BB2F7D008
:10C500008023838140F2E93301E0002B3ED0028991
:10C51000013B12F0010F9BB2F7D0838940F2E9335F
:10C5200001E0002B2ED00289013B12F0020F9BB2DA
:10C53000F7D00023838140F2E93300E013B302898E
:10C54000013B12F0010F9BB2F8D08089C0B2A36802
:10C5500013B11A6899881183394D3A4E2A78376891
:10C5600082420CD1384A12783AB9DFF8E880D8F81C
:10C57000FC21BA1AB2F57A7F0CD8BDE8F081BDE88B
:10C58000F041BBE511F0A4FDC0B2E0E711F0A0FD61
:10C590006068C3E713B11A689B885383A021606861
:10C5A000FFF7C8FA00216068FFF7C4FAA36813B167
:10C5B0001A689B881383254C2378182B0FD12B786E
:10C5C000234A03F04003002B00F007010CBF4FF09B
:10C5D0000D0C4FF0100C13805180A2F806C04107DB
:10C5E00006D50023C8F80032C8F8FC71BDE8F08118
:10C5F00000F00500012819D00028F5D12B785B0642
:10C60000F2D5D8F800223368A2B19B1A642BEBD97B
:10C61000FFF774FD2378182BE6D1B8F804320C4AE2
:10C6200001339BB2A8F804329380DDE72B785A06D9
:10C63000E7D5D9E7C8F80032D6E700BFB4840020B8
:10C64000A80200204085002000850020F5840020FD
:10C65000F8840020202700200E4B10B41C888CB1D9
:10C660000D4B0E4A1878117F88420FD11C441C32A2
:10C67000013305E013F8011B12F8010F884205D1C0
:10C68000A342F7D101205DF8044B704700205DF80C
:10C69000044B7047B4000020504E0020202700209B
:10C6A0001378C3B130B41E240B4D14FB010129448F
:10C6B000801A84181D2C07DC01F8013B12F8013F99
:10C6C000002BF6D130BC704712F8013F0131002B2E
:10C6D000EFD130BC70477047504E002070B5264DEA
:10C6E000C1F10301AB6841EA8006F6B213B11A68E2
:10C6F0009B885383B6B21024686840F2E93301E0A6
:10C70000002B31D00289013B12F0020F9BB2F7D00F
:10C71000A3B2838140F2E93300E02BB30289013BED
:10C7200012F0010F9BB2F8D0838940F2E93300E0A8
:10C73000F3B10289013B12F0020F9BB2F8D086815F
:10C7400040F2E93300E09BB10289013B12F0010F96
:10C750009BB2F8D083890134202CCDD1AB6813B1C2
:10C760001A689B88138370BD11F0B2FC6868DCE71F
:10C7700011F0AEFCEFE700BFB484002038B5264BC3
:10C78000DD7E00283ED105F0F705244CDD76A36858
:10C7900013B11A689B885383606840F2E93301E063
:10C7A000002B35D00289013B12F0020F9BB2F7D06B
:10C7B0000423838140F2E93300E04BB30289013B5B
:10C7C00012F0010F9BB2F8D0838940F2E93300E008
:10C7D000DBB10289013B12F0020F9BB2F8D0ADB27F
:10C7E000858140F2E93300E07BB10289013B12F020
:10C7F000010F9BB2F8D08389A36813B11A689B8894
:10C80000138338BD45F00805BFE711F061FCF3E77D
:10C8100011F05EFC6068D8E720270020B484002077
:10C82000144B984223D003F5806398421FD00388AD
:10C8300023F040031B041B0C0380038823F0380300
:10C840001B041B0C59B141F48071002991FAA1F12C
:10C85000B1FA81F108BF4FF0FF310139C900194326
:10C8600089B20180038843F0400303807047490880
:10C87000DDE700BF00380040F0B587B00023604A14
:10C8800000930193136843F48033136003E0009B2B
:10C89000B3F5A04F09D0136803F400330193009B54
:10C8A00001330093019B002BF1D0554B1B6813F40F
:10C8B000003318BF01230193019B012B63D0514D1D
:10C8C0004F4B514AEA605149586F514A0860AA607B
:10C8D0005E6B504C504F514A514826F080065E63C3
:10C8E0005E6F46F080765E67196B0C431C63596B74
:10C8F0005963196C39431964596C06AC0A4348F200
:10C90000FF715A6444F8101D0123002621468DF85A
:10C910000F304FF6FF778DF80C608DF80D608DF8B5
:10C920000E6026F0DBF821463E48029726F0D6F846
:10C9300021463D48029726F0D1F821463B4826F093
:10C94000CDF821463A4826F0C9F8204626F0CAF923
:10C95000384B394C1B68029A38483949A4FB0343C9
:10C960009B09A0FB0202013B920CB3F1807F0A609D
:10C9700007D2344AF0200721536085F823009660DF
:10C98000116007B0F0BD1E4B2F4C1A6C2F4942F0BE
:10C9900080521A64206840F44040D1E90152C968CD
:10C9A00020609868986098689860120642EA85123C
:10C9B000986842F48002490842F00802013942EACC
:10C9C000014240F4805098605A601A6842F08072C8
:10C9D0001A601A689201FCD51D49094A40F202709A
:10C9E0000860996821F003019960996841F002019B
:10C9F0009960936803F00C03082BFAD15FE700BF3E
:10CA00000038024000ED00E00005FA0594AF002078
:10CA1000000000081F906700FFC9FE36335F070063
:10CA2000000002400004024000080240000C0240E6
:10CA300000100240B0A20020D34D621083DE1B43E1
:10CA40004485002010E000E000700040000000205D
:10CA5000003C0240074A08B51168074B994208D1CB
:10CA6000064B00201968106081F308885B689847BE
:10CA7000FEE708BDD4C20020EFBEADDE0000FF1F00
:10CA800008B5054B1B6803B19847044B044A1A606C
:10CA900072B63AF061FE00BFB8410020D4C2002057
:10CAA000EFBEADDE2DE9F04F054690F8650085B08C
:10CAB000002840F01A8202AF5B4B686993F8063297
:10CAC00005F11006002B00F0B380584B984200F09F
:10CAD000FF8103F58063984200F0FA81038823F018
:10CAE00040031B041B0C0380038823F038031B0442
:10CAF0001B0C382213430380038843F04003038058
:10CB000095F85F30032B00F28D8095F86240012C80
:10CB100000F01283A4F10204B4FA84F46409AB694E
:10CB200013B11A689B88538340F2E93304E0013B58
:10CB30009BB2002B00F0488402899207F7D51A2394
:10CB4000838140F2E93304E0013B9BB2002B00F00B
:10CB50003B840289D107F7D5838940F2E93304E0A9
:10CB6000013B9BB2002B00F02B8402899207F7D582
:10CB7000848140F2E93304E0013B9BB2002B00F0DA
:10CB80001F840289D107F7D58389AB6913B11A686D
:10CB90009B88138301200DF0ADF86969234B9942FE
:10CBA00000F0B78203F58063994200F0B2820B88EF
:10CBB00023F040031B041B0C0B800B8823F038036D
:10CBC0001B041B0C082213430B800B8843F040030B
:10CBD0000B803A4630460623432111F0DBFA002849
:10CBE00000F0DE819DF80A609DF80B309DF808404A
:10CBF0009DF809109DF80C009DF80D2043EA0623CE
:10CC00001BB2A5F852305BB241EA042142EA00228D
:10CC10000133A5F85010A5F8542000F0C78105B0E5
:10CC2000BDE8F08F00247AE720270020003800407C
:10CC3000CF4B984200F0B78303F58063984200F031
:10CC4000B283038823F040031B041B0C038003887A
:10CC500023F038031B041B0C4FF4807242F48072E3
:10CC6000002A92FAA2F2B2FA82F208BF4FF0FF3223
:10CC7000013A43EAC2039BB203800388BD4CDFF84C
:10CC800010A3DFF810B343F04003038080226B2130
:10CC9000304611F039FA9623DFF8FCC2DFF8FCE2E7
:10CCA0000093B54B5B68C3F30803002B40F04A8345
:10CCB000EFF31183002B40F045832068DCF8082057
:10CCC00023689842F9D1DEF800309A42F5D8DAF8B4
:10CCD00000804FF47A7101FB08F39B1AB3FBF8F361
:10CCE00001FB00304FF47A78A34B5B68C3F3080371
:10CCF000002B40F0D182EFF31183002B40F0CC8267
:10CD00002368DCF8081022689342F9D1DEF800208D
:10CD10009142F5D8DAF8009008FB09F2521AB2FBFA
:10CD2000F9F208FB03231B1AB3F57A7FDCD3009BCF
:10CD3000013B0093B5D103226821304611F0E4F99C
:10CD4000DFF850B2DFF850C2DFF850E296230093CC
:10CD5000894B5B68C3F30803002B40F0CF82EFF3ED
:10CD60001183002B40F0CA822068DCF80820236879
:10CD70009842F9D1DEF800309A42F5D8DAF800800E
:10CD80004FF47A7101FB08F39B1AB3FBF8F301FB34
:10CD900000304FF47A78784B5B68C3F30803002BBC
:10CDA00040F05882EFF31183002B40F05382236848
:10CDB000DCF8081022689342F9D1DEF80020914295
:10CDC000F5D8DAF8009008FB09F2521AB2FBF9F232
:10CDD00008FB03231B1AB3F57A7FDCD3009B013BCE
:10CDE0000093B5D103226B21304611F08DF90F204D
:10CDF0000CF080FF10226A21304611F085F90F20D7
:10CE00000CF078FF009A6C21304611F07DF90F206C
:10CE10000CF070FF95F864201921304611F074F978
:10CE20000F200CF067FF18221B21304611F06CF91F
:10CE30000F200CF05FFF18221C21304611F064F91E
:10CE40000F200CF057FF10223721304611F05CF90B
:10CE50000F200CF04FFF01223821304611F054F919
:10CE60000F200CF047FF6A69414B9A4200F08E8216
:10CE700003F580639A4200F08982138823F040030F
:10CE80001B041B0C1380138823F038031B041B0C9A
:10CE9000042141F48071002991FAA1F1B1FA81F1E4
:10CEA00008BF4FF0FF31013943EAC1039BB2138041
:10CEB000138843F04003138001200CF01BFF2F4A1E
:10CEC0006869012382F80632294B98427FF401AE4B
:10CED000038823F040031B041B0C0380038823F00A
:10CEE00038031B041B0C302204E60BF001FD05F196
:10CEF0000C060446002800F019810068204900F162
:10CF00003F4303F57E039A0A01238A5C02F01F0166
:10CF1000520920278B40032A4FF00001A771E171CD
:10CF200000F09381042A00F08B81022A03D1154A74
:10CF3000516C0B435364A388029302AF002339461C
:10CF4000039325F0CBFD104BEB60314620462EF0CD
:10CF500077F8A388B3FA83F3C3F11F03012212FA0F
:10CF600003F33FF4A9AD09490A6813430B60A3E535
:10CF7000003800404085002000ED00E02027002020
:10CF800074C304080038024049890008003C01408D
:10CF9000448500203C85002010E000E0488500200A
:10CFA000B5F952305BB201337FF439AE95F95030A8
:10CFB00001337FF434AE0A23C84CDFF838A3C84FDE
:10CFC000C84DC94E01932DF097FD4FF4FA73DFF869
:10CFD00028E300934FF010087B68C3F30803002B8D
:10CFE00040F0EA80EFF31183002B40F0E5802068E9
:10CFF000AA6823689842FAD133689A42F7D8DAF8D7
:10D0000000C04FF47A7101FB0CF39B1AB3FBFCF3E5
:10D0100001FB00304FF47A7C4FF001097B68C3F3C9
:10D020000803002B40F0A980EFF31183002B40F0A0
:10D03000A4802368A96822689342FAD13268914299
:10D04000F7D8DAF800200CFB02FBABEB0101B1FBD7
:10D05000F2F10CFB03131B1AB3F57A7FDED3009BAE
:10D06000013B0093B8D107202DF0A2FB4FF47A7357
:10D07000DFF884E200934FF010087B68C3F30803E5
:10D08000002B40F0BB80EFF31183002B40F0B68003
:10D090002068AA6823689842FAD133689A42F7D880
:10D0A000DAF800C04FF47A7101FB0CF39B1AB3FB62
:10D0B000FCF301FB00304FF47A7C4FF001097B68F0
:10D0C000C3F30803002B39D1EFF31183002B35D1C3
:10D0D0002368A96822689342FAD132689142F7D84E
:10D0E000DAF800200CFB02FBABEB0101B1FBF2F123
:10D0F0000CFB03131B1AB3F57A7FE0D3009B013BB3
:10D100000093BAD1019B013B01937FF45CAFFFF721
:10D11000B7FC0B8823F040031B041B0C0B800B880F
:10D1200023F038031B041B0C00224CE56F4BEB6013
:10D1300031462DF085FFBEE40724F0E4EFF31181C2
:10D1400088F31288D5F808B02B68DB0344BFCEF80B
:10D150000090D5F808B02368DEF80020C9B281F34A
:10D160001188DAF8001013440CFB01F2A2EB0B0259
:10D17000B2FBF1F20CFB0323BCE7EFF3118188F360
:10D180001288D5F808B02B68DB0344BFCEF80090B6
:10D19000D5F808B02368DEF80020C9B281F3118801
:10D1A000DAF8001013440CFB01F2A2EB0B02B2FB05
:10D1B000F1F20CFB03234EE7EFF3118388F312889F
:10D1C000D5F808C02A68D20304D50122CEF8002081
:10D1D000D5F808C02068DEF80090DBB283F3118830
:10D1E000DAF800104FF47A72484402FB01F3A3EB23
:10D1F0000C03B3FBF1F302FB00300BE7EFF31183F9
:10D2000088F31288D5F808C02A68D20304D5012211
:10D21000CEF80020D5F808C02068DEF80090DBB218
:10D2200083F31188DAF800104FF47A72484402FB55
:10D2300001F3A3EB0C03B3FBF1F302FB00303AE77D
:10D240002B4A116B0B43136375E6294A116C0B4390
:10D25000136470E6EFF31181102383F31288DCF876
:10D260000890DCF80030DB0304D50123CBF8003054
:10D27000DCF808902368DBF80020C9B281F311883C
:10D28000DAF80010134408FB01F2A2EB0902B2FB2A
:10D29000F1F208FB03239DE5EFF31181102383F3E3
:10D2A0001288DCF80890DCF80030DB0304D5012399
:10D2B000CBF80030DCF808902368DBF80020C9B216
:10D2C00081F31188DAF80010134408FB01F2A2EB95
:10D2D0000902B2FBF1F208FB032324E5408500209C
:10D2E00000ED00E010E000E04885002049890008DA
:10D2F00000380240448500203C850020EFF3118275
:10D30000102383F31288DCF80880DCF80030D9039E
:10D3100004D50123CBF80030DCF808802368DBF863
:10D320000000D2B282F31188DAF800104FF47A725A
:10D33000184402FB01F3A3EB0803B3FBF1F302FB78
:10D34000003026E5EFF31182102383F31288DCF816
:10D350000880DCF80030D90304D50123CBF8003075
:10D36000DCF808802368DBF80000D2B282F3118871
:10D37000DAF800104FF47A72184402FB01F3A3EBC1
:10D380000803B3FBF1F302FB0030ABE4138823F096
:10D3900040031B041B0C1380138823F038031B0469
:10D3A0001B0C022175E5038823F040031B041B0CB2
:10D3B0000380038823F038031B041B0C80224DE4F8
:10D3C00010F086FEFFF7E1BB10F082FE6869FFF700
:10D3D000C4BB00BF08B5034B1B6803B1984772B6C6
:10D3E0003AF0BAF9B8410020074A002302E00133BD
:10D3F000102B07D05168814202F12002F7D1581C4E
:10D40000C0B2704700207047642400200138F0B596
:10D4100040013C4CDFF820C125583B4FDCF8306020
:10D42000BD420CBF4FF400154FF4800527182E4362
:10D430007D68CCF83060354EF960B54283B07B61D1
:10D4400051D0334B9D424ED0A3F57A739D4236D0D6
:10D4500003F580639D4232D0A3F57A739D4246D096
:10D4600003F580639D4242D0A3F57A739D4240D07C
:10D4700003F580639D423CD0A3F57A739D4234D07E
:10D4800003F580639D4230D0A3F57A739D4232D07C
:10D4900003F580639D422ED0A3F57A739D422CD074
:10D4A00003F580639D4228D0A3F57A739D4226D070
:10D4B0001849194B8D420CBF1D46002500E0174D41
:10D4C00004449209667CE5610021012301A88DF8DE
:10D4D00004608DF805208DF806108DF807302DF0CA
:10D4E000A1FC03B0F0BD0E4DEAE70E4DE8E70E4D8E
:10D4F000E6E70E4DE4E70E4DE2E70E4DE0E7064DA0
:10D50000DEE700BF6424002000600240106002409B
:10D5100010640240B86402400080002800880010B7
:10D520002080001020800020008020100080001843
:10D530000088002000802020003802400138F0B42C
:10D5400044010948094D0359094F2E6B2044BB4241
:10D550000CBF4FF400134FF4800333432B63017669
:10D560004276F0BC704700BF6424002000380240BF
:10D57000006002402DE9F04F534C54F8204083B036
:10D58000002C00F09C80656E002D00F09A8098467B
:10D59000174604F16A034D4A064628692260636112
:10D5A00004F1EA028023A261E3604FF480726B68A9
:10D5B000A1602261E365A24668B1FFF715FF721C06
:10D5C000D2B20C21FFF7BAFFE36DA9682A69A26302
:10D5D00004332164A365E868A0B1FFF705FF721C5E
:10D5E0008146D2B20B21FFF7A9FF2346EA7F3849D3
:10D5F0004846FFF70BFFD5E90212E36D616404337F
:10D600006365E26394F869000BF072F9814694F85F
:10D6100068000BF06DF98346287F00284CD118F084
:10D62000080F36D1BA070DD5B9F1000F0AD00B2279
:10D63000731C89F8062089F8073048466A7F222142
:10D640000AF0F0FFFB0715D4236C7BB995F8202076
:10D65000A97F8DF8063001A8930901228DF80530C5
:10D660008DF804108DF807202DF0DCFB504603B038
:10D67000BDE8F08FBBF1000FE6D0701C0C238BF8D7
:10D6800007008BF8063058466A7F22210AF0CAFF4D
:10D69000DAE7B9F1000F05D0701C0B2389F80700F9
:10D6A00089F8063018F0100F484614BF02211221E5
:10D6B0006A7F0AF0B7FFC7E72DF0D6FBAFE7A246B7
:10D6C000D4E7AA46D2E700BF9C360020EC900408BD
:10D6D000598900080348D0F8EC3113B100F5F07017
:10D6E00018477047642400200348D0F8CC3113B1A8
:10D6F00000F5E07018477047642400200348D0F814
:10D70000AC3113B100F5D070184770476424002085
:10D710000348D0F88C3113B100F5C070184770473A
:10D72000642400200348D0F86C3113B100F5B070C8
:10D7300018477047642400200348D0F84C3113B1D7
:10D7400000F5A07018477047642400200348D0F803
:10D750002C3113B100F590701847704764240020F5
:10D760000348D0F80C3113B100F5807018477047AA
:10D77000642400200348D0F8EC300BB1E0301847A7
:10D78000704700BF642400200348D0F8CC300BB1B0
:10D79000C0301847704700BF642400200348D0F809
:10D7A000AC300BB1A0301847704700BF6424002094
:10D7B0000348D0F88C300BB180301847704700BF59
:10D7C000642400200248C36E0BB1603018477047D4
:10D7D000642400200248C36C0BB1403018477047E6
:10D7E000642400200248C36A0BB1203018477047F8
:10D7F000642400200248C36803B11847704700BF83
:10D8000064240020F8B584894FF6FF764FF47A74CB
:10D8100033B319B30F78013101E0B44218D0058950
:10D82000013CAD07A4B2F8D5BCB284814FF47A7440
:10D8300002E0BCB2B4420BD00589ED0704F1FF371A
:10D84000F7D58589ADB20AB115700132013BDFE72A
:10D8500010F03EFC003018BF0120F8BDFF27DEE7C6
:10D860000120F8BD2DE9F84F2D4A2E4E01231370EB
:10D87000FEF732FEB6F808222B4BDFF8B8E0B3F81B
:10D88000008002F1640C1FFA8CFC00234FF0050BA2
:10D890004FF0060A4FF0070901E062453CD0B4188A
:10D8A0001EF80200217F814202F1010503F105010A
:10D8B00010D07718F1182077140A81F80CB281F88B
:10D8C0000EA281F80F2281F8109281F80D420633E2
:10D8D00087F80C02AAB24245DFD30022A6F808223C
:10D8E00023B90F4A00231370BDE8F88F0F4CA268CC
:10D8F00012B1116892884A8300220D496068FFF7CF
:10D9000081FFA368002BECD01A689B881383044A1C
:10D9100000231370BDE8F88FA6F80822E0E700BFE7
:10D920005562002020270020B4000020B48400208D
:10D930002C290020504E0020F8B5624D04012F190B
:10D940000646387A2DF090FA3B7A03F01F015B0906
:10D950000122032B02FA01F26DD0042B66D0022BB8
:10D960005CD02B19013618790AF0C2FFF6B20746CF
:10D9700010B11223C67183712B1958790AF0B8FFC0
:10D9800010B11323C67183712B1998790AF0B0FF77
:10D9900010B11423C67183712E190A21F279384609
:10D9A0000AF040FE70790AF0A3FFF2790A210AF02A
:10D9B00039FEB0790AF09CFFF2790A210AF032FEB2
:10D9C0002B59414A934246D0404A93424ED0404A56
:10D9D000934256D03F4A93425ED03F4A93422FD063
:10D9E0003E4A934263D02B191B7BE3B901200222EC
:10D9F0002B59198801F4415141F445710A430243FE
:10DA00001A809A8B22F400621204120C07219A8366
:10DA100019821A8842F040021A80F8BD304B596AC8
:10DA20000A435A629DE700200246E1E72C4B196940
:10DA30000A431A6195E72A4B196A0A431A6290E76A
:10DA400002F568424FF48010536A43F48013536226
:10DA500025F08AF8C7E702F584324FF48050536A04
:10DA600043F48053536225F07FF8BCE702F500329F
:10DA70004FF48040136A43F48043136225F07CF82E
:10DA8000B1E702F5FE324FF40040136A43F400435D
:10DA9000136225F071F8A6E702F582324FF40050C8
:10DAA000536A43F40053536225F05EF89BE702F596
:10DAB00064424FF40010536A43F40013536225F09C
:10DAC00053F890E7C4840020003001400038004043
:10DAD000003C00400034014000500140005401402F
:10DAE00000380240431C00F014812DE9F04F4FEA4A
:10DAF000C00808EB00039B00DFF8009359F803A06F
:10DB000087B009EB0304BAF1000F00F0FF80143373
:10DB100009EB03010022DAF8047049F80320C1E997
:10DB20000122CA60D4E9025B034601330190DBB2F3
:10DB3000002D00F008811522EB71AA719AF81800E7
:10DB4000BBF1000F00F0E68016228BF806208BF860
:10DB500007302DF089F9BB8823F440731B041B0C9C
:10DB6000BB8028460FF0BEFA58460FF0BBFA1121D1
:10DB700028460FF0DBF8112158460FF0D7F8092698
:10DB8000332405E0013C4FF00A0006D00CF0B2F857
:10DB9000284610F061F90028F4D028460FF09CFACE
:10DBA00005200CF0A7F828460FF09CFA05200CF091
:10DBB000A1F8013EE4D128460FF08EFA05200CF0C2
:10DBC00099F858460FF088FA05200CF093F828468B
:10DBD0000FF088FA05200CF08DF858460FF082FA05
:10DBE000019B08EB030409EB84042846E37C227CB8
:10DBF000002B0CBF122132210AF014FDE37C627C61
:10DC0000002B0CBF1221322158460AF00BFD714B3C
:10DC10009F4200F0B180704B9F4200F0C1806F4B7B
:10DC20009F4200F0B380BB886D4A6E4C23F4407372
:10DC30001B041B0CBB80019B98443B8809EB8809A3
:10DC400043F0010399F812103B80BD8802A8002917
:10DC500018BF144625F046F8049A6348B2FBF4F363
:10DC600025F03F05A0FB02122D04900C2D0C05435E
:10DC7000BD8039885D4C4FF496729BB202FB00F276
:10DC8000002BA4FB020221F0010108BF012392092D
:10DC9000090443F400430132090C39803A84BB8300
:10DCA0003A88534B42F001023A803A88134043F4D9
:10DCB00080634FF480423B803A813B8823F08003AD
:10DCC0001B041B0C3B809AF81A308DF80830002496
:10DCD00002A801258DF809408DF80A408DF80B50F7
:10DCE0002DF0A0F89DF80B209AF819308DF8083027
:10DCF0008DF809408DF80A40FAB95A09203203F02C
:10DD00001F033C4905FA03F341F8223007B0BDE890
:10DD1000F08F70472DF0A8F8BB8823F440731B04E4
:10DD20001B0CBB8028460FF0DDF958460FF0DAF9DE
:10DD3000112128460EF0FAFF21E702A82DF072F813
:10DD400007B0BDE8F08F9AF81800BBF1000F31D092
:10DD500016228BF807308BF806202DF085F8BB884B
:10DD600023F440731B041B0C2846BB800FF0BAF948
:10DD700058460FF0B7F9FEE61F4A136A43F4001342
:10DD800013624FF4001024F0F7FE4CE71A4A136AAE
:10DD900043F4000313624FF4000024F0EDFE42E769
:10DDA000154A136A43F4800313624FF4800024F091
:10DDB000E3FE38E72DF058F8BB8823F440731B04CA
:10DDC0001B0C5846BB800FF08DF958460FF08AF9AE
:10DDD000D5E600BF0054004000580040005C004001
:10DDE000009F2400804F120083DE1B43D34D62103E
:10DDF000F5FBFFFF00E100E000380240D4360020D0
:10DE0000F0B5C60033189B00244DEA585468A28A26
:10DE100083B092B20192019A2B4412F4706F1CBF2E
:10DE200001221A75019B13F4E06F07460CD1A38AF7
:10DE30003E4423F4706305EB86051B041B0C002293
:10DE4000A3826A7503B0F0BD238BA38823F480639B
:10DE50001B041B0CA380019B9B05E8D42388980519
:10DE6000E5D42388D9050DD52388DA05FCD4238889
:10DE700043F40073238023889B05FCD43846FFF7C6
:10DE800031FED4E7238843F400732380A38823F46E
:10DE900040731B041B0CA380C9E700BFD4360020CD
:10DEA000F0B583B0441C8DF8073001D0032802DDA3
:10DEB000002003B0F0BDC700274E3B1806EB8303DC
:10DEC0005C68002CF4D04900C9B299750125002185
:10DED000DA755D7699761D765D751975A1880DF1F7
:10DEE00007028905C3E9072212D42388DA050BD477
:10DEF0004FF4805501E0013D25D023889B05FAD4DD
:10DF0000238843F480732380A38843F44073A38061
:10DF1000074406EB87024FF4805401E0013C09D02E
:10DF2000537D002BFAD106EB8707387D80F0010086
:10DF300003B0F0BD094A138801339BB21380FFF789
:10DF4000D1FD2046B5E7054A138801339BB2138003
:10DF5000FFF7C8FD2846ACE7D436002090420020E9
:10DF60000220FAF731BF00BF022049E70120FAF78B
:10DF70002BBF00BF012043E70020FAF725BF00BFF9
:10DF800000203DE7044B187828B1044A1268520774
:10DF900044BF00201870704742320020002001402A
:10DFA00043680B4A23F0407323F4807343F4807377
:10DFB000436083681A4042F002028260C36A0139FA
:10DFC000C9B223F4700343EA0153C362704700BF30
:10DFD000FDF7FFC01D4B1B68022B30B432D81C4A22
:10DFE0001C4903EB43035B0098189B5A42888088C6
:10DFF0004B60C1E90202B3FBF2F21748174D184912
:10E00000184B194C00FB02F22A60D1F8882042F428
:10E010007002C1F888201A68002042F001021A60DC
:10E0200098601A6822F0847222F480321A605C6070
:10E030001A684FF0006422F480221A60D8608C6065
:10E0400030BC7047034A5368D268D4E7D8C2002076
:10E05000A09404080000002040420F00B0A200205D
:10E0600000ED00E00038024010300024D0E9092023
:10E07000101AB0FA80F04009704700BF0171704774
:10E0800003799B070AD5436A8269D154436A0169BF
:10E090000133B3FBF1F201FB12334362704700BF5F
:10E0A000037913F0010317D0D0E90731C26810B427
:10E0B0005B1A541E23400BD043694C1C5B5CB4FBC1
:10E0C000F2F102FB114202625DF8044BD8B27047D4
:10E0D00018465DF8044B704718467047037913F0F3
:10E0E000020308D0D0E909210369581E531A0340DE
:10E0F000DBB2C01A70471846704700BF037913F0AF
:10E10000010306D0D0E90731C268581A531E1840DF
:10E1100070471846704700BF10F8113C0133DBB25E
:10E120000A2B00F8113C07D9044A10F8131C0023ED
:10E1300022F8113000F8113C704700BFEC3F00207E
:10E14000F0B45D4E5D4832785D4B5E4DDC6B2D78F2
:10E150000132A0FB0270000900EB8000A2EB8000FE
:10E160001A683070914201EB04005C6811D293F898
:10E170004520002A4ED000F58030B0FBF5F08442F7
:10E180000BD2041B4FF4803292FBF5F2A21A9A6074
:10E190000AE0B0FBF5F0844244D34FF4803292FBA6
:10E1A000F5F2121B02449A6040F68C240025A2422C
:10E1B000C3E9001083F8455017D993F8402093F92C
:10E1C00042108A4256B241D0002093F9411083F8A0
:10E1D00043008A4247D00121002283F8426083F83D
:10E1E000441083F84020F0BC704793F84410002995
:10E1F000F9D0A2F2EF2040F2DA5188421AD893F80F
:10E2000040100B2916D803EB81000131C26083F85E
:10E210004010E8E7B0FBF5F08442BED2041BA21A1E
:10E220009A60C1E793F84520002AAAD1041BA21ADC
:10E230009A60B9E7244A002102F1300083F84410C3
:10E2400042F8041F8242FBD1F0BC7047111F08291D
:10E25000BAD893F84310182926D8013183F843100F
:10E2600093F94110B5E793F844100029B3D0FAB1FF
:10E270001649154C0FFA82FC084601EB4C0754F87E
:10E28000045F20F8025BB842F9D10B2A07DC104882
:10E2900001EB4C02002122F8021B9042FBD10D49F8
:10E2A0000A7801320A7096E783F84160314690E7B8
:10E2B00094460649EBE700BF8C2B0020CDCCCCCC9C
:10E2C000A4A1002060240020ACA10020EC3F00208D
:10E2D00004400020E03F002030B40E4D0E4B2A7861
:10E2E0000E4C0132A3FB02031B09E06B03EB83031B
:10E2F000A2EB83034FF6FF72914200F101002B70F5
:10E30000084408BF0123E06308BF84F8453030BCEF
:10E31000704700BF8C2B0020CDCCCCCCA4A100201A
:10E32000002800F03881B14B1A7CF0B4002A40F08C
:10E330009D801968002201280A6043D093F82810B4
:10E34000002941D19969002202280A603AD093F845
:10E350004010002961D1196B002203280A6031D0D6
:10E3600093F85810002940F09680996C00220428F8
:10E370000A6027D093F87010002940F00D81196EC3
:10E38000002205280A601DD093F88810002940F06B
:10E390003981996F002206280A6013D093F8A010E3
:10E3A000002940F05781D3F89010002207280A6016
:10E3B00008D093F8B810002940F0B980D3F8A830FD
:10E3C00000221A60F0BC7047DC69894DA10AA9429D
:10E3D00000F0B88140F2D580864DA94208D0864A27
:10E3E000914200F0AD814D3A914200F08D81FE22C4
:10E3F000EFF31181502585F31288804E676AA58A54
:10E4000002EB820206EBC202013745F001055762BA
:10E41000C9B2A58281F3118894E75C6B744DA10A9F
:10E42000A94200F0658140F23D81724DA94208D0B9
:10E43000714A914200F05A814D3A914200F0868132
:10E44000FE22EFF31181502585F312886B4E676A27
:10E45000A58A02EB820206EBC202013745F00105F4
:10E460005762C9B2A58281F3118874E75C6860497C
:10E47000A20A8A4200F058813CD95E498A4200F0E3
:10E48000558110318A4200F04B814D398A4200F0AB
:10E490003781FE2136E0DC6C554DA10AA94200F01F
:10E4A000578140F20881534DA94208D0524A914207
:10E4B00000F022814D3A914200F04C81FE22EFF3B0
:10E4C0001181502585F312884C4E676AA58A02EBAC
:10E4D000820206EBC202013745F001055762C9B25C
:10E4E000A58281F31188996C002204280A607FF4C8
:10E4F00041AF67E7B2F5801F00F0148101398A420D
:10E50000C7D10221EFF31182502585F312883B4ECB
:10E51000676AA58A01EB810106EBC101013745F06D
:10E5200001054F62D2B2A58282F3118801E7D3F8C8
:10E53000AC002F4C810AA14200F0248140F2CD8032
:10E540002C4CA14208D02C4A914200F01F814D3A38
:10E55000914200F01981FE22EFF31181502484F3DF
:10E560001288264D466A848A02EB820205EBC205B8
:10E57000013644F001046E62CAB2848282F31188CB
:10E580001CE7B1F5801F00F0DF801D4A91427FF447
:10E590002EAF02222CE770475C6E154DA10AA942EE
:10E5A00000F0DC8040F29080124DA94208D0124A5F
:10E5B000914200F0A7804D3A914200F0CD80FE22BA
:10E5C000EFF31181502585F312880C4E676AA58AF6
:10E5D00002EB820206EBC202013745F001055762E9
:10E5E000C9B2A58281F31188C9E600BFF0A100205D
:10E5F000020010004000100050001000608F00204A
:10E6000001001000DC6F624DA10AA94200F0AE804B
:10E610007ED9604DA94208D05F4A914200F0A280A5
:10E620004D3A914200F09C80FE22EFF3118150257B
:10E6300085F31288594E676AA58A02EB820206EBBF
:10E64000C202013745F001055762C9B2A58281F3C4
:10E6500011889EE6D3F894404D4DA10AA94200F0DE
:10E66000898065D94B4DA94207D04B4A914200F0B1
:10E6700085804D3A91427FD0FE22EFF311815025E3
:10E6800085F31288454E676AA58A02EB820206EB83
:10E69000C202013745F001055762C9B2A58281F374
:10E6A000118880E6B1F5801F24D03D4A91427FF465
:10E6B000C7AE0222C5E6B1F5801F1FD0384A91428D
:10E6C0007FF4FCAE0222FAE6B1F5801F1ED0344A78
:10E6D00091427FF474AF022272E7B1F5801F4FD0F0
:10E6E0002F4A91427FF437AF022235E70522A8E690
:10E6F0000322A6E60122A4E60522E0E60122DEE6E8
:10E700000421FFE605225BE7042271E6012257E7B8
:10E71000B1F5801F28D0224A914285D1022284E798
:10E720000521EFE60121EDE60321EBE60021E9E614
:10E73000B1F5801F1CD01A4A91429DD102229CE75C
:10E74000052255E6032253E6012251E6042278E62B
:10E750000322B4E60422B2E6042231E703222FE7C3
:10E76000042262E7052260E701225EE703225CE7FC
:10E77000012282E7032280E704227EE705227CE76C
:10E780000122E9E60322E7E60422E5E60522E3E6C4
:10E79000020010004000100050001000608F0020A8
:10E7A00001001000704700BF70B4150BC2F30324C2
:10E7B000064605EB450504EB44044800C2F3031389
:10E7C0001835183402F00F02356003EB430346F8A6
:10E7D000214002EB420201441833183246F820303F
:10E7E000062046F8212070BC704700BF2DE9F04F8D
:10E7F00012F4004F14BF4FF00E0B4FF0070B12F442
:10E80000804F14BF4FF00E0A4FF0070A12F4005F5A
:10E8100014BF4FF00E094FF0070912F4805F14BFC8
:10E820004FF00E084FF007084FEA410C12F4006F4A
:10E8300083B001EB0C0714BF4FF00E0E4FF0070E24
:10E8400012F4806F01EB070614BF0E2307238D1906
:10E850000193034612F4007F01EB0504C3F800B0F6
:10E8600018BF0E2043F821A008BF072043F82C90C2
:10E8700012F4807F01EB040C43F8278043F826E074
:10E8800001EB0C0714BF4FF00E084FF00708019E74
:10E8900043F8256012F0800F01EB070614BF4FF01C
:10E8A0000E0E4FF0070E12F0400F43F8240001EB5C
:10E8B000060514BF0E20072012F0200F43F82C800D
:10E8C00001EB050414BF4FF00E0C4FF0070C12F0D3
:10E8D000100F43F827E043F8260018BF0E2701EB7E
:10E8E000040008BF072712F0080F43F825C018BF1F
:10E8F0000E2643F8247008BF07260C1812F0040FE8
:10E9000043F8206018BF0E2501EB040008BF07255F
:10E9100012F0020F43F82450014414BF0E240724C0
:10E9200012F0010F43F8204014BF0E2207221220DC
:10E9300043F8212003B0BDE8F08F00BF704700BF4F
:10E9400070B4044600F16C06064D0FCD2D8825826B
:10E9500020606160A260E3601234B442F4D170BC04
:10E96000704700BF1C910408034B33F8142F02803A
:10E970009B788370704700BF1C91040807280AD851
:10E9800000EB4000044B10B553F8304014B139F09F
:10E990008DF8206010BD70473899002070B505468D
:10E9A0006C0039F083F82849631901EB43131E7B8F
:10E9B00006B970BD254A566880B21EB1167B0EB9E5
:10E9C000567B66BB2C4401EB4414214B227D2081F5
:10E9D00042EA400290B2021282EA1012424002F071
:10E9E0000F0242EA00121B781A480026267592B2DE
:10E9F0000668DBB9602000FB051018300121B04724
:10EA000021696368B1F82C216489DB682243A1F88D
:10EA10002C2158601A6842F001021A6070BD2A4425
:10EA2000907B0028CED001221A75CBE7636820695D
:10EA30005B7903F0FC030C3318440421B0472369CD
:10EA40008000188170BD00BFE0A200208C2B002048
:10EA5000DCA20020D4A2002038B500EB4000084D15
:10EA6000C4002B1993ED027AD3ED037AE7EE007A16
:10EA7000B0EE670A39F01AF82B59186038BD00BF9C
:10EA8000F0A10020F8B5A0F5197423796179DB07AE
:10EA900046D594F84832206C0BBB94F84B32012BCE
:10EAA0003FD0002B41D194F84A3294F849629E42FB
:10EAB0000CD9B4F85222012707FA03F501332A438F
:10EAC000DDB2AE4292B2F7D8A4F852220123C94374
:10EAD00084F84B321940BDE8F8402DF095B8026833
:10EAE000D36A5B08536294F85932012B07D094F82B
:10EAF0004D3223B1B4F854320133A4F85432C9432F
:10EB000001F001012DF080F80023012284F84B224E
:10EB100084F8493284F84A32A4F8523284F84832F0
:10EB2000F8BD94F8493284F84A32002384F84B3215
:10EB300001F00101BDE8F8402DF066B810B5437949
:10EB400003F0200113F0010F036C04461A7A806B66
:10EB500017D000290CBF4221022109F063FD226C6D
:10EB6000012384F84C32A4F84832517912688B4062
:10EB7000118C9BB221EA03011184118C0B43138485
:10EB800010BD00290CBF2221022109F04BFDE6E750
:10EB90000A4B1A6810B41446B4FBF1F3B3F5803F86
:10EBA00007D3012CFAD96408B4FBF1F3B3F5803F25
:10EBB000F7D299B25DF8044B0AF00EBAB0A2002069
:10EBC0008160006CE4E700BF436CC06B1BB11A7A34
:10EBD000012109F027BD2CF0D5B900BF4379C06BE6
:10EBE000DB0748BF81F0010109B90EF075BA0EF0DC
:10EBF00079BA00BF38B5A0F517742379990747D4BF
:10EC0000D80700D438BD94F84832002BFAD194F8D4
:10EC100049320133DBB2092B84F8493270D00A2B18
:10EC2000F0D194F84B52B4F85232002D00F0AA8083
:10EC3000990503F0010200F1AC80002A00F0A980E0
:10EC40001A46E36A5208002B00F0AF80D0B2216B65
:10EC5000984794F84B5201220023954284F8493298
:10EC600084F84822CED1617984F84B321140206C6F
:10EC70002CF0CAFF236C1A68597905FA01F3118C3C
:10EC80009BB221EA03011184118C0B43138438BD1C
:10EC900094F84D226ABBD4E90950854294F84C128D
:10ECA00046D0451CA369A5621B5C2069DBB2854286
:10ECB0004FEA430328BFA26243F400730A200122F3
:10ECC000A4F8503284F84E0284F84D2211B16179D3
:10ECD0000D073FD45A08A4F8502203F00101204642
:10ECE000FFF77CFF94F84E222379013A84F84E22F4
:10ECF00086E794F94E22002A66D184F84D227FE7F8
:10ED000094F84B32002B7FF47DAF94F84A32082BF5
:10ED10003FF678AFB4F85222012000FA03F1013334
:10ED20000A43D9B2082992B2F7D9A4F8522238BDC1
:10ED300000297FF465AF627912077FF561AF636CDC
:10ED4000E06B63B31A7A09F06DFC2046FFF7F6FE1C
:10ED5000237955E7216CA06B0B684D79198CAA407B
:10ED600021EA02021A841A8C92B21A8410B100218C
:10ED70000DF0DCFF002384F84C322046FFF724FF1F
:10ED800023793DE743F001029B05A4F852227FF569
:10ED900058AFB4F856320133A4F856325BE7002876
:10EDA000D3D019460DF0C2FFCFE7E3696169D2B253
:10EDB000CA54E369E16894F84B520133B3FBF1F2B2
:10EDC00001FB1233E36146E7B4F8503282E700BF3B
:10EDD00010B5242009F08CFD044618B1112200233F
:10EDE0008271C371202120460EF0DAF80A200AF061
:10EDF00081FF20460FF030F8034B00280CBF0122A2
:10EE000002221A7010BD00BF38BC002070B52A4D18
:10EE10002A4C2B496A792B4E2B4804230B702376FE
:10EE200000216423012A84F821306183A18384F8BE
:10EE3000201061623170016020D0022A11D0A979BE
:10EE4000224A00230129136084F87830C2E9013393
:10EE500022D0022904D11E4AC4F8B030C2E90133DD
:10EE600070BD2822A01838F00BFD44F620619FEDFC
:10EE7000190A04F12C00FCF7D5F9E0E7282204F187
:10EE8000500038F0FDFC44F620619FED120A04F1B9
:10EE90005400FCF7C7F9D2E70F4AE367C2E9013330
:10EEA000D3609FED0E0A02F1100044F62061BDE828
:10EEB0007040FCF7B7B900BF9C7B00208C2B002072
:10EEC000487E00208A7B0020847B0020AC7B0020D1
:10EED0003C2C0020CDCCCC3D082C0020CDCCCC3E11
:10EEE0002DE9F84FAD4E3468E50500F1F880AC4AE5
:10EEF000AC4B92F80090DFF8F08200221A70B9F162
:10EF0000000F00F0FA800921A748FBF71DFD00283B
:10EF100000F0DB8044F01004A44AA54B176834606D
:10EF200017F48057B3F9065040F08D80A14B9B8AAF
:10EF3000AB4200F39F8044F040049F4B346093F851
:10EF400000B01BF0080F06D11E219748FBF7FCFC10
:10EF5000002800F0FE8024F08004984B1B88642B6E
:10EF6000974B1B688CBF44F4806424F4806458077A
:10EF700004D5B8F8BE20002A40F08180B8F8C0203F
:10EF8000002A7AD18F4BD3F8B03024F4006A002BDA
:10EF900075D18D4CC6F800A004F17805234602E037
:10EFA0000633AB421DD01A781F2AF9D19978DA7846
:10EFB000914202D35A79002AF2D01F217A48FBF7F6
:10EFC000C3FC20B1814B1B785A0740F1D5802378D0
:10EFD0004AF4007A0A2BC6F800A005D00634AC42E9
:10EFE00018D023780A2BF9D1A278E3789A4202D379
:10EFF0006379002BF2D0764B1B7F002B68D01BF07F
:10F00000010F65D1714B1B789B0761D44AF4802AAC
:10F01000C6F800A022216448FBF796FC90BBB9F12A
:10F02000000F36D0BAF1000F4DD1002388F8C2305E
:10F030000AF00EFED8F8C430C01A00284DDBBDE837
:10F04000F84F27F0CFBC18215748FBF77DFC00286C
:10F050007FF46CAF5F4B1A7B002A7FF467AF554992
:10F06000DA884B8A991AA942BFF665AF1344AB42BE
:10F070007FF761AF24F040045FE7990782D544F43D
:10F08000006A86E74AF4003AC6F800A0B9F1000F1A
:10F0900019D1514B1C78002C51D1002F5CD100218B
:10F0A0004148FBF751FC002839D0BAF1000FBCD021
:10F0B0004CB9002F65D030B92AF4002AC6F800A058
:10F0C000BAF1000FB1D00223B0E724F0100423E717
:10F0D0002AF4802AC6F800A09CE7BDE8F88F3F4AD2
:10F0E0003F4B91791A684FF47A7303FB01F3934213
:10F0F0009CBF24F480743460F9E63A4A98F8BC3036
:10F100001578002B33D1002D33D049462648FBF724
:10F110001BFC00286AD124F00804346029E02AF09E
:10F12000200A01462048C6F800A0FBF70DFCBAF102
:10F13000000F2ED0002CBED1002FBCD121E02AF42C
:10F14000002424F40064B4FA84F46409002FA6D0E7
:10F1500002E044F0800400E718211348FBF7F4FBB9
:10F16000A8B91C4B1B7B002B44D0074697E7002D0A
:10F1700048D188F8BC50C6E62AF4007AC6F800A048
:10F180002FE7002898D04AF4002333609BE700273C
:10F1900085E700287FF449AF8EE700BF047E00209A
:10F1A00020000020326500204C440020B0A0002048
:10F1B0008ABA002068AF0020247E002096420020FA
:10F1C0009C720020F8990020644700205E7B00209C
:10F1D000286400201CC0002098440020E8980020EB
:10F1E00040850020454E00208C2B002044F0080470
:10F1F0003460BEE72AF4002727F04007B7FA87F704
:10F200007F094CE749460348FBF79EFB0028B0D135
:10F2100081E700BF4C440020F8B55B4A1378D9075A
:10F2200000D4F8BD23F0010313700AF011FD574B11
:10F23000574D9A78C5F8C80002BB564B1B88002B67
:10F2400043D1554A554B1178186881F001010DF0F2
:10F250004FFF534E534C33782BB123781BB1524B95
:10F260001B68DA043AD5514B1B6800229B062270BA
:10F27000D7D40420BDE8F84027F01CBE1B79022B30
:10F28000DBD04B4C23780B2B18D801229A4040F648
:10F29000030112EA0106D0D112F4C06F0ED0093B6F
:10F2A000012B0BD8452020F04BF9FF2020F048F926
:10F2B000404820F031F9304620F042F93E4A3F4BB9
:10F2C00012685A600B232370B7E73D4B5A69002A36
:10F2D000BFD0196800220A605A74BAE7394B1F7808
:10F2E0000AF0B6FC3378002BBDD06A68002ABAD188
:10F2F00000F51C5010300A214FF47A72686069736F
:10F30000AA60002F3BD03A4614212F4838F0B8FAB3
:10F310002E4A1389012FB3FA83F34FEA53132ED0E9
:10F32000B2F86810002918BF0023022F27D0B2F8C6
:10F33000C810002918BF0023032F20D0B2F82811CD
:10F34000002918BF0023042F19D0B2F88811002912
:10F3500018BF0023052F12D0B2F8E811002918BFFA
:10F360000023062F0BD0B2F84812002918BF002343
:10F37000072F04D0B2F8A822002A18BF002383F078
:10F3800001032B736FE700BF5E7B0020347E0020FB
:10F390008C2B0020188500201A8500201C85002059
:10F3A000CCA2002032650020B0A00020047E002006
:10F3B0008A5F0020ECCE0408408500207C440020B9
:10F3C00020850020F57100209A2B0020E0A200206B
:10F3D0002DE9F04FDFF8A4B2964ADBF8CC101368A1
:10F3E000954CCBF8CC002DED108B411A97B00B4407
:10F3F000079013602046636808919847069000289C
:10F4000000F09C80D4F8B050002384F86030002DC8
:10F4100040F05485894B0993987DB4F95010B4F9A4
:10F42000522094ED086AD4ED096AB4F954300028EA
:10F4300000F0A28407EE901AB8EEE77A07EE902A61
:10F44000F8EEE77A37EE467A77EEE67A84ED0B7AD5
:10F45000C4ED0C7A07EE903A94ED0A7A94F85E10B7
:10F460007748F8EEE77A77EEC77AC4ED0D7A16F0B2
:10F4700023F9744B1D78002D00F03984724BDFF8AE
:10F48000C091724E1F783568D4ED077A059309F55F
:10F49000B678B9EC018A132F05F000554FF0000A39
:10F4A00028EE278A42D0062F06D1B0EE480A38F05F
:10F4B000FDFA674B23F81A001DB1BAF1000F03F0F3
:10F4C000D182B0EE480AD4F8943140469847D4F837
:10F4D000043208F170009847D4F8B430A8F1E00085
:10F4E0009847D4F82431A8F170009847356805F0A2
:10F4F0000055B0EE408A0AF1010A2B46002D41F07A
:10F500009780059A1778032F01F07B80BAF1030FDB
:10F5100089ED028A00F01B84B9EC018AD4ED077AE8
:10F52000132F08F1240828EE278ABCD104EB4A03E4
:10F53000474AB3F8503022F81A30BDE7424B454AEB
:10F540001F78059306921146D4ED0E7AD4ED0F6A1A
:10F5500094ED107A94F8E8323F4D94F8F022C1ED22
:10F56000017AC1ED026A81ED037A8BF8D0302A70FE
:10F5700053BBDBED354A394BCBED357A77EEA47AC8
:10F58000DDED084ADBED363A9BED374A93ED005A44
:10F5900093ED026AD3ED015ACBED366AFAEEEF4AEB
:10F5A00076EEA33A37EE044AA4EEA75AF0EE467A76
:10F5B000E4EEA35AE4EE247A83ED005AC3ED015A37
:10F5C000C3ED027A8BED377A052F00F08783244A4A
:10F5D000DBF8E0301178B3FBF1F201FB12320133BA
:10F5E000CBF8E0304AB1059B1B78012B00F0698312
:10F5F00017B0BDEC108BBDE8F08F1A4B1B78002BB9
:10F6000042D0194A194BB2F906209B8A9A423BDC38
:10F61000174B1B78012B33D0192B31D00E2B33D045
:10F62000082B31D01349144A0A91002393608B6050
:10F630002CE000BF44BC0020F899002080A00020EE
:10F64000249A0020B5410020F5840020B0A00020BD
:10F65000F8840020A0A0002060C0002048BC00204A
:10F660007E420020200000208ABA002068AF0020DF
:10F670001C460020B0C100208C7B00208C2B002079
:10F68000D44B9B7B002BCDD0D34B0A9336F0C4F8E0
:10F69000059B1A78052A01F0048300230D9329782D
:10F6A0000991CE49CE4B096808911B78CD499BED55
:10F6B00039AA91ED008A002B40F0F282CA4B1B78E8
:10F6C000002B00F0ED82C949C94BD1ED006A1B88BF
:10F6D000DFEDC87AC849B0EEE67AA3F57A7327EE73
:10F6E000277A07EE903AF8EEE77AF7EE009AE7EE1F
:10F6F000879A2B2AC1ED009A01F05B87BF4B9FEDE3
:10F70000C06AD3ED007ABF4BDFF870A3D3ED006A77
:10F71000BD4DDFF86C93DFF86C83BC4FB7EE007A19
:10F7200037EE488A10AE68EE277A0024F4EEC77AE6
:10F73000F1EE10FA88BFF0EE477AF4EEC67AF1EEF9
:10F7400010FAB8BFF0EE467A67EEA67A67EEA99A8D
:10F75000AF4AD9F80030BAEC010A10199847AD4AFF
:10F76000D8F800301019984728463B689847243449
:10F770006C2CA6EC010A05F10805E9D1A64B1A7814
:10F78000A64BD3ED005A069BD3ED018A002A40F028
:10F790005583F5EEC05AF1EE10FA3FDD994B9FED1F
:10F7A000A06AD3ED007A069B67EE867AD3ED026AF3
:10F7B00093ED037A27EEA86A66EEA76A67EE277ACA
:10F7C0008DED136ACDED146ACDED157A954BDDED17
:10F7D000136AD3ED025A93ED016AD3ED004A9DED11
:10F7E000147ADDED157AB0EE655AA6EEC65AA6EE8D
:10F7F000A56AF0EE645AE7EE455AA7EE245AF0EEF9
:10F80000464AE7EEE54AE7EE865A83ED025AC3ED33
:10F81000014AC3ED005A002A40F02E83824F834AEA
:10F82000834BB2F800A0804CDFF85C929FED81BA68
:10F830009FED81DADFED81AA9FED71CADFED80CA0D
:10F84000DFED80BADFF844820C97002635461F466C
:10F850007D4B3344D3ED007A0A9BF5EE407A334476
:10F86000F1EE10FA0B93D3ED00DA17D0774B334457
:10F8700093ED007A7DEEC76AB0EEE66AF4EEC67AE2
:10F88000F1EE10FA08D5F5EEC06AF1EE10FACCBF31
:10F8900077EE87DA77EE67DAC3ED00DA40F6030C2D
:10F8A0001AEA0C0C00F09186022D00F09186684B4C
:10F8B000684953F825300898674A90F82D0081FB75
:10F8C00003E1DB17C3EB611307EE903A07EE100A72
:10F8D0003244B8EEC76AF8EEE77AD2ED006A4342E6
:10F8E00007EE103AE6EE267AB8EEC77AF4EEC77A5B
:10F8F000F1EE10FA0AD407EE100AB8EE477AB4EE29
:10F90000E77AF1EE10FA88BFB0EE677A534B5449AC
:10F9100003EB450331F91520B3F90C30D21A07EE89
:10F92000902A40F60103F8EEE77A1AEA030FA7EEF1
:10F93000EC7A00F0DB854B4BD3ED00DA67EE2DDA85
:10F94000494B9BF800011A78002800F06784002AD0
:10F9500000F0C883089B3DEEE8EA93F84E10434B55
:10F96000DBF80C2107981B68821A9A4240F3BF8388
:10F97000022901F031823E4B022D186840F0A08729
:10F980003C4B93ED007AF1EE477AB4EEE7EAF1EE04
:10F9900010FA08D4B4EEC7EAF1EE10FA8CBFF0EE1C
:10F9A000477AF0EE4E7A824284ED01CA01F3548127
:10F9B000B0EE67EA0B4B93ED007AF7EE007AB4EE07
:10F9C000E77AF1EE10FA01F12381F0EE4CEA2A4BCE
:10F9D0001A785DE028990020B0C100203480002012
:10F9E000F9BF0020E8C000202DC10020E4C00020A5
:10F9F000CCBF00200AD7233CE8020020C8BF00206B
:10FA000000000000DCB90020B0BE0020ACBE002029
:10FA100040BE0020CCBE0020F8BF00200CC000205B
:10FA200035FA8E3C50C00020A8460020B87B00204C
:10FA3000742C0020000096428988083D0000C842CE
:10FA4000CDCCCC3D6F12033BBCBF0020802C0020EE
:10FA5000EC6300201F85EB5198C100203441002049
:10FA6000F47B0020A4BF002046640020D4BF002007
:10FA7000D0BF0020ECBF00204CBF0020A4A000207D
:10FA80003CBE0020C8BE002070B9002074BF00201A
:10FA9000D34B93ED006A002A00F0CA83022D00F0D8
:10FAA000B586D04B03EBC50393ED008AD3ED016A15
:10FAB0003DEEC87AF5EEC0EAA6EE878AF7EE007A48
:10FAC0003DEEC89AF1EE10FAB0EEC99AF1EE49FA9D
:10FAD00083ED008AEFEE8D7A05DDB5EEC0EAF1EE3A
:10FAE00010FA00F1D685F5EEC0EAF1EE10FA00F159
:10FAF000CA85BD4B1B78012B01F06980002B01F0FA
:10FB000072809FEDBAFA002D02F05E87F0EE007A67
:10FB1000B0EE487AAFEEA77AA9EE278AB4EEE87A7B
:10FB2000F1EE10FA00F29684B4EEE88AF1EE10FAE3
:10FB300078EE687AC0F29784AD4B3344D3ED006A17
:10FB4000AC4B66EEA75A93ED005AF5EEC05AF1EEB3
:10FB500010FA58BF77EE687AB0EEE67A65EE275A6B
:10FB6000F0EEE55AF4EEC75AF1EE10FA40F37B845A
:10FB7000F1EE666AB0EE4E9A86EE85EAB5EEC06AA0
:10FB8000F1EE10FA00F35E8398ED000A2AEE000A07
:10FB9000022D20EE090A84ED000A00F04F86D8ED10
:10FBA000017A954B69EEA77AB0EE6E6AA7EE8F6A7E
:10FBB000D3ED006AB1EE667AB4EEC76AF1EE10FAE0
:10FBC000F0EE467A12D4F4EEE67AF1EE10FA8CBF3B
:10FBD000B0EE667AB0EE677A022D07D1874B1B78BC
:10FBE000012B00F01C85192B00F01985844BD3EDF7
:10FBF000006AF7EE007AF4EEE76AF1EE10FAACBFB5
:10FC00000123002343B1F0EEEEEAF0EEC77AF4EE02
:10FC1000EE7AF1EE10FA01D584ED017AD8ED027A90
:10FC200010ABF5EEC07A3344F1EE10FAD3ED008A52
:10FC300000F3E283734B84ED02CAB3F800A0724B69
:10FC40003344C3ED008ABAF1000F00F05F8384ED06
:10FC500003CA099BE7EC01DA002B40F0498394EDDD
:10FC6000037A94ED006AD4ED017AD4ED026A76EE5F
:10FC7000277A013577EEA67A032D77EE877A08F199
:10FC80001008C4ED047A09F1240906F1040604F110
:10FC9000140400F0F985069B3344D3ED018AD7E5BF
:10FCA0005A4B2B2AD3ED009A7FF428ADDFF86C81F4
:10FCB0009FED570A29EE800A37F0F8FEA8F80000F9
:10FCC0001CE5544B544A19681288544BC969198071
:10FCD0005A8017B0BDEC108BBDE8F08F09F0B8FF6B
:10FCE000079BDFF83881C01AA8F800006FE44C4F7A
:10FCF0004C4E07F5B67A07F18C0807F51379D4ED69
:10FD0000077AB7EC010AD4F8943120EE270A0AEBFF
:10FD100005009847444AD4F8043250199847D4F85B
:10FD2000B43008EB05009847404AD4F82431501904
:10FD300098473368980000F1928424356C2D87ED44
:10FD4000020ADCD13A4A0592177803F00053099A67
:10FD5000927D22B1374A1078002800F0E187099A95
:10FD6000527E002A40F06681002B40F09881324B91
:10FD700006931946FFF7E8BB2E48007800287FF469
:10FD800059AB606C0D1A002DB8BF6D42B5F5804FB0
:10FD900041F3728307EE900AA16CB8EEE77A501A2D
:10FDA000002837EE467AB8BF4042B0F5804F84ED68
:10FDB0000B7A41F35D8307EE901AE16CF8EEE77A77
:10FDC0005A1A002A77EEE67AB8BF5242B2F5804F4F
:10FDD000C4ED0C7A41F349830B46FFF73BBB00BFF0
:10FDE0000CC0002050BF0020FBBF0020000000001E
:10FDF00050C00020DCB90020F0BF002030BE002041
:10FE0000E8C00020B87B0020A02C0020E8020020E1
:10FE100000007A442084002096420020F8840020CC
:10FE2000249A0020B0A00020009C0020209B0020ED
:10FE3000F5840020A5000020A0A00020AD4BDFED40
:10FE4000AE6A93ED006A069B26EE266A93ED027A6F
:10FE5000D3ED037A66EE286A27EE067A67EE867A95
:10FE6000F5EEC05AF1EE10FACDED136A8DED147A6D
:10FE7000CDED157A3FF7AAACA04FD7ED0B4A97ED21
:10FE8000066A97ED015AF0EE645AE6EE665AA4EE61
:10FE9000A66AF0EE466AB0EE456AA7EE656AE5EE40
:10FEA000075AB0EE467AA7EEA67AE7EEC66AC7ED25
:10FEB0000B5A87ED017AC7ED066AB0E4904A914E7D
:10FEC0009148918B09920596577832780368DFF84C
:10FED0004082069042F2107606FB01F6B6FBF3F67E
:10FEE000B4F95030B8F90600B54207EE903A02F086
:10FEF000418194ED1A7AD4F88410F8EEE77A4B1C1D
:10FF000037EE277A012BC4F8843084ED1A7A02F098
:10FF10003285D4ED1D5AD4ED1F6A07EE103A37EE44
:10FF2000E56AB8EEC75A012D86EE057A37EE257AD6
:10FF300077EEC77A84ED1E7AE7EE866A84ED1D7A45
:10FF4000F0EE667AC4ED206AC4ED1F6A02F06082AA
:10FF5000B4F9523094ED1B7A07EE903AD4F8983009
:10FF6000F8EEE77A5A1C37EE277A012AC4F898206F
:10FF700084ED1B7A02F0FC81D4ED225AD4ED246A80
:10FF800007EE102A37EEE56AB8EEC75A012D86EE65
:10FF9000057A37EE257A77EEC77A84ED237AE7EE95
:10FFA000866A84ED227AF0EE667AC4ED256AC4EDA5
:10FFB000246A02F05882B4F9543094ED1C7A07EEAA
:10FFC000903AD4F8AC30F8EEE77A5A1C37EE277A3C
:10FFD000012AC4F8AC2084ED1C7A02F0FF80D4ED35
:10FFE000275AD4ED296A07EE102A37EEE56AB8EEF3
:10FFF000C75A012D86EE057A37EE257A77EEC77A55
:020000040801F1
:1000000084ED287AE6EE276A84ED277AF0EE667AA8
:10001000C4ED2A6AC4ED296A02F04E82A8F80600EF
:10002000D4F8B030059A06991778013BC4F8B0307F
:10003000FFF78ABA94F8E8225ABBD4ED107AFDEEA5
:10004000E77A17EE902A002AB8BF5242099994F82D
:10005000F002B1F91A10002801F0598207EE901A47
:10006000DFED2A6AB8EEE77A07EE902A37EE667A75
:10007000F8EEE77AB4EEE77AF1EE10FA42F3E583B0
:10008000D4F8EC22079844F62061821A8A427FF75E
:100090006BAE002284F8F022002B3FF468AE94F897
:1000A000F43294F8F5220133DBB29A4284F8F43248
:1000B00002F0C98094F8F834002B3FF458AE102FAA
:1000C00001F04E8394F8F9144FF00009062901F26B
:1000D0000C85DFE811F0310DA40CB50C6F0B390C59
:1000E000600EF00DBCF1000F14D03DEEE8EAD4ED47
:1000F00001EA6CE4DCB9002035FA8E3CA846002009
:1001000080A00020F5840020A0A000200000C842AC
:10011000F8840020D74BD849DFF8A8E331F915104F
:10012000DFF8A4A35EF806C0DAED006A03EB45032E
:10013000F5EEC0DAB3F90C30C91A07EE901AB8EE32
:10014000E70AF1EE10FA20EE2C0AB7EE007AFFEE85
:10015000007AB5EEC00AD4BFF0EE675AF0EE475A07
:10016000CCBF4FF0010A4FF0FF3AF1EE10FAC8BFD2
:10017000F0EE477ACCBF01234FF0FF33B0EEC07AE8
:10018000BCF1000F04D0D44502F014814EF80620D3
:10019000B4EEE67AF1EE10FA02F30281B74BF0EE1C
:1001A000E87A67EEAB7A93ED007AB7EE006AF4EE88
:1001B000C67AF1EE10FA28EE877A88BFF0EE467A1A
:1001C000B0EE408AA7EE878AB5EEC08AF0EEC87A14
:1001D000F1EE10FAF4EEE67ACCBF01234FF0FF33D4
:1001E000F1EE10FA02DD9A4502F003814FF0000AA9
:1001F000002A42F00981A24B1B78AB427FF475AF15
:10020000059B1B78272B02F00284022D7FF46DAF33
:10021000099B002B42F0D7859A4B1A783DEEE8EA0D
:10022000002A3FF464AF089B93F84E10FFF797BB8A
:10023000B5EEC06AF1EE10FAB0EE4E9AB0EE4EFA9C
:100240007FF7A2AC9BF81031002B3FF49DAC8E4B96
:100250008E4A334492ED007AD3ED007A8C4AEEEE6A
:10026000077AD2ED006AB1EE667AF4EEC77AF1EE63
:1002700010FA08D4F4EEE67AF1EE10FA8CBFB0EE84
:10028000667AB0EE677A834A83ED007AD2ED006A2F
:1002900027EE066AF1EE667AB4EEE76AF1EE10FA3E
:1002A00008D4B4EEE66AF1EE10FA8CBFF0EE667A8E
:1002B000F0EE467A7DEEA7DA3FEE27FA002D7FF4C6
:1002C00063AC059B1B78262B07D1B2EE040A27EE00
:1002D000000A37F0EBFB704BD880704BD3ED007AFF
:1002E0000C9B6AEE277A67EE897AC3ED007A56E4B2
:1002F000022D84ED01CA00F0D381B0EE4C7A84ED7A
:1003000000CA84ED02CA84ED03CAAAE498ED039AF8
:10031000B5EEC09AF1EE10FA7FF799AC604BD3EDD1
:10032000007AF5EEC07AF1EE10FA00F3CF80B7EE66
:10033000008A5C4BD7ED008A1B78AB427DEEE88AE1
:1003400000F04E81584A12787AB3584A1278012A3E
:1003500000F03383022A25D199ED027AD9ED067A8D
:10036000D9ED056A99ED016AD9ED035AC9ED066A1E
:1003700067EE277A99ED077AC9ED058AE6EE267AC7
:10038000D9ED086A99ED046A89ED087AE5EEC77A35
:1003900099ED007AE6EE667AE8EE877AF0EE678A03
:1003A000C9ED077AAB4200F0F682414A414BD2EDEB
:1003B000007A1B7829EE279A29EE088A68EE288AA7
:1003C000C4ED038A002B3FF444ACD4ED007A28EE50
:1003D000A77AB5EEC07AF1EE10FA7FF73AACF0EEFC
:1003E000E88AF0EEE77AF4EEE78AF1EE10FA7FF7AA
:1003F0002EAC84ED00CA2CE42F4B2D4A334493EDF0
:10040000008A089B92ED007A93F84E3038EE688AA5
:1004100028EE078A2BB9294BB3F800A01AF4006F15
:1004200010D09BF8D03053B9254B164A1B78127860
:1004300013F0010340F0D984002A40F02C851F4BB3
:10044000B3F800A028EE0A8A68EE277AC4ED027A93
:10045000FFF7F5BBB4EEE88AF1EE10FA4CBF78EE88
:10046000687A77EE687AB0EE4E9AB0EE67EAFFF7F8
:1004700085BB00BF34410020F47B002000C0002079
:1004800004C000204664002050C00020DCB90020D9
:1004900014C0002010C00020F884002074BF002089
:1004A00070BF00206DB900206FB900206EB9002028
:1004B00038BE0020FABF0020A02C0020B87B00200E
:1004C0005E7B0020902C0020FCBF0020B84B334402
:1004D00093ED008A27EE888AF7EE007AB4EEE78A79
:1004E000F1EE10FA88BFB0EE678A22E7B04AB1F9A0
:1004F0000030D2ED007AD2ED016AB1F90220AD49A7
:10050000F4EEE76AF1EE10FAB4BFB0EE676AB0EE4F
:10051000666A002BB8BF5B42002AB8BF52429342C2
:10052000B8BF134607EE903AA34A0B7892ED005AF3
:10053000F8EEE77A67EEAC7A002B00F00682B5EEB3
:10054000C05AF1EE10FA40F332829C4BD3ED004AD0
:10055000F5EEC04AF1EE10FA40F3298274EEE77A24
:10056000DFED975AC7EEA46A66EE255AF7EE007AD9
:1005700085EE856AF4EEE76AF1EE10FA88BFF0EED8
:10058000676AF5EEC06AF1EE10FA76EE277AB8BF28
:10059000F0EE4C6A66EEA77AB7EE006AF4EEC67A21
:1005A000F1EE10FA88BFF0EE467AF5EEC07AF1EE81
:1005B00010FAB8BFF0EE4C7A824BD3ED006A27EE0A
:1005C000267AE7EE27DAFFF7BBB9022D7FF4B8A948
:1005D000099B002B7C4B18BFF0EE4CDA1A781DE615
:1005E000059A1278282A7FF4ADAE28EEAA0A0B935A
:1005F00037F05CFA754A0B9B5080A3E605F0005576
:100600002B46B0EE480A0A9337F050FA6F4B03EBD3
:100610004A01032721F8020C0A9BFEF777BFB4EECC
:10062000CB9AF1EE10FACCBF01230023FFF7EABA10
:10063000D9EDB37AD4F8743237EE808A08F1E0004D
:1006400089EDB38A9847BAF1010FB0EE408A02F003
:100650009D82356805F000552B46FEF752BF97ED99
:10066000B37AD4F8743277EE007A09EB0500C7ED5F
:10067000B37A984724356C2D87ED020A7FF43FAB9F
:100680003368FFF75FBBB5EEC0EAF1EE10FA7FF713
:1006900030AA022A7FF62DAAB0EE4EFAFFF733BA3F
:1006A0000C9F9BF82031D7ED0A7AD7ED0C6A97EDB5
:1006B0000D7A77EEA67A77EE877AC7ED0E7A002B61
:1006C00040F0E88000233B607B60BB60FB603B61E7
:1006D0007B61BB61FB613B627B62BB62FB623B6334
:1006E0007B63BB63059B1B78052B00F0F082384BC6
:1006F0001B78DB0708D5374B1B78DE0604D4364B56
:100700005B78002B40F0BC86344C059B1B780022A4
:10071000202BCBF8242100F04D81012B00F0C88262
:10072000052B00F02A84002306932378002B40F049
:10073000B7802B4B07981B6893F8461032F070F97E
:10074000284B1B68002B40F07381274B1B788BB123
:10075000264D287858B1264F264E0024E0B2336843
:10076000B7EC010A9847287801348442F6DB224B23
:100770001B689847059B1B78052B00F077821F4A62
:100780001478002C7EF431AF1D4DAA78002A40F079
:100790009583059B1B78052B7EF427AF09F058FA4B
:1007A0000A4A059B001B1B78D080FEF71EBF00BFC6
:1007B000A4C10020B0BF0020ACBF0020B4BF002007
:1007C0000000C8C2A8BF002046640020F8840020B2
:1007D0005E7B0020247E00207E42002032650020C7
:1007E0003480002034BE002064AF0020F57100206A
:1007F000E4460020D0A20020D8A20020507D002096
:10080000347E0020000000005FED02DA022A3FF48F
:1008100048A9042A3FF445A9B5EEC06AF1EE10FAE2
:1008200000F3808698ED000A2AEE000AB0EE4E9A98
:1008300020EE0E0AB0EE4EFA84ED000A674B6848CF
:100840001B689847674BD3ED097A674B69EEA77A27
:10085000B0EE6E6AAFEE276AD3ED006A0C9BB1EE84
:10086000667AB4EEC76AF1EE10FA83ED0A0A3FF534
:10087000B5A9B4EEE66AF1EE10FA8CBFB0EE667A76
:10088000B0EE467AFFF7AAB99BF820310C9F002BF7
:100890003FF418AF9BF8D030002B7FF413AF21E763
:1008A000524B534A1B781278DC0700F18983002AE7
:1008B0003FF446AF92004F494F4836F07BFF3FE789
:1008C0004E4B1B68990740F1E5814D4B4D49DFF8D0
:1008D0005CA131F915E0DAED00DA84ED01CA03EB31
:1008E000450C6DEEACDABCF90CC0ACEB0E0C07EEAF
:1008F00090CAF8EEE77A824267EEADDA3DEEE8EABA
:100900007FF758A8B1F900C0B3F90C203E48ACEB12
:100910000202002A0068B8BF52428242BFF655A8C0
:10092000B1F90220B3F90E30D31A002BB8BF5B42E5
:1009300098427FF74AA80023344A184613700DF0F6
:100940004FFAD4ED01EAFFF742B8314BDFED316ADF
:10095000D3ED005AF4EEE65AF1EE10FA0FD5F7EEA9
:10096000004A34EEE54ADFED2C6ADFED2C4A76EEE4
:10097000E77A64EE244AE7EEA45A25EE255AB5EE4E
:10098000C05AF1EE10FA12D9CAEE856AF7EE007A73
:10099000E6EE667A00E6059B1B78282B7FF405AD12
:1009A00028EEAA0A37F082F81D4B9880FDE4DFEDAF
:1009B0001D7A01E61A4B1A60B5E61B4A02EBC50226
:1009C000D2ED007A92ED017A78EEE78AE7EE287AA6
:1009D000F0EE678AC2ED007AE4E400BF40BF002079
:1009E00038BF002074BF0020F0BF00205E7B0020D5
:1009F000F571002098420020E44600209C720020FF
:100A000034410020F47B0020D8BF00204664002041
:100A1000B8BF0020AE47813F00003443610BB63BB6
:100A2000F884002000000000E0B90020A4BF0020EE
:100A3000AA4F3B78192B0AD80122A94902FA03F3DD
:100A4000194011B9A74A134201D033F037FEA64E20
:100A5000A64D3368980600F14482A54CB4F90020F5
:100A6000B5F90430B5F906109A4203DB91420B4602
:100A7000A8BF1346B4F90220B5F9100023809042B4
:100A8000B5F9123003DC9342A8BF13461846B4F9F7
:100A90000430B5F91C1060809942B5F91E2003DCC2
:100AA0009A42A8BF1A461146B4F90630B5F9282073
:100AB000A1809A42B5F92A1003DC99420A46A8BFE0
:100AC0001A46B4F90830B5F93410E2809942B5F904
:100AD000362003DC9A42A8BF1A461146B4F90A3000
:100AE000B5F9402021819A42B5F9421003DC9942C0
:100AF0000A46A8BF1A46B4F90C30B5F94C10628109
:100B00009942B5F94E2003DC9A42A8BF1A46114615
:100B1000B4F90E20B5F95830A1819342B5F95A10B5
:100B200003DC91420B46A8BF1346E381714B9B89BE
:100B300023B3DFF8E091DFF8E081DFF8B0A109F13D
:100B4000100539F9023F00EE103A4046B8EEC00AEF
:100B5000F7F706FC36F0AAFFBAF90430BAF9062016
:100B600000B298422ADB9042A8BF1046A945A9F8D6
:100B7000000008F124080AF10C0AE2D13B78013B9D
:100B8000182B00F2C987DFE813F06D05C707C70708
:100B9000D304C707C707C707C905C707C707C707DC
:100BA000C707C707B8059D05C707C707C707C70712
:100BB000D304DA05C707C707B8056D05A945A9F825
:100BC000003008F124080AF10C0ABAD1D6E7B3EED6
:100BD0000E7AB4EEC79AF1EE10FA7EF592AF27EED8
:100BE0008EFAFEF790BF38EE68FAB0EECF7AB4EE28
:100BF000C79AF1EE10FA3EF784AFB5EEC0FAF1EE07
:100C000010FAACBF3FEE49FA39EE0FFAFEF77BBFA0
:100C1000069A394BD2ED017A93ED007AF0EEE77A3D
:100C2000F4EEC77AF1EE10FA7EF5CFAED2ED027A8D
:100C3000F0EEE77AB4EEE77AF1EE10FA7EF7C5AEA1
:100C4000D2ED037AF0EEE77AB4EEE77AF1EE10FA3D
:100C50007EF7BBAEF0EE4E7A284B1B689A07B0EEDB
:100C600067EA7FF568AE2649264B4BE608F0F0FFB1
:100C7000059B06991B78244A401A052B908040F06A
:100C8000138108F0E5FF214B1B780446002B7FF40D
:100C900080AD79E5824284ED01CA3FF74CAEFEF7A4
:100CA00089BE08F0D5FF059B0D901A78FEF7F7BCBA
:100CB00008F0CEFF164ADBF8283112681249069078
:100CC000C31A9A1ACBF82801CA808B802DE508F048
:100CD000BFFF0D9A0C4B801A588008E530BE0020EB
:100CE00030C1300102000002B0A0002064480020A2
:100CF0000447002028990020DCBF00209C720020BF
:100D0000F47B002034410020F8840020507D002036
:100D1000C0B80020024700209CBC002000D8F94643
:100D2000D4ED0E7A94F8E822D4ED076AFDEEE77A66
:100D300017EE901A0029B8BF494207EE901AF8EE54
:100D4000E77A002A40F04C841FED0C6A94ED0F7A8C
:100D50008C4866EE866ABDEEC77AF4EEE76A17EE57
:100D6000102AF1EE10FA4CBF01210021002AB8BF71
:100D7000524207EE902AF8EEE77A0078F4EEE76A3E
:100D8000D4ED107AFDEEE77AF1EE10FA17EE902A24
:100D900048BF41F00201002AB8BF524207EE902A34
:100DA000F8EEE77AF4EEE76AF1EE10FA48BF41F0A8
:100DB0000401014200F04F84012100220798C4F889
:100DC000E40284F8E81284F8F022099A527E002A9C
:100DD0003EF4CAAFFFF75DB901200DF001F8DBF872
:100DE0000C21079B9A1AFEF7C6BD674BD3ED006A2C
:100DF000B7EE007AF4EEC76AF1EE10FAC0F2E583BE
:100E0000002A40F0E583614B93ED007AF0EEC86A6A
:100E1000F4EEC76AF1EE10FA7FF711AB5C4B93ED7D
:100E2000007AF0EEC96AF4EEC76AF1EE10FA7FF7C5
:100E300006AB0B99574B91ED007AD3ED006AB0EEFB
:100E4000C77AB4EEE67AF1EE10FA7FF5F8AA0799C0
:100E5000CBF80C11504901230B70504B1B68934287
:100E60007FF7EDAA4A4B93ED007AB0EEC99AB4EE43
:100E7000C79AF1EE10FA0DD40B9A464B92ED007A18
:100E8000D3ED006AB0EEC77AB4EEE67AF1EE10FA6E
:100E90007FF7D5AA0023404A184613700CF0A0FF34
:100EA000D8ED027AFFF7CBBA3D4A1478002C7EF4D5
:100EB0009CAB3C4DAA78002A3EF497AB3A4E33786F
:100EC000013B0A2B01F24880DFE813F0C207250935
:100ED000F008D108B9089E088A087308510832083A
:100EE000EE07EB7AFF2B00F07883304A12789A42B3
:100EF00040F273832E4A32F91380EB7D2D4CFF2B89
:100F0000A4F8008001F03082284A12789A4241F217
:100F10002B82274A32F91390A4F802900D2033F067
:100F2000C7FB00283FF49AAD234B95F916001A88A9
:100F300022499BF82CC1B3F902A095F90A3010FBA5
:100F400002F281FB02E00011D217BCF1010F1FFA7F
:100F500088F81FFA89F9A0EB020E01F0188513FB3F
:100F60000AF381FB0321DB17C3EB21139844F144FF
:100F7000A4F80080A4F8029070E508F069FE0690DD
:100F8000FFF7D3BBB4410020E8C00020E4BF00203D
:100F9000E0BF0020E8BF002046640020D4BF00204E
:100FA000507D0020347E00208A5F0020BC64002039
:100FB0008ABA002004470020F47B00201F85EB51F3
:100FC000EA49EB4BD1ED017A93ED006A91ED005ABD
:100FD000D3ED016A91ED027AE64993ED024A487831
:100FE000F5EEC07AF1EE10FAB5EEC05A26EE065ACA
:100FF000F7EE007AA6EEA65AFFEE005A54BFF0EEC6
:10100000654AF0EE674AF1EE10FAB5EEC07A54BFC9
:10101000B0EE657AB0EE677AF1EE10FA54BFF0EEFA
:10102000653AF0EE673A58BFF0EE675AF1EEC57ACE
:101030000028B4EEE66A18BFF0EE635AF1EE10FA3B
:10104000B4BFF0EE663AF0EE463AF4EEC43AF1EE92
:1010500010FA9FEDC95A4ABF9FEDC87ADFEDC75A13
:10106000F0EE447A27EE855A36EE263A9FEDC44AD2
:10107000C3EE053A48BFF0EE474AF4EEC43AF1EE4B
:1010800010FA0BD5B4EEE66ADFEDBC6AF1EE10FAA9
:10109000D8BFB0EE667A88BFF0EE664A9FEDB95AC7
:1010A0009FEDB66ADFEDB86A77EEC57AF4EEC67AE0
:1010B000F1EE10FAB8BFF0EE467A67EEA67A002A93
:1010C0003FF43EAB8B78B149DFEDB16A91ED005A48
:1010D000B048B14990ED004AD1ED003A06EE103A21
:1010E000B8EE463AB3EE046A23EE263A35EE066AC7
:1010F000002B41F00982A94BA949D3ED016AD3ED38
:10110000022A93ED033A67EE266AE4EEA26AE5EE60
:10111000836AB7EE003AF5EEC06AF1EE10FA48BF06
:10112000F0EE446A67EEA66AF4EEC36AF1EE10FAD6
:1011300088BFF0EE436AB0EE453AA3EEA63AB4EEAD
:10114000C36AF1EE10FAF0EE436A9ABFB3EE043AC6
:1011500076EEC36AF0EE446A012AC1ED006A3FF4FC
:10116000EFAAD3ED056AD3ED062A93ED073A67EEB1
:10117000266AE4EEA26AE5EE836AB7EE003AF5EE7F
:10118000C06AF1EE10FA48BFF0EE446A67EEA66A54
:10119000F4EEC36AF1EE10FA88BFF0EE436AB0EEE7
:1011A000453AA3EEA63AB4EEC36AF1EE10FAF0EEB9
:1011B000436A9ABFB3EE043A76EEC36AF0EE446A2D
:1011C000022AC1ED016A3FF4BBAAD3ED096AD3ED4F
:1011D0000A2A93ED0B3A67EE266AE4EEA26AE5EE80
:1011E000836AB7EE003AF5EEC06AF1EE10FA48BF36
:1011F000F0EE446A67EEA66AF4EEC36AF1EE10FA06
:1012000088BFF0EE436AB0EE453AA3EEA63AB4EEDC
:10121000C36AF1EE10FAF0EE436A9ABFB3EE043AF5
:1012200076EEC36AF0EE446A032AC1ED026A3FF427
:1012300087AAD3ED0D6AD3ED0E2A93ED0F3A67EE30
:10124000266AE4EEA26AE5EE836AB7EE003AF5EEAE
:10125000C06AF1EE10FA48BFF0EE446A67EEA66A83
:10126000F4EEC36AF1EE10FA88BFF0EE436AB0EE16
:10127000453AA3EEA63AB4EEC36AF1EE10FAF0EEE8
:10128000436A9ABFB3EE043A76EEC36AF0EE446A5C
:10129000042AC1ED036A3FF453AAD3ED116AD3EDDA
:1012A000122A93ED133A67EE266AE4EEA26AE5EE9F
:1012B000836AB7EE003AF5EEC06AF1EE10FA48BF65
:1012C000F0EE446A67EEA66AF4EEC36AF1EE10FA35
:1012D00088BFF0EE436AB0EE453AA3EEA63AB4EE0C
:1012E000C36AF1EE10FAF0EE436A9ABFB3EE043A25
:1012F00076EEC36AF0EE446A052AC1ED046A3FF453
:101300001FAAD3ED156AD3ED162A93ED173A67EEAF
:10131000266AE4EEA26AE5EE836AB7EE003AF5EEDD
:10132000C06AF1EE10FA48BFF0EE446A67EEA66AB2
:10133000F4EEC36AF1EE10FA88BFF0EE436AB0EE45
:10134000453AA3EEA63AB4EEC36AF1EE10FAF0EE17
:10135000436A9ABFB3EE043A76EEC36AF0EE446A8B
:10136000062AC1ED056A3FF4EBA91BE098C10020F5
:10137000A4C100201C460020F304B53F000000007B
:10138000D7B35D3F9A99193E9696963F3CC0002090
:101390000AD723BCECC0002038C0002064C0002065
:1013A000E4460020D3ED196AD3ED1A2A93ED1B3AD7
:1013B00067EE266AE4EEA26AE5EE836AB7EE003ACB
:1013C000F5EEC06AF1EE10FA48BFF0EE446A67EE3F
:1013D000A66AF4EEC36AF1EE10FA88BFF0EE436A33
:1013E000B0EE453AA3EEA63AB4EEC36AF1EE10FAB7
:1013F000F0EE436A9ABFB3EE043A76EEC36AF0EEBB
:10140000446A072AC1ED066A3FF49AA9D3ED1D6A22
:10141000D3ED1E2A93ED1F3A27EE267AA4EEA27A88
:10142000A5EE837AB5EEC07AF1EE10FA48BFB0EEC1
:10143000447A67EE877AB7EE007AF4EEC77AF1EE77
:1014400010FA88BFF0EE477AA3EEA75AB4EEC56A49
:10145000F1EE10FAF0EE457A03D8B3EE044A37EE17
:10146000C44A81ED074AFFF76BB9E364FDF7F2BFA9
:10147000A2641146FEF79FBC61640846FEF78ABC71
:101480009BF82131BF4C002B7FF43FA92378002B20
:101490007FF43BA99BF82231002B7FF436A9BA4B8D
:1014A0001B68DD0601F1478497ED097ADFEDB77A15
:1014B000B0EEC77AB4EEE77AF1EE10FA81F28883E3
:1014C00097ED047AB0EEC77AB4EEE77AF1EE10FA4F
:1014D00081F27E8397ED0E7AB0EEC77AB4EEE77AAA
:1014E000F1EE10FA81F274830023CBF82431059BCE
:1014F0001B78202B7FF411A9DBF82431A44A003398
:1015000018BF0123012153801180FFF70CB99142CC
:10151000BEF62AAC01220799C4F8EC1284F8F02236
:10152000FEF722BCB0EE4E9AB0EE4EFAFEF78ABE3F
:10153000984B1A6812B1B4F9081011609B69002B1E
:1015400001F08B81B4F90A201A60032704220225D6
:101550003368990601F17081DA027FF5F6A88E4BA7
:10156000DC7B112C3FF7F1A88C4F37F9143000EEDB
:10157000103A2846B8EEC00AFDF700FAC4F1120886
:101580004FF0010905EB0900C14509EB0403C0B2A6
:1015900009F101093FF4D9A837F9133000EE103AE8
:1015A000B8EEC00AFDF7EAF9B9F10E0FEAD1FFF77C
:1015B000CCB89FED7B0ADFF8D88126EE800A36F0A2
:1015C00075FAA8F80200FEF773BB002A3EF437AFA5
:1015D000DBF80C21079B9A1A3FE4B5F908808CE4EC
:1015E0009FED707A66EE876AF4EEE76AF1EE10FA24
:1015F00041F32681D4ED0F7AFDEEE77A17EE902ABB
:10160000002AB8BF524207EE902AF8EEE77AF4EECD
:10161000E76AF1EE10FA41F31381D4ED107AFDEE92
:10162000E77A17EE902A002AB8BF524207EE902AB6
:10163000F8EEE77AF4EEE76AF1EE10FA41F3008192
:10164000D4F8E412079E4CF25035711AA9427FF784
:10165000BCAB84F8E8020999497E00293EF484ABCA
:10166000FEF7F4BC4C4B4B4A9B7B1268002B41F0BD
:10167000A2814D4B1B7813F0010341F09C81002A9D
:1016800001F07C82136001203368990603D43A7814
:10169000052A41F0DF80851C471CEDB2FFB2B4F98A
:1016A000003000EE103AB8EEC00AFDF767F9B4F961
:1016B000023000EE103A3846B8EEC00AFDF75EF987
:1016C000336849E7334B1A6812B1B4F9001011605E
:1016D0009A6912B1B4F9021011601A6B12B1B4F91F
:1016E000041011609B6C002B01F05F82B4F906209E
:1016F0001A600527062204252AE7DFF8B0900025A6
:1017000039F9023F00EE103AE8B2B8EEC00A0135EE
:10171000FDF734F9062DF3D12846B5E71D4B1A68BD
:1017200012B1B4F9061011609B69002B01F095808D
:10173000B4F908201A6003270422022508E7DFF81D
:101740007090002539F9023B00EE103AE8B2B8EE8D
:10175000C00A0135FDF712F9042DF3D1284693E7AD
:1017600008F076FA059B1F78102F05BFDFF8208060
:1017700094F8F91494F8F914A8F800108146FEF7CB
:10178000A5BC00BF32650020B0A0002000001644B8
:10179000F884002038990020289900208ABA002077
:1017A00000007A440008ED465E7B002006470020DA
:1017B0000A470020D94B1A46B2EC011A93ED033ABE
:1017C000D2ED002AD3ED094AD3ED021A93ED082A8F
:1017D000D3ED053A93ED074A93ED0B5AD3ED0D5A2D
:1017E00093ED0F6AD3ED116A93ED137AD3ED157A69
:1017F00093ED049AD3ED068A93ED0A0AD3ED0C0A11
:1018000093ED0E8A62EEA22A23EE033A64EEA44A16
:10181000E1EE012A102FA1EEA13AE2EE024A93ED89
:10182000101A93ED142AD3ED121A63EEA33A24EEA4
:10183000044A25EE055A65EEA55A26EE066A66EEBE
:10184000A66A27EE077A67EEA77AE9EE093AE2EE92
:10185000027AA8EEA84AA0EE005AE0EEA05AA8EE3E
:10186000086AE1EE016AA1EEA17AB1EEE22AF1EE98
:10187000C32AB1EEE33AF1EEC43AB1EEE44AF1EE36
:10188000C54AB1EEE55AF1EEC65AB1EEE66AF1EE9E
:10189000C76AB1EEE77A03ED1E3A43ED1D3A03ED58
:1018A0001C4A43ED1B4A03ED1A5A43ED195A03ED46
:1018B000186A43ED176A03ED202A43ED1F2A03ED52
:1018C000167AD3ED175A93ED196AD3ED1B6A93ED8F
:1018D0001D7AD3ED1F7A93ED1E5A93ED163AD3ED90
:1018E000183A93ED1A4AD3ED1C4A65EEA55A26EE36
:1018F000066A66EEA66A27EE077A67EEA77AE3EE37
:10190000035AA3EEA36AE4EE046AA4EEA47AE5EE19
:10191000057AB1EEE55AF1EEC65AB1EEE66AF1EE9D
:10192000C76AB1EEE77A03ED155A43ED145A03ED99
:10193000136A43ED126A03ED117A01F0DC8194F829
:10194000F934013384F8F934754B764D1B782F88C0
:10195000591C07EE907A0F29B8EE670A01F3A180AF
:101960000C2B04EB830203F10200DFED6F5A00F24F
:10197000798702F2145203F5A373D2ED007A069E22
:10198000B0EE656A04EB830300222EE027EEA77A0F
:10199000B4EEE65A27EE277A66EEA67AF1EE10FA52
:1019A00076EEA64A00F10101A7EEA67A27D4D3ED80
:1019B000017A26EEA67AF4EEE74A67EE266A27EE6B
:1019C000A77AF1EE10FAE7EE876A08D507EE101A4B
:1019D000B8EEC77A36EE266AE6EE875A324602300D
:1019E0000E2803F1080300F34087D3ED006A37EEB9
:1019F000A75A26EEA67A002AC8D027EE267AD3ED7B
:101A0000017A05EE100A67EEA76AB8EEC55A36EEFF
:101A1000076A66EEA76AE5EE075A411CD6E7D4F8D6
:101A20000425B4F80815414834F03CFF059B1F78A5
:101A3000102F01F0498194F8F934013384F8F93416
:101A40003A4BB4F8FC04D4F810251946B1EC016AFD
:101A5000D1ED007A77EEA77AF0EE006AB0EE677A01
:101A6000A6EE267A013803EBC001D6EE267A0839B5
:101A70001032F6EE003A27EE237A67EEA37A83ED72
:101A8000207AC3ED217A103391ED027A91ED036A49
:101A900053ED016A53ED027A52ED014A12ED025AFA
:101AA00037EE674A76EEC65A77EE277AE4EE845A26
:101AB0000138A1F10801E5EE047A02F1080203F110
:101AC000080336EE267AE4EE877AE5EE475A67EEAB
:101AD000A37A25EEA37AC3ED1C7A83ED1D7AD3D1C8
:101AE000102F00F0AF8794F8F914114B0693114BA7
:101AF00094F8F8240131A3FB0103C81A03EB500347
:101B00009B08C3EBC303CB1A013A84F8F93484F879
:101B1000F8240699FDF718BD0020B5E58C9F00203C
:101B2000C6410020C4410020000000000C9F00209E
:101B3000A0A0002025499224B4F8FC14CF48D4F882
:101B400000254FEA510E4FEA8E0600EB8105C908C9
:101B500006EB000300F0A08003EB011C1036A9196E
:101B60000CF1100C1030103302F1100705F11006C3
:101B700056ED032A56ED043A10ED043A10ED032A0F
:101B800056ED026A16ED016A10ED020A10ED018AA7
:101B900011ED044A11ED035A53ED044A53ED035A73
:101BA00013ED027A53ED017A51ED020A11ED011A9B
:101BB00073EE238A72EE221A40ED048A40ED031A76
:101BC00070EE268A78EE061A40ED028A40ED011A80
:101BD00074EE848A75EE851A43ED048A43ED031A88
:101BE00077EE208A77EE811A43ED028A43ED011ADF
:101BF00073EE633A75EE655A17ED035A32EE623AA8
:101C000074EE644A65EE631A17ED044A23EE052A62
:101C100064EE652AE3EE041A10339C4524EE843A00
:101C2000A3EE842A00F1100007F11007A5EE853A13
:101C300006F1100601F11001E4EE852A46ED071ABF
:101C400006ED082A01ED073A41ED082A57ED055A3D
:101C500017ED065A70EE666A38EE466A30EEC77ABD
:101C600071EE677A26EE253A65EEE63A25EE674A8A
:101C700067EE054AE6EE053AA6EE853AA7EE254A56
:101C8000E7EEA54A06ED063A46ED053A01ED064AAD
:101C900041ED054A7FF46CAF1FFA8EF63146774866
:101CA00029F0D2FB31462846D4F8002529F0CCFB98
:101CB000059B1F7814E7724A94F8FA34069294F858
:101CC000742302F1DE05C2F12002D0B205EB43130A
:101CD000860804EB830500F0C187360106F1100C7D
:101CE0006849694AAC4405F1100313ED024A13ED4B
:101CF000035A13ED017A13ED046A51ED024A51EDD6
:101D0000035A51ED046A51ED017A64EE244A65EEFE
:101D1000255A66EE266A67EE277A10339C4542ED17
:101D2000024A42ED035A42ED046A42ED017A01F1A2
:101D3000100102F11002D8D1544B504935449A1980
:101D40000E4410F003011BD095ED007AD2ED007A1D
:101D500067EE877A0129C6ED007A11D095ED017AF8
:101D6000D2ED017A67EE877A0229C6ED017A07D0B3
:101D700095ED027AD2ED027A67EE877AC6ED027AA5
:101D800094F87453002D40F08F86102F00F01287C6
:101D900094F8F914ABE694F8FA543D4A04EB450381
:101DA000D2ED007AB3F8803608EE103AB8EEC87A71
:101DB00067EE277A17EE900A34F040FF0022354B89
:101DC00006460F4635F018FA08B9324F0026394654
:101DD000304635F063FA07EE900AB8EE480A67EE2F
:101DE000E70A2D4B264A0692E0EE000A05EBC505F0
:101DF00003EB850567EE807A2846C7EEA00A1168D6
:101E0000D5F818A0D5F81C802E6A95ED058A2AF021
:101E10008BF9059B85ED058A1F78C5F818A0102F52
:101E2000C5F81C802E6200F07A8794F8FA341B4AB9
:101E300094F8F9140133A2FB0302520802EB4202A8
:101E40009B1ADBB2013184F8FA3484F8F91436E7CE
:101E5000134B1B78DB0700F121872B79012B00F056
:101E60000F86022B7EF495AC0E4B1B78002B7EF474
:101E700090AC13F0DDF9FEF78CBC00BF0C9F002086
:101E8000A0A00020D84100201C9F0020C8410020B5
:101E90004842002000405A40709C0020ABAAAAAAE9
:101EA0005E7B00202D460020A14BDFF8BC825B68E2
:101EB000D8F80010C8338B4204D31DF01DFB002856
:101EC0004AD0AA78032A00F042872B790122934254
:101ED0003270C6D1974B1B78D80740F1D385DBF819
:101EE0003011D8F80020337891423CD8012B3EF4D1
:101EF00050AC914F3A78002A3EF44BAC0B2B0DD8E6
:101F000001229A4040F6030112EA01050CD112F4B5
:101F1000C06F03D0093B012B40F24787844BD8F8B0
:101F200000205A600B23337000233B70FEF731BC56
:101F3000824B1B78002B00F02486162032F0B8FB71
:101F4000002840F01E867C4B1B78002B40F0198641
:101F50000923337012F0EEF92B79012B3DD0022BBF
:101F60007EF417AC3378012B7EF413AC7CE716209B
:101F700032F09EFB0028EDD0714B1B88002BE9D17D
:101F8000704B45201F681DF0DBFA0E201DF0D8FABB
:101F9000384612F0DDF8079F384612F0D9F86A4A41
:101FA0006A4B12681A6038460A23337013F04CFEED
:101FB000D0E71DF081FA12F0F3F90028CCD01DF023
:101FC0009BFA0028C8D0604A604B12681A600A2346
:101FD00033702B79012B7EF4DCABDFF88C8179E751
:101FE0001DF06AFA5A4B052000210090A3F1080267
:101FF000CDE90111532012F009FF0028ACD14C4A61
:10200000082310603370E4E71DF056FA514A02923B
:10201000A2F10C03072101930091A2F10803002112
:10202000143A472012F0F2FE002895D1404B0022CE
:102030004FF0FF311A60072259603270C9E71DF076
:102040003BFA454B022000210090A3F10802CDE9A4
:102050000111482012F0DAFE00287FF47DAF344BE6
:102060004FF0FF310622186059603270B1E71DF061
:1020700023FA3A4A0292A2F10C032921019300911A
:10208000A2F10A035021163A492012F0BFFE00289F
:102090007FF462AF324B1B681F06C7D5244B4FF04D
:1020A000FF31052218605960327092E7204FDFF847
:1020B000B8801DF001FA7B68D8F8002064339342A1
:1020C000BFF44AAF40201DF0DBF900287FF444AF95
:1020D0003B68DFF89880DFF88CA04FF040090DE0F6
:1020E0001DF02EFADAF800203B68013A0133B9F10D
:1020F0000109CAF800203B6000F0798643441B7E4A
:102100001846002BECD100234FF0FF323B60042334
:102110007A6033705DE7DFF85080054AD8F8003008
:10212000536010490023136003220B60327050E7A4
:102130007C4400205E7B00202D4600201F460020AE
:102140006844002064440020584400205444002087
:10215000DC93040894930408789304089A91040883
:10216000B0A0002000650020408500201C910408DC
:102170000AD7233CF8EEE77A012300219D42C4ED03
:102180001A7AC4ED1E7AC4ED1D7A2162E167C4F8A3
:10219000843000F0F983B4F9523007EE903A01220E
:1021A000F8EEE77A00239542C4ED1B7AC4ED237A5A
:1021B000C4ED227A6362C4F89030C4F8982000F02D
:1021C000E180B4F9543007EE903AF8EEE77A002255
:1021D0000123C4ED1C7AA262C4F8AC300023012DA7
:1021E000C4ED287AC4ED277AC4F8A4307DF416AF84
:1021F00007EE906AD4ED1C5A099B5FED236AB3F990
:102200001430BA4AA8F80600B8EEE76A07EE103AAA
:10221000C5EE867AB64B11781B680022B8EEC77AF5
:10222000E7EE667AC4ED0A7A9A62C3E90B2229B115
:10223000B04B1B6833F400637DF4F2AE012024F050
:1022400039FEFDF7EDBE94EDBE8AD4EDBF6A94ED84
:10225000C70AD4EDC24A94EDC87A94EDC35AD4EDBE
:10226000C67AD4EDC55A94EDC46A94F87453DFF875
:10227000948268EE266A04EB8503A4EEA60A002287
:102280000F2FA5EE267A84F8F422B8F9040083ED26
:10229000DE0A67EEC07AA5EEC07AE6EE267A84ED15
:1022A000C77AC4EDC87A00F06A8594EDC05AD4EDBF
:1022B000C10AD4EDD04A94EDD97A94EDCB1AD4ED7D
:1022C000D41AD4EDD15A94EDD54AD4EDDA6A94ED0E
:1022D000CC2A94EDCF6AD4EDD87AD4EDCE2A94ED01
:1022E000CD3AD4EDD73AA8F8040028EE055A28EEE6
:1022F000208AE1EE054A6B1C04EB8501A8EE217AE9
:1023000003F01F0305F16002E8EE046A84F87433F9
:102310000C23E2EE055A04EB820284F8F83426EE30
:10232000646A67EEC77A94EDD64AC1EDFE4AE2EEE2
:10233000E45A0599A3EE056A00230F78C4EDD05A3C
:10234000E7EE636AC4F8FC32C4F80033E8EE047ABE
:10235000C4F8043384EDD16AC4EDD96A82EDBE7A43
:10236000C4EDDA7AFDF7ABBEB5F91490FEF7D4BD33
:102370000023012DC4ED237AC4ED227AC4F89030F5
:102380007DF419AE07EE906AD4ED1B6AF8EEE77A99
:10239000B54286EEA77A84ED097A7DF40CAE10E79B
:1023A0009A457DF4FBAE4EF806A00246BAF1000F46
:1023B0003DF4F4AEF0EE40DAD7EEA6DA4E4BD3EDB4
:1023C000006A9FED4E7ADFED4E7A6DEEA6DAB0EE42
:1023D0004C8AF4EEC7DAF1EE10FA88BFF0EE47DA75
:1023E000F4EEE7DAF1EE10FAB8BFF0EE67DAFDF7D7
:1023F000FFBEF0EE48DAD5EEA6DA3F4BD3ED007A19
:102400006DEEA7DA4FF0000A84ED01CAFDF7F3BEC6
:10241000012B40F3B98207EE101AB8EEC77AC7EE67
:10242000876AB1EEE68A132A17D047B107EE907A91
:10243000F8EEE77AF4EEC87AF1EE10FA29D407EE56
:10244000906AD4ED1A6AF8EEE77AB54286EEA77A7A
:1024500084ED087A7DF47CAD9DE6B0EE480A35F057
:1024600025FB00B2E1E7012A8CDD07EE103AB8EE59
:10247000C77AC7EE876AF1EEE67A002F82D007EEC0
:10248000107AB8EEC77AF4EEC77AF1EE10FA7FF759
:1024900079AF099B05999A8B0F78A8F8060042F24C
:1024A000107303FB02F3069A06991268B3FBF2F36A
:1024B000C4F8B030FDF748B8012A7FF799AE07EEAF
:1024C000103AB8EEC77AC7EE876AF1EEE67A002FC7
:1024D0003FF48EAE07EE107AB8EEC77AB4EEE77A24
:1024E000F1EE10FA7FF584AED3E700BFB6410020CD
:1024F00020840020047E002008C0002000007A44D0
:1025000000007AC4F8840020EE4BEF49D3ED016A55
:1025100093ED022AD3ED032A67EE266AE4EE826A7F
:10252000E5EEA26AF7EE002AF5EEC06AF1EE10FAC7
:1025300048BF66EE836A67EEA66AF4EEE26AF1EEE1
:1025400010FA88BFF0EE626AF0EE452AE3EEA62AA2
:10255000B4EEE26AF1EE10FAF0EE626A9ABFF3EEC0
:10256000042A76EEE26AF0EE446A012AC1ED006ABE
:102570003EF4E6A8D3ED056A93ED062AD3ED072ACB
:1025800067EE266AE4EE826AE5EEA26AF7EE002ABA
:10259000F5EEC06AF1EE10FA48BF66EE836A67EEA8
:1025A000A66AF4EEE26AF1EE10FA88BFF0EE626A13
:1025B000F0EE452AE3EEA62AB4EEE26AF1EE10FA56
:1025C000F0EE626A9ABFF3EE042A76EEE26AF0EE6B
:1025D000446A022AC1ED016A3EF4B2A8D3ED096A49
:1025E00093ED0A2AD3ED0B2A67EE266AE4EE826A9F
:1025F000E5EEA26AF7EE002AF5EEC06AF1EE10FAF7
:1026000048BF66EE836A67EEA66AF4EEE26AF1EE10
:1026100010FA88BFF0EE626AF0EE452AE3EEA62AD1
:10262000B4EEE26AF1EE10FAF0EE626A9ABFF3EEEF
:10263000042A76EEE26AF0EE446A032AC1ED026AE9
:102640003EF47EA8D3ED0D6A93ED0E2AD3ED0F2A4A
:1026500067EE266AE4EE826AE5EEA26AF7EE002AE9
:10266000F5EEC06AF1EE10FA48BF66EE836A67EED7
:10267000A66AF4EEE26AF1EE10FA88BFF0EE626A42
:10268000F0EE452AE3EEA62AB4EEE26AF1EE10FA85
:10269000F0EE626A9ABFF3EE042A76EEE26AF0EE9A
:1026A000446A042AC1ED036A3EF44AA8D3ED116AD4
:1026B00093ED122AD3ED132A67EE266AE4EE826ABE
:1026C000E5EEA26AF7EE002AF5EEC06AF1EE10FA26
:1026D00048BF66EE836A67EEA66AF4EEE26AF1EE40
:1026E00010FA88BFF0EE626AF0EE452AE3EEA62A01
:1026F000B4EEE26AF1EE10FAF0EE626A9ABFF3EE1F
:10270000042A76EEE26AF0EE446A052AC1ED046A14
:102710003EF416A8D3ED156A93ED162AD3ED172AC9
:1027200067EE266AE4EE826AE5EEA26AF7EE002A18
:10273000F5EEC06AF1EE10FA48BF66EE836A67EE06
:10274000A66AF4EEE26AF1EE10FA88BFF0EE626A71
:10275000F0EE452AE3EEA62AB4EEE26AF1EE10FAB4
:10276000F0EE626A9ABFF3EE042A76EEE26AF0EEC9
:10277000446A062AC1ED056A3DF4E2AFD3ED196A59
:1027800093ED1A2AD3ED1B2A67EE266AE4EE826ADD
:10279000E5EEA26AF7EE002AF5EEC06AF1EE10FA55
:1027A00048BF66EE836A67EEA66AF4EEE26AF1EE6F
:1027B00010FA88BFF0EE626AF0EE452AE3EEA62A30
:1027C000B4EEE26AF1EE10FAF0EE626A9ABFF3EE4E
:1027D000042A76EEE26AF0EE446A072AC1ED066A40
:1027E0003DF4AEAF93ED1D2AD3ED1E2AD3ED1F6A43
:1027F00027EE027AA4EEA27AA5EEA67AB5EEC07A0A
:10280000F1EE10FA48BF27EE037A27EE877AF7EE4B
:10281000007AB4EEE77AF1EE10FA88BFB0EE677A8C
:10282000F0EE457AE3EE877AB4EEE76AF1EE10FA5D
:102830003EF617AEFEF711BE28461546FEF72FBF2F
:10284000079AC4F8E422FEF7C0BA079AC4F8EC224B
:10285000FDF78ABA0546FEF77FBE0327042202254C
:10286000FEF776BEB0EE656A002201F5A27304EBB6
:10287000830306980CE026EEA77A07EE901AF8EE8E
:10288000E77A36EE076AE7EE275A02460F291DDC83
:10289000D3ED017AB3EC017A013137EE075A67EED6
:1028A000A76A002AE7D1B4EEE75A67EE076AF1EEAD
:1028B00010FA27EEA75A26EE877AE7D5A5EE277AF3
:1028C000DBE700BF64C00020E4460020B5EEC06A2C
:1028D000F1EE10FA40F3E58085EE868AE24BF7EEE2
:1028E000007A38EE678AD3ED007A68EE277AFDEE3B
:1028F000E77A17EE903A7C2B40F33D81BB42A8BFAC
:102900003B4607EE903AB8EEE70A94F8FA0424231F
:1029100003FB004000F21460F5F722FDFDEEC07AE3
:102920002B8817EE902A7C2A40F38A809342A8BF16
:10293000134607EE903AF8EEE77AFCEEE77A17EEE8
:10294000903A9BB2059994F8FA240F7804EB42016F
:10295000A1F8803612B90F2F00F07081112F7FF48B
:10296000BFA8DFF8108394F8F91428F81230BF4B91
:102970000693FFF7BCB80023012DC4ED1E7AC4ED09
:102980001D7AE3677DF4E4AA9FEDB98A4BE55B42CB
:102990000AFB03F381FB03C1DB17C3EB2113121AFC
:1029A0009E441344CE44A8EB0308A4F802E0A4F824
:1029B0000080FEF753B8002A00F0E080B4F90A3036
:1029C00013600120FEF760BE059B1B78262B7DF46B
:1029D0009DA8B0EE490A8DED0F6ACDED0E7A35F067
:1029E00065F8DDED0E7ADFF88CA227EEAA0AAAF8C8
:1029F000000035F05BF8B0EE4F0AAAF8020035F09F
:102A000055F89DED0F6AAAF80400FDF77FB8B2EE05
:102A1000049A20EE090A35F049F8964B0E93B0EE71
:102A20006D0A1880A3F802A035F040F80E9B28EE3E
:102A3000090A988035F03AF80E9BD880FDF755BB0F
:102A40007D237FE707F004F9059BDFF828821F78D4
:102A5000864B94F8F9140693A0EB0900A8F802003D
:102A6000FFF745B80F2F00F01181112F7CF429AD2D
:102A7000B0EE480A35F01AF87E4BD880FCF721BD3D
:102A8000DFF8048232F0FEFA00283FF428AAD8F8D2
:102A90000020337802F59C520832CBF83021FFF742
:102AA00062BA9FED738A30E794F8FA64800000F20E
:102AB000145E04EBC6165FEA95081844A64406F5B2
:102AC0005E7634D04FEA081808F1100CB44406F1D1
:102AD000100300F110010EF1100213ED024A13ED84
:102AE000035A13ED017A13ED046A51ED024A51EDD8
:102AF000035A51ED046A51ED017A64EE244A65EE01
:102B0000255A66EE266A67EE277A10339C4542ED19
:102B1000024A42ED035A42ED046A42ED017A01F1A4
:102B2000100102F11002D8D146444044C64415F0C9
:102B300003053FF42AA996ED007AD0ED007A67EEFE
:102B4000877A012DCEED007A3FF41FA996ED017A28
:102B5000D0ED017A67EE877A022DCEED017A3FF44F
:102B600014A996ED027AD0ED027A67EE877ACEED5F
:102B7000027AFFF70AB99FED400AC6E60120FEF788
:102B800083BD079813F060F8FFF7E4B9059B1F7841
:102B90000F2F00F0BA80032F35683DF42FAD89ED7B
:102BA000028A05F00055FCF7B7BC0527062204256C
:102BB000FEF7CEBC07F04CF8DFF8B880059B94F820
:102BC000F9141F78A0EB0900A8F80200FEF78FBFE8
:102BD0000699D1ED027AF0EEE77AFCEEE77A4FF64D
:102BE000EF7217EE903A103B9BB293421AD9D1ED97
:102BF000017AF0EEE77AFCEEE77A17EE903A103BB6
:102C00009BB293420ED9D1ED037AF0EEE77AFCEE57
:102C1000E77A4FF6CC7217EE903A333B9BB2934271
:102C20003EF662ACDBF82431002B59D1079B03F54B
:102C30009233F833CBF82431FEF759BC9FED0F0ADD
:102C40000A4B069328EE000A34F030FFDFF82480A8
:102C500094F8F914A8F80600FEF749BF084B094E8E
:102C60001A46FFF76EB800BFC0410020A0A00020A8
:102C700000000000F88400200000FA420000C84272
:102C8000C84100200C9F002040850020B0EE480A7B
:102C900034F00CFF594B1880FCF713BC2BF088FE66
:102CA000074668B1DFF87881D8F80030834274D0E5
:102CB000D8F8DC30BB4267D0D8F8B8319F4255D045
:102CC00012F074F9FFF748B906F0C2FFDFF82C8163
:102CD000059BA0EB09001F78A8F80200FEF7ABBE29
:102CE000079A9A427EF603AC202025F02FFCFCF7D1
:102CF00093FAFEF7FCBB06F0ABFFDFF80081A0EB18
:102D00000900A8F80400FEF71ABE34F0CFFE3568BB
:102D10003A4B05F0005558802B46FCF7F7BB06F000
:102D200097FFDFF8D880059BA0EB09001F78A8F873
:102D30000200FFF77AB831F063FE00287EF4B4ABEE
:102D400032F0F2FA00283DF4E0ACFEF7ADBB2C4FB8
:102D5000386823F074FE2B4B1B780022022B3A605C
:102D60007FF4B3A824F018F8FFF7AFB8384623F083
:102D700066FEDC220021244834F082FDA0E734F016
:102D800095FE00B2FFF791BA384623F058FEDC22D8
:102D900000211E4834F074FD8EE723F050FEDC2243
:102DA0000021404634F06CFD82E745201CF0C8FB52
:102DB000FF201CF0C5FB16481CF0AEFB28461CF09B
:102DC000BFFBFFF7ABB8134BD4ED01EA1A78124BF7
:102DD000B1EE68EA93ED006A002A7DF415ADB0EE1D
:102DE0004E9AB0EE4EFADFED0DDAFCF7C7BE434463
:102DF0001B7E002B7FF4B0A8FFF785B9F884002074
:102E0000046500209B440020FC97002020970020B0
:102E1000ECCE04084CBF00200CC0002000000000D5
:102E2000449600202DE9F04F83B01C4606468846A4
:102E3000174606F00DFF8A4B1B78002B72D02F2F00
:102E400070D8DFF83CA2DAF80430002B6AD1152FD5
:102E50006BD80123834903FA07F20A4240F0ED8060
:102E6000814912F03E0F9B460CBF4FF47A730B461C
:102E70000193002C5FD100F51C501030019BCAF863
:102E800004008AF80DB0CAF80830B8F1000F47D036
:102E900042463946754834F0F3FC754A1389B8F157
:102EA000010FB3FA83F34FEA531335D0B2F8681029
:102EB000002918BF0023B8F1020F2DD0B2F8C810B6
:102EC000002918BF0023B8F1030F25D0B2F828114C
:102ED000002918BF0023B8F1040F1DD0B2F88811E3
:102EE000002918BF0023B8F1050F15D0B2F8E8117A
:102EF000002918BF0023B8F1060F0DD0B2F8481210
:102F0000002918BF0023B8F1070F05D0B2F8A82296
:102F1000002A08BF1C4600E01C4684F00104E4B20D
:102F20008AF80C4003B0BDE8F08F4FF47A73019338
:102F30004FF0010B9DE708F1FF3942F228305FFAAC
:102F400089F906F0D7FE09F10109CDF800804FF4A8
:102F50007A7006F0CFFE009B002B58D0454DDFF86D
:102F60002481002404E001344C4505F160054ED075
:102F7000E3B29E4201D0FF2EF5D13D4963001A19FC
:102F800001EB42124FF0010C82F814C0297AB8B25A
:102F90000029E8D0DAF8041031B19AF80C1019B908
:102FA0009AF80D10002940D1314AA880234402EB41
:102FB00043134FF0000C1A7D98F8001083F814C0EA
:102FC00042EA4000021282EA101242402A4B02F00A
:102FD0000F0242EA00121B68002934D1012105F1D9
:102FE00014009847E9682B68B5F806C0B1F82C21A1
:102FF000DB6842EA0C02A1F82C2158601A680134FF
:1030000042F001024C451A6005F16005B0D1002084
:103010000BF1FF3BF5F76CFD1BF0FF0B97D101980F
:1030200003B0BDE8F04F06F065BE14492144887A2C
:103030000028B9D082F814C0B6E74FF47A73019330
:103040004FF00A0B15E72868E968407900F0FC00AA
:103050000C30084404219847EB688000188182E70F
:10306000CCA2002080173000A08601009A2B0020FF
:10307000E0A20020E4A20020D4A20020902B002097
:103080008C2B0020DCA200202DE9F0472DED028BD7
:10309000BE4D2B78002B7FD1BD4C2378D90724D48B
:1030A000FBF71EFFBB4B1A685ABB2378DA0703D520
:1030B000BDEC028BBDE8F08706F0CAFDB64BB74AFF
:1030C0001B68C31A934206467BD8DFF8E092D9F812
:1030D0000030002BECD11E2032F08AF8002840F09E
:1030E00049810123C9F80030E2E7AD4AAD4B1178C0
:1030F000186801F0010109F0FBFFA64B1A68002ACD
:10310000D3D0A94BA9491B780020086023B1A84B54
:10311000D3F8B030002BCBD1A64C002A92FAA2F300
:10312000B3FA83F3D4F8382108BF4FF0FF330133EB
:103130009A42BDD0A048C4F83831DBB2A0FB0320CE
:1031400080089E4900EB80029B1A43F205254FF050
:103150000534DBB200F0FF020D81C1E90044002814
:1031600000F076811920012A887200F0C180023AAD
:10317000D2B20732C872044652000C200C54451CCF
:103180000230824201EB000600F0EF80402806F892
:10319000014CF3D10246B7E0834A1378002B7FF449
:1031A0007BAF8749874B888B1C68814942F210733B
:1031B00003FB00F30120B3FBF4F31070C1F8B0304F
:1031C0006AE7814BDFF828A21B78DAF80080002B31
:1031D00040F01081DFF8D491764F94F800C07B4B1B
:1031E00000224CF003012170C9F8002003F178019E
:1031F000C7F80421C7F8082102E0063399420DD030
:103200001A781F2AF9D19878DA78904202D35A793D
:10321000002AF2D04CF0070C84F800C06C4AB2F9D6
:103220000030002BB8BF5B42B3F5E17F3DDAB2F965
:103230000230002BB8BF5B42B3F5E17F35DA654B56
:10324000654C93ED057AD3ED077AD3ED096A93EDDA
:10325000030A77EEA67A30EE070AF7EE000AB0EE20
:10326000007AE7EEC70A30EE000AF7F7FDF9BEEE86
:10327000008A20EE088AB0EE480AF7F763FAFDEEFE
:10328000C87A84ED010A17EE903ADFED547A2033C4
:10329000402BC4ED027AC4ED037A00F2C380B0EE95
:1032A000480AF7F76FF984ED040A6B78DFED4C6A92
:1032B00007EE103A07EE906AB8EEC77AF8EE677A32
:1032C0000023E7EE267A18F0800FC7F83831FCEEBD
:1032D000E77AC7ED4D7A3DD0424B1B789B0739D535
:1032E000414B9B7C042B35D9062023F0E3FD34E0D1
:1032F0003222CA720C20002B3FF44CAF0524012B64
:103300000C5400F1010208D1FF238B54BDEC028B59
:103310000E20BDE8F04723F0CDBD851C19263E2DBB
:103320008E5400F2A380022B4C5500F10302EBD027
:10333000051D3E2D8E5400F29980032B4C5500EB59
:103340000402E1D0831D3E2B8E5400F28D80C21DFD
:10335000CC54D9E7052023F0ADFD0023C7F83C315C
:10336000C7F84031C7F82431A2E632243E2A4C5532
:10337000C1D9C9E71E211D48F7F7E6FA00283FF436
:10338000B0AE0223C9F8003092E600BF9844002096
:103390005E7B0020047E00202C6500207F4F120001
:1033A000098500200C850020B64100204C7E0020BD
:1033B000F89900208C2B0020CDCCCCCC504C002098
:1033C00080A00020A0A00020CCA200206447002004
:1033D000F47B002074260020200000200000000064
:1033E00000247449247E00200C7E00204C440020E0
:1033F000B0A000201E2031F0FBFE00283FF4EAAE12
:103400001E211B48DFF87890F7F79EFA08F48053E6
:1034100058B9D9F80020022A07D0164A1070CBB14B
:10342000154FDAE6B0EE670A3DE7124A124F012166
:103430001170002287F82121002B7FF4CEAE0F4AB5
:10344000FF2011781522FFF7EDFCDAF80080C4E6C2
:103450000A2050E7094A084F1178FF201422FFF78D
:10346000E1FCDAF80080B8E61A464DE72A464BE759
:103470004C440020326500208C2B0020F571002088
:103480004C7E00202DE9F04FDFF84CC204460A3094
:103490000CEB000E87B09EF80C801CF80090039196
:1034A0004FF41A7C404601920CFB04FA049305F099
:1034B000BDFE0646484605F0B9FE0090404605F0C0
:1034C00017FA9DF84450804B0590484603F5A27BBF
:1034D00005F00EFA15F008039DF8407002930BEB0F
:1034E0000A08DDE9001200F09180002900F0E58073
:1034F00091F807C01CF0020F40F0DF80724B03EB25
:103500000A0C07F002030093CCF88411CCF8800178
:10351000CCF87C0130B14FF00B0C04EB0C0180F8BF
:1035200006C0C171684B049E4FF41A7909FB043937
:103530000AF1480089F84871039FC9F8707158442E
:10354000624FC9F844710AF5A47100275944C9F8BB
:1035500058014FF48070C9F8742189F84951C9F8AD
:103560005C11C9F85001C9F854013146D9F88401F9
:10357000C9F84C6189F89C43C9F86471C9F8607155
:10358000C9F86C71C9F86871C9F89873A9F8907393
:10359000FBF7FEFA05F00101D9F8840128F034FBAD
:1035A000009A4B484B49C9F8A4730AF519750AF5F6
:1035B00017735D44C9F8A803C9F8A0139B44002AF7
:1035C0005CD0D9F88801002858D0D9F88421036844
:1035D0001268934252D0012389F89D333146FBF79C
:1035E000D7FA5946D9F8880128F072FA3A4629469E
:1035F000D9F8840105F05AFC029B002B4FD04046BD
:10360000FBF79CFA404607B0BDE8F08F17F00103C6
:10361000019318D117F00203009383D0B9F1000F82
:103620004BD0294B4FF41A7C0CFB043C019BCCF88B
:103630008001002B3BD100293FD0CCF88411002819
:103640007FF469AF6EE7002E37D096F807C01CF004
:10365000020F32D11C4B03EB0A0C059BCCF87C31DA
:10366000059BCCF88461002BD4D04FF00C0E04F1F4
:103670000B0C83F806E083F807C0CBE7124A4FF43F
:103680001A7303FB0424002384F89D335A46294609
:10369000D4F8840105F00AFC029B002BAFD1404610
:1036A000FBF792FA01214046FBF798FAA7E7CCF81E
:1036B000881100287FF42FAF34E74FF00008404610
:1036C00007B0BDE8F08F00BF8C2B0020FC930408EE
:1036D00085EA0008F5EB000898AF002030B4454BB0
:1036E0001B78012B14BF0024032439B30429038C55
:1036F00047D0082961D023F480531B041B0C03849A
:10370000838B058C40F6FF41194045F6FF732B4033
:1037100043EA023241F4807192B241EA043142F448
:10372000805281830284838B23F440631B041B0C2F
:103730008383838B9BB2838330BC7047018C21F0E1
:1037400001010904090C0184018B038C89B223F067
:103750000A0321F0F3011B0442F0010241F00101D0
:103760001B0C134341EA041101830384038B23F0F0
:103770000C031B041B0C0383038B9BB2038330BC21
:10378000704723F010031B041B0C0384058B038C70
:103790009BB223F0A00340F6FF4143EA0212294006
:1037A00041F4807192B241EA043142F01002018387
:1037B0000284038B23F44063DBE723F480731B0450
:1037C0001B0C0384818B038C9BB223F4206389B28E
:1037D00043EA022221F0F30141F0010192B241EAF1
:1037E000041142F4807281830284838B23F00C03E2
:1037F0009CE700BFB4A00020F8B550F8043C10F8D6
:103800000E4C5E7902461868C4B114460B4632F875
:103810000C1C14F80F7C24F80A3C0D4A5B1A9BB26E
:10382000002524F8083C314622F817302A4604F8CF
:103830000E5CFFF753FF04F80D5CF8BD012302F89E
:103840000E3C22F80C1C31460222BDE8F84045E748
:10385000EC3F0020134B1A680AB1002111609A69ED
:103860000AB1002111601A6B0AB1002111609A6C33
:103870000AB1002111601A6E0AB1002111609A6F1D
:103880000AB100211160D3F890200AB10021116023
:10389000D3F8A8300BB100221A60034B00221A7033
:1038A000704700BFF0A1002064AF00202DE9F04F69
:1038B0000C68B94EB94F25883668B6FBF2F285B070
:1038C000013B013ABC429BB292B2ADB2BDF8388026
:1038D0009DF83CC011D0B24EB4420ED0B4F1804F2E
:1038E0000BD0A6F58036B44207D006F58066B44208
:1038F00003D006F58066B44202D125F07005ADB262
:10390000A84EB44211D006F58066B4420DD025F41D
:10391000407506F56C46ADB2B4422580E36222855F
:1039200040F04E810023238602E02580E362228559
:103930000123A3824A79CB79BCF1000F01D083F037
:10394000010313F0020140F0FA804FF480665B003F
:1039500003961026019603F00203029189468B46D6
:103960004FF480454FF4805E4FF480764FF0010CA9
:103970000C2A00F2CA80DFE802F098C8C8C869C8FB
:10398000C8C837C8C8C80700218C844E21F48051AC
:103990000904090C2184B4F820C0A788A18B1FFA60
:1039A0008CFC21F4E6412CF4005C09044EEA0C0E78
:1039B000090CB4424EEA0333BFB241F4C04100F0F7
:1039C000CF8006F58066B44200F0CA80A780A1834C
:1039D000C4F840802384A38B23F400631B041B0CD6
:1039E00043F40063A38396E0258C6C4F25F4807527
:1039F0002D042D0C2584B4F820A0B4F804C0A58BA8
:103A00001FFA8AFA25F073052AF4007A2D0446EA93
:103A10000A062D0CBC4246EA03231FFA8CFC45F033
:103A2000600500F0C1805E4EB44200F0BD80A4F895
:103A300004C0A583C4F83C802384A38B23F008032F
:103A40001B041B0C43F00803A38364E0218C534D3B
:103A5000019F21F010010904090C2184B4F820C051
:103A6000A688218B1FFA8CFC21F4E6412CF0200C57
:103A7000090447EA0C07090CAC4247EA0313B6B243
:103A800041F4C0417BD005F58065AC4277D0A6807B
:103A90002183C4F838802384238B23F400631B0420
:103AA0001B0C43F40063238335E0218C3B4D21F054
:103AB00001010904090C2184B4F820E0A788218BB6
:103AC0002EF0020E21F073014FEA0E4E09044CEA6B
:103AD00003034FEA1E4E090CAC424EEA0303BFB289
:103AE00041F0600140D005F58065AC423CD0A78034
:103AF0002183C4F834802384238B23F008031B0420
:103B00001B0C43F00803238305E0042AC4D0082AD1
:103B100093D0002AF0D0B4F8443043F40043A4F822
:103B200044302188234641F0010123F8341B002151
:103B30009D18C0E90054995005B0BDE8F08F0025EC
:103B4000DB00402703F00809AE46039501952E4699
:103B50002B46AC464FF4806102974FF0040B07E709
:103B600027F480472F4331E74FF6F3751D4027F4C4
:103B7000407745EA0903374343EA0B03B7E723F0ED
:103B80008003029D43EA091323F040032B43039D66
:103B900026F440662E437AE7B0A2002000000140E0
:103BA000000401400010004023F4006343EA0923AD
:103BB00023F480632CF4405C0B434EEA0C0C36E794
:103BC000024B9C423FF4AEAEB2E600BF000401409F
:103BD000F0B583B006460C4605F028FB0546304696
:103BE00004F086FEF8B1F5B1104E01222521706176
:103BF0008171C271022109F0D3F90027DFF838C0C2
:103C00000B4B93FBF4F39BB20A4A0093294692FBB9
:103C1000F4F330469BB20197ACF80040FFF746FE44
:103C200033681F60777403B0F0BD00BF20850020AB
:103C300020A1070040420F0038850020F8B5244C31
:103C400094F8143683B104280ED8224B224E94F8EF
:103C50002C56B4F82E2603EB80000027D0F8100372
:103C60003760B4F8323605B1F8BD07EE902A9FED03
:103C70001B7A9FED1B6AF8EEE77A642267EE877A7B
:103C800007EE100AB8EEC77A02FB030367EE877AE5
:103C900007EE103AB8EEC77AD4F8243687EE870AD2
:103CA0000D4606EE903AF8EE666A66EE866A20EEFB
:103CB000260A33F0FBFED4F81C260A4B10601B6862
:103CC000B4F8301619442944C4F83816F8BD00BFBA
:103CD0008C2B00201C910408907D00200AD7233CE7
:103CE000CA269B3E40850020052819D8052917D8EB
:103CF000884215D070B40B4B01EBC10103EB4101BD
:103D000000EBC00040000E684D688C68CA68C65061
:103D1000184445608460C2600B8A038270BC70479F
:103D2000704700BF065F0020064B074A05288CBF7E
:103D300058785870054B00EBC00003EB4000106052
:103D400031F04EBBE898002038800020065F00204C
:103D50002DE9F04F864B2DED028B1B68DA048DB0F8
:103D6000044600F1D186834B1B78022B00F0DA86E3
:103D7000042B01F06780012B00F042827E4BDFF8BC
:103D80003CA200937D4B7E4A9C42927800F26C826A
:103D9000002A40F06C827B4B019331F0C5FA744BE2
:103DA0001E68009BB3F90670F304804600F180861C
:103DB000754B9B8A6425FF1A05FB07F5C3F5FA636B
:103DC00095FBF3F5642DA8BF642525EAE575EDB2F2
:103DD000019B1A786D4B1B681F0202F0010240F133
:103DE000EF80002A00F0EF80674B1B7FAB4241F26F
:103DF0008B81B8F1000F40F0ED809AF81031002B64
:103E000040F0E880624B63491B680027CF6293F85B
:103E10002C00614B4F608F611F605F609F600028C6
:103E200040F0D8805D4B8AF820011F78002A40F0CE
:103E3000D9805B4B9FED5B7A5B7807EE903AF8EEAA
:103E4000E77A202F67EE877AFCEEE77A17EE905A32
:103E500000F07F82544F2C44CAF83441534B1B78F6
:103E6000002B40F08382484B009A998AB2F90000F7
:103E7000DA8A8142B4BF8023002382420098B0F9DD
:103E80000200C8BF43F040039B088142BCBF63F0FF
:103E90007F03DBB282420098B0F90400C8BF43F050
:103EA00040039B088142BCBF63F07F03DBB28242C8
:103EB0000098B0F90600C8BF43F040039B08814258
:103EC000BCBF63F07F03DBB282429AF84526C8BFCD
:103ED00043F040039A4201F0EE81354A8AF84536B4
:103EE00011780022AAF846268AF84826002901F00F
:103EF000B2815F2B00F03A826F2B00F037822D4B9E
:103F000000221A60019B1A78194BD0071B6807D44E
:103F10009AF8482622B9BAF94626322A01F3818650
:103F2000254A02925C0740F128829AF84A365BB132
:103F3000019B1B78D80707D5134B009A9B8AB2F9CF
:103F400006209A4201F34A8210211048F6F7FCFC41
:103F5000002801F00E809AF850362BB99AF84B36AB
:103F600013B93223AAF84E3601238AF8503604E2F8
:103F7000B0A00020AA3D00208ABA0020404B4C008F
:103F8000607B00205E7B002068AF00204C44002056
:103F900034800020A846002050C00020F584002076
:103FA0009844002000247449B87B0020C06200209F
:103FB000200000204C7E00209C7200208C2B0020D2
:103FC00070023FF50EAF00238AF81031B8F1000FF0
:103FD0003FF418AF01238AF82031B94B1F78002A2B
:103FE0003FF427AFB74B5978002900F0A1819AF828
:103FF0002111002940F09C81B3490978002940F043
:1040000097819AF82211002940F09281AF490978EE
:10401000C90600F18D81DAF83C210292F20601F125
:10402000CD861A790392AA4261D8009AA849B2F9BA
:104030000020B1F812C0A7496FF47A769619B6B28B
:1040400040F2E6308642CCF5FA6B91F800E091F848
:10405000019055D80CEB0E06964281F24387A2EBF5
:104060000C026421A2EB0E0201FB02F2ABEB0E018B
:1040700092FBF1F2D2B20E2A42D8009AB2F9022093
:104080006FF47A70111889B240F2E630814237D865
:10409000B24242F39480A2EB0C02A2EB0E00642227
:1040A000ABEB0E0102FB00F292FBF1F2D2B20E2A50
:1040B00026D8009AB2F904206FF47A71511889B2A7
:1040C00040F2E63081421BD80CEB09018A4242F3F0
:1040D0006580A2EB0C02A2EB09016422ABEB09099B
:1040E00002FB01F292FBF9F2D2B20E2A08D8039A2F
:1040F00052004B2AA8BF4B22D2B2AA4201F26986D3
:10410000754ADFED767A92ED097AB0EEC77AB4EEB1
:10411000E77AF1EE10FA41F15C8692ED047AB0EEA6
:10412000C77AB4EEE77AF1EE10FA41F1528692EDD9
:104130000E7AB0EEC77AB4EEE77AF1EE10FA41F1FA
:104140004886029A0AB9CAF83C415A88DAF83C1102
:10415000DAF840314A2D88BF52084FF47A705B1A62
:10416000234400FB02F2934202D901228AF8212162
:10417000002901F039865A4A9FED5A7A527807EEA3
:10418000902AF8EEE77A202F67EE877AFCEEE77A3E
:1041900017EE905A07D15449544AA1FB03139B09C7
:1041A0000121D3809180524B1E68F2067FF552AEFA
:1041B000464B1B78DB063FF54DAEF7043FF54AAEA4
:1041C00030F01EFC4B4F00287FF445AE3B881E05A7
:1041D0003FF541AE484B1B78002B01F07386B8F1D8
:1041E000000F41F0D28725B1DAF834319C4201F258
:1041F000C687102022F05EFE01238AF844362DE6A1
:10420000DFF828A1DAF83C36E31A002B24DB3B4A1E
:104210003B4B517C2E4A33F81130507C04F59C42C4
:1042200020329908CAF83C2618B1C1F57F730333D0
:1042300099B23448344E0278344D36F812702B68F7
:1042400026F81210DB1B0B44013231492B6002F0BF
:104250000F021B0902700B802E4B00932E4B2F4A2E
:104260009C4292787FF694AD002A00F078872C4B20
:104270002A4A1E780193092092F8215030F018FA4A
:1042800006F00107814620B1264B9B79022B00F0F6
:10429000E583012D40F0E2834FF0000B1F4B224ECF
:1042A00093F82030DFF87C80062B00F2C685DFE82B
:1042B00013F07703B2073003430350036303C503CE
:1042C000F58400207E42002032650020247E0020FC
:1042D00068AF002050640020A84600200000C842BB
:1042E0009844002000247449D34D6210F8840020C3
:1042F000B0A00020B87B0020200000201C870020F8
:1043000040870020AB3D0020B03D0020AC3D0020A8
:10431000D03D00208ABA0020404B4C00607B00203A
:104320005E7B0020A0630020408500208C2B0020B5
:104330001C4B9FED1D7A5B7807EE903AF8EEE77A1A
:10434000202F67EE877AFCEEE77A17EE905A7FF41B
:104350002CAF164B00215960002A3FF47BAD144B63
:104360001E6822E74FF4C873AAF8C030104B114AF8
:104370001B6802925C073FF5D8ADDFF840B09FEDB7
:104380000E8A0DF1200806AD00230422C8F804307F
:10439000069308930A936B600BF178065C460B92C8
:1043A00015E000BF9844002000247449F8840020E0
:1043B000B0A000209C7200208096984A644700209C
:1043C000B9F1280F40F26A810634A64249D06379D8
:1043D000002BF9D194F800900AA84946F6F7B4FAF0
:1043E0000028EDD04946B948F6F7AEFA002840F06B
:1043F0005B814946B648F6F7A7FA002840F04E819F
:1044000005F026FC07EE900AF8EE677AF4EEC87A1B
:10441000F1EE10FAD8DBA278E07882421AD2637803
:104420000099043340F6330C31F913306345A8BFCB
:104430006346B3F5617F4FF0190140F2833CB8BF8A
:104440004FF4617311FB02C29A4203DA11FB00C1FF
:104450009942B9DA21789E480634F6F765FAA64201
:10446000B5D19DF821009DF819109DF818309DF8E0
:1044700020609DF81A2041409DF822008DF8191007
:10448000734042408DF818309DF823009DF81B3092
:104490008DF81A2043408DF81B3001209BF8053021
:1044A0000CA95A0901EB820203F01F0100FA01F185
:1044B000ABB19BF8003052F818CC5E0903F01F0333
:1044C00055F8262011EA0C0F00FA03F343EA020123
:1044D0000ABF22EA030345F8261045F826300BF1FF
:1044E000060B5C45DAD17B4B784A1B7895E80300D4
:1044F00082E80300002B40F08384774B1B78002B6D
:1045000000F0338301217148F6F71EFA3C88002839
:1045100040F01F81714BDB78002B40F01A8124F0B2
:1045200001039BB2A3423B8009D06D4B41F2024193
:10453000FF220E2019809A7022F0BCFC3C88634850
:104540000221F6F701FA23B2002800F00B8123F0D4
:1045500001039BB2A3423B8009D0614B41F202416F
:10456000FF2219800E209A7022F0A4FC3C88A50737
:1045700040F13E8655480A21F6F7E6F9002800F09A
:104580000981200540F1ED8414F0030100F01F8142
:10459000544A554B11785868C1F3400108F0A8FD02
:1045A000524B4FF4FA62C3F8E0201F214748F6F758
:1045B000CBF930B9019A1378590744BF23F00403AB
:1045C0001370029B3C881B6813F00A0F1BD0032159
:1045D0003E48F6F7B9F9002800F0B084660740F1CC
:1045E0004F863A480721F6F7AFF9002800F0948487
:1045F000650640F13D860C213448F6F7A5F9002800
:1046000040F032843C8831480821F6F79DF90028B3
:1046100000F0618144F48073A3423B8008D0304BAA
:1046200041F20241FF220E2019809A7022F042FCD2
:104630002F4B1B78082B00F05A810E2B00F057816E
:104640002C4B1B685C0500F1CB80019B1B78D907C4
:1046500040F1D680284B01241C7028211B48F6F716
:1046600073F99AF80031002868D1002B4AD1002C48
:104670004DD10B211548F6F767F9002859D01F4B8B
:104680001A78824203D01E4A4FF07E511160187092
:1046900001200DB0BDEC028BBDE8F08F2A464146EB
:1046A000204630F0CBFD8FE64FEA591C09F01F0180
:1046B00058F82C3001228A4023EA02034946284652
:1046C00048F82C30F6F730F97EE600BF4C44002065
:1046D000E0310020CCA20020507D0020607B002033
:1046E000504C0020098500200C8500207C1E0020F5
:1046F0001C460020B0A00020D07C00202DC100204E
:10470000E802002000208AF80001002CB1D0B54B4F
:1047100093F82530012BACD1B34B1B78002BA8D1DB
:10472000172022F0C7FB0B21B048F6F70DF900283F
:10473000A5D1AF4B1868C0F30070A0E7029A1268C9
:10474000920792D5002B92D1CAF80431CAF80831E9
:10475000D9E7029B1B689B077FF5E1AEE60740F1B6
:10476000978523B223F002039BB2A3423B803FF420
:1047700001AFA04B41F20241FF220E2019809A7036
:1047800022F098FB99483C880A21F6F7DDF80028CA
:104790007FF4F7AE984BDB7823B1984BDB79022B93
:1047A0003FF4EFAE24F400639BB2A3423B803FF49E
:1047B000EBAE904B41F20241FF2219800E209A701D
:1047C00022F078FB3C8814F003017FF4E1AE012075
:1047D00008F096FC8A4B42F21072C3F8E020E4E63F
:1047E000122030F005FD9AF8B246002840F0AC8562
:1047F000019B1B78D80700F19884002C40F0E585D8
:10480000804B1E78002E64D17F4B1C68002C3FF437
:1048100024AFDFF824827D4C18F8030C277D414635
:10482000A8F1030530F056FD002800F00D84002F9C
:1048300040F05E8405F10801687930F04BFD0028F6
:1048400041F0E5827249A87A30F044FD002800F07A
:104850000E84022F41F0E3826E49E87B30F03AFD8E
:10486000002841F0D8826C49287D30F033FD0028C3
:1048700000F00E84042F41F0E2826849687E30F037
:1048800029FD002841F0D7826549A87F30F022FD3C
:10489000002800F00E84062F41F0C982614995F886
:1048A000230030F017FD002841F0BD825E4995F8E5
:1048B000280030F00FFD002800F00E84082F41F092
:1048C000C2825A4995F82D0030F004FD002840F0CE
:1048D0000E840024C1E624F480739BB2A3423B8083
:1048E0007FF49DAE524B1B78082B7FF4A6AE3A881E
:1048F00022F040039BB29A423B803FF4A1AE3D4B75
:1049000041F20241FF220E2019809A7022F0D2FA61
:1049100096E6002D40F03F83002F40F04383364A57
:10492000336852699A4280F04783334947F23052E4
:104930000323CA6181F82030022023F007FEFAF732
:104940006BFC2D493268CB69134404228B6181F8DA
:104950002020002D01F09982274A336892699A42FB
:1049600080F06B82294B1878002800F04483314A8C
:10497000136823F0020313603268B8F80230642130
:1049800001FB03231C4900224FF480600B6181F876
:104990002020CA7023F0AAFD174991F8203083E443
:1049A000002F00F03F8230F0BFFC012800F0268489
:1049B000B9F1000F40F01083002D40F03E820E4A06
:1049C000336812699A4251D298F80730022B4DD0C1
:1049D00030F0F0FB0849032240F6B83381F820207C
:1049E000CB61A9E768AF0020C4B800204C44002088
:1049F000B0A00020504C0020607B0020A06300206D
:104A00007C1E0020D07C0020807C00202000002024
:104A10000D44002012440020174400201C440020B4
:104A200021440020264400202B4400203044002054
:104A30001C460020047E00200344002065B3AE4ADB
:104A4000052382F82030002F3FF46FAF30F09AFB3F
:104A5000A94B4FF0030B93F8203025E416F0020524
:104A60003FF41AAC00254FF0020B17E4A24A0123D1
:104A700082F8203098F80730012B00F06E84C1F0E6
:104A8000B780022BF6D130F095FB9B49062240F609
:104A9000B83381F82020CB61002F3FF446AF30F0CF
:104AA00071FB4FF0030B584622F004FAFFF775B97B
:104AB00018219248F5F748FF00287FF479A9904B18
:104AC0001D7B002D7FF474A96FF47A7C07EB0C0238
:104AD00092B240F2E6318A4201F210818949DA88C5
:104AE0004B8A99188F4200F38F849B1A9F42BFF61E
:104AF0006FA9DF1B642505FB07F5A3F57A7395FB0A
:104B0000F3F3DDB2FFF764B900217C48F5F71CFF31
:104B100000287FF428A9FAF77FFB7B4B1B78022B38
:104B20007FF426A9774A7949D37B527C0091013BD7
:104B300031F913301AB1C3F53B6308331BB2A3F547
:104B40007A7307EE903A9FED727A724ADFF8E0A12D
:104B5000F8EEE77A67EE877AFDEEE77A17EE903A9D
:104B600083F30A031380FFF70DB9DFF8C8916A4E8B
:104B700009F1FF3409F196054FF00108A3464946B3
:104B800019F8010C30F0A6FB10B3B9F80540FCB9D8
:104B900099F8040099F8023000EB40010AEB81011A
:104BA000013BD1F8602603EB4303334493420FD01B
:104BB0009AF88C26C1F8603608FA00F022EA000064
:104BC00099F80330C1F864468AF88C0681F85C369F
:104BD00009F10A094D45D2D1504A514B51491B7830
:104BE000096803935C46D2F800B04F4D04913B46F0
:104BF0004FF0FF395F460026A0469B4669680029B2
:104C00006BD00C78002C68D0AA68BA1A002A0EDB88
:104C10009AF88C2607F5FA730120B040AB60434B3D
:104C200022EA00024FF0FF308AF88C261860039BBE
:104C3000002B52D02A7848780432D2B200283ED1D4
:104C40003048009B408A33F912C09AF88C2600F154
:104C5000C80EF44540F35D8242FA06F08A78C10737
:104C60003BD4002A0CBF01200220059222F03AFA20
:104C7000611E059A1F2900F2B387DFE811F04F0487
:104C80001F041606F9030206E505C805AB059105E4
:104C90008E047504B107F9030C04E505C805AB05DE
:104CA000BC045D05430527050B05D604B1074F0479
:104CB00062041F043704B1070B05F10477050128CE
:104CC00000F05282B9F1FF3F40F088829AF88C16CA
:104CD0000122B2400A438AF88C260136042E05F1DF
:104CE0000C058BD1444604F19609DFF84C80CDF8D1
:104CF0000CB0009F25E000BF607B00204C440020EA
:104D00001CC0002068AF0020AA3D00208ABA002005
:104D1000AAF1823FD03D0020409404084085002045
:104D2000454E002038800020E8310020F0020020AD
:104D30008C2B0020894A00201E3200200A344C456A
:104D40005BD0227938F9021F0432D2B237F91250FF
:104D5000A942F3D0E688002EF0D0E278AB4B02F106
:104D6000FF3B0BEB4B01194491F825130029E5D1CA
:104D7000611C2078009230F0ADFA009A0028DDD056
:104D8000049BA8F800502189DAF89006002B00F067
:104D90005F82002800F05C82A5F2DC559C4B01FB91
:104DA00005F583FB0531ED17C5EB61110E44BBF131
:104DB0001F0F00F24D82DFE81BF0D905B705A205F1
:104DC00032029305FC06E506CE06BB06A80695064C
:104DD0004B0232029006FC06E506CE067C0668060B
:104DE000540644062D0618064B02D9051406B705CD
:104DF0000D064B022D06F8050A04039FFFF782BB40
:104E00001E2030F0F5F900283FF477AB1E218148D1
:104E1000F5F79AFD00283FF470AB142022F04AF811
:104E2000FFF76BBB4FF48060B9F1000F01F03880E1
:104E300023F074FB784A00231361BBF1000F3EF4AA
:104E4000ACAF30E6DFF8FCA104F002FFDAF8403640
:104E5000724AC31A93427FF7FFA9714A714B0092BD
:104E600000221A80FEF78EBF6F4AB2F90030002B85
:104E7000B8BF5B42B3F5E17FBFF6C4ABB2F9023015
:104E8000002BB8BF5B42B3F5E17FBFF6BBAB674B0E
:104E900093ED057AD3ED077AD3ED096A93ED030A12
:104EA00077EEA67A30EE070AF7EE000AB0EE007A47
:104EB000E7EEC70A30EE000AF5F7D6FBBEEE008A31
:104EC00020EE088A9FED5A0A38EE000AFDEEC07AFD
:104ED00017EE903A2033402B40F2C0829FED550AE6
:104EE000554CDFED547A84ED010ABDEEC87AC4ED6D
:104EF000027A17EE103A2033402BC4ED037A00F209
:104F00002687B0EE480AF5F73DFB0A2084ED040A37
:104F100021F0D0FFFFF776BB24F040039BB2A34201
:104F20003B803FF468AB454B41F20241FF220E202B
:104F300019809A7021F0BEFFFFF75DBB24F00403D7
:104F40009BB2A3423B803FF44CAB3C4B41F202414D
:104F5000FF2219800E209A7021F0ACFF3C88FFF7E9
:104F600040BB44F40063A3423B807FF422ACFFF7D4
:104F70000BBB9AF84B36002B3FF4FFA9019B1B7823
:104F800013F001037FF4F9A901228AF84B368AF85D
:104F90004C26FFF7F2B9204A052382F82030002F73
:104FA0003FF4BDAC30F0EEF81B4A336852699A42C8
:104FB0004FF0030BFFF4B9AC214B1B78002B7FF4AF
:104FC000B4AC002F3FF4B1AC002D3FF436AF124B20
:104FD00093F82030FFF768B998F80630012B7FF47A
:104FE000EBAC30F0E7F80C4903224FF47A7381F808
:104FF0002020CB61A0E42FF05BFB00283FF4B7AC8E
:10500000BBF1000F3EF4C9AE4DE500BF1C91040892
:10501000D34D62104C440020607B002060E31600FA
:105020008ABA0020D03D0020F47B002074260020A6
:10503000DB0FC93F0000000020000020504C002082
:10504000466400208C2B002008F10501687930F0BF
:1050500041F900283FF4F6AB012F40F0D88605F166
:105060000D01A87A30F036F9002840F0D886C04902
:10507000E87B30F02FF900283FF4F5AB032F40F028
:10508000CA86BC49287D30F025F9002840F0D78633
:10509000B949687E30F01EF900283FF4F5AB052FC2
:1050A00040F0C986B549A87F30F014F9002840F0D7
:1050B000BE86B34995F8230030F00CF900283FF480
:1050C000F5AB072F40F0AF86AE4995F8280030F0D9
:1050D00001F9002840F0B786AB4995F82D0030F073
:1050E000F9F800283FF4F5AB092F3FF4F2AB09269D
:1050F000334603EB83031D44A44B6978AA782675D5
:1051000019705A70FFF7E5BB01238AF81031FEF7DA
:1051100061BFC838844580F272853241D2078978F0
:105120003FF5DBAD4A4201209FE5002C7FF492AAB7
:10513000974C94F8DA30002B40F0878194F8B63120
:10514000002B40F0788194F89232002B40F0698176
:1051500020F0A0FD01238AF8B236FFF776BA8D4A17
:1051600001239370FFF783B8009B91F802C033F9D5
:1051700012200C2C00F0A485B2F5617FC0F23C81B6
:1051800040F633099145A8BF9146182CA9F56179DD
:105190004FF4966292FBFCFC99FBFCF95FFA89F9EB
:1051A0001CD14A46C82AA8BFC822D0B2DAF8903625
:1051B00093F81CE0864511D0B2EB0E0276491877C1
:1051C00048BF0732D21089780132D2B2002940F0AC
:1051D000488112B1104621F085FF69680A780C2ACF
:1051E0003FF474AD6D4B1C606D4BC3F800906DE5E2
:1051F000022023F093F93C88FFF7BCB93268B8F875
:105200000230642101FB0323624A1361B9F1000FEC
:105210003FF4D2ABE0E6002D7FF4AEAB2AE45E4B68
:1052200086F308069978049BF5B29D7229B1314640
:105230000D20009230F0ACF8009A0D2A06D0564BA3
:105240009A78049B5D72002A40F03486DAF8900662
:105250002DF0E0F972E500215248F5F775FB0028C2
:1052600065D000238AF84936FDF70EFFFEF74ABEE7
:1052700044F04003A3423B807FF455AEFFF7BBB937
:1052800044F00403A3423B807FF45FAEFFF7A9B96B
:1052900044F00103A3423B803FF463AA424B41F236
:1052A0000241FF2219809A700E2021F003FE3C88F3
:1052B00023B2FFF757BA3D483D490068BAF9464660
:1052C000C56981FB05018911ED17681A00F5FF40DA
:1052D0007F30844240F39E84364909780029BAD051
:1052E0005F2A00F019856F2B7EF409AEB4F5FA7FC2
:1052F000FFF63CA89AF84836002B7FF437A8019AAD
:105300001278012112EA01048AF8481640F0238538
:10531000FDF7BAFE284B1B68002B3FF427A8274B4C
:10532000274A8AF848461B680292FFF723B8019B78
:10533000214A1B78CAF83801DC07106000F1A98403
:105340001E4B1B68FEF7E4BD12211648F5F7FCFA68
:10535000C0B3002C7FF479A9EAE62FF02BFF0D49AA
:10536000032240F6B83381F82020CB61FFF7E4BA7E
:1053700012440020174400201C4400202144002037
:10538000264400202B44002030440020547B002081
:1053900044960020607B0020347E0020346500208D
:1053A000F00200204C440020504C002020840020BB
:1053B000D34D6210200000204C7E0020B0A00020C1
:1053C0009C720020002C3FF440A920F063FC21F0E7
:1053D000E3FC00238AF8B236FFF737B90021C5484D
:1053E000F5F7B2FA00287EF4AFAD32238AF84A0608
:1053F000AAF84E36FEF7A8BD182C40F0B4844FF042
:10540000000948464A46D1E6F91A891AC3F5FA63F3
:1054100064259B1A05FB01F595FBF3F5EDB2FEF74C
:10542000D7BCD4F8B80121F00AFBDC220021B24835
:1054300032F026FA8CE6D4F8DC0021F000FBDC2206
:105440000021AE4832F01CFA7DE6206821F0F7FA20
:10545000DC220021204632F013FA6FE6F5F792F8CD
:105460003EE54946182005922FF092FF059AB0E6D6
:10547000049BA34993F80A908978914489F3080919
:1054800083F80A9029B149460D2005922FF080FF3C
:10549000059A0D2C0CD0049B994993F809908978B2
:1054A000914489F3080983F80990002940F02A857E
:1054B000DAF890062DF0AEF869688FE6049B904903
:1054C00093F8069089789144B9F1640FA8BF4FF022
:1054D000640929EAE97983F8069029B149461B2035
:1054E00005922FF055FF059A1B2CE1D0049B8449AF
:1054F00093F8079089789144B9F1640FA8BF4FF0F1
:10550000640929EAE97983F807900029D0D01C20A2
:1055100049462FF03DFFDAF89006CBE7049B784927
:1055200093F803908978914489F3080983F80390EC
:1055300029B14946192005922FF02AFF059A192C06
:10554000B6D0049B6E4993F804908978914489F30E
:10555000080983F804900029AAD01A2049462FF0A0
:1055600017FFDAF89006A5E7DAF89006644B90F892
:10557000169099789144B9F1C80FA8BF4FF0C809A7
:1055800029EAE97980F81690002993D00B20494642
:105590002FF0FEFEDAF890068CE7DAF89006584B0A
:1055A00090F8159099789144B9F1C80FA8BF4FF0C1
:1055B000C80929EAE97980F8159000293FF47AAF03
:1055C0000A2049462FF0E4FEDAF8900672E74C4BC9
:1055D000B6F5FA6F31469A78A8BF4FF4FA6121EA1E
:1055E000E1710183002A3FF433AE20202FF0D0FE7A
:1055F000DAF890062CE6DAF8900690F80890404B1E
:105600009144B9F1C80FA8BF4FF0C809997829EAA9
:10561000E97980F8089000293FF44CAF1220494600
:105620002FF0B6FEDAF8900644E7DAF89006344B2D
:1056300090F8479099789144B9F1640FA8BF4FF062
:105640006409B9F1010FB8BF4FF0010980F8479024
:1056500000293FF42FAF494617202FF099FE27E786
:10566000DAF89006B0F80C90254B9144B9F5FA6F32
:10567000A8BF4FF4FA69997829EAE979A0F80C9063
:1056800000293FF417AF1F2049462FF081FEDAF8BA
:1056900090060FE7DAF89006194BB0F81290997857
:1056A0009144B9F5FA6FA8BF4FF4FA6929EAE9798C
:1056B000A0F8129039B11E20494605922FF068FEDD
:1056C000DAF89006059A1E2CCCD1F3E6049B0C491F
:1056D00093F805908978914489F3080983F8059037
:1056E00000293FF4E5AE152049462FF051FEDAF8C7
:1056F0009006DFE64C440020FC9700202097002015
:10570000347E0020DAF8900690F80A90C04B91445D
:10571000B9F1C80FA8BF4FF0C809997829EAE9790B
:1057200080F80A9000293FF4C5AE142049462FF0B6
:105730002FFEDAF89006BDE6DAF8900690F80990A8
:10574000B34B9144B9F1C80FA8BF4FF0C80999787D
:1057500029EAE97980F8099000293FF4ABAE1320DB
:1057600049462FF015FEDAF89006A3E6DAF890061F
:10577000A74BB0F8189099789144B9F5FA6FA8BF83
:105780004FF4FA6929EAE979A0F8189000293FF462
:1057900091AE202049462FF0FBFDDAF8900689E60D
:1057A000DAF890069A4B90F8149099789144B9F1F0
:1057B000C80FA8BF4FF0C80929EAE97980F814900A
:1057C00000293FF477AE092049462FF0E1FDDAF8D1
:1057D00090066FE6DAF890068D4B90F81090997865
:1057E0009144B9F1C80FA8BF4FF0C80929EAE97977
:1057F00080F8109039B11120494605922FF0C8FD6C
:10580000DAF89006059A112C7FF47EAF52E6DAF8AA
:1058100090067F4B90F80F9099789144B9F1C80F9A
:10582000A8BF4FF0C80929EAE97980F80F9039B18B
:105830001020494605922FF0ABFDDAF89006059A44
:10584000102C7FF47BAF35E6DAF89006704B90F8B9
:105850000E9099789144B9F1C80FA8BF4FF0C809CC
:1058600029EAE97980F80E9039B10F20494605926E
:105870002FF08EFDDAF89006059A0F2C7FF4BDAE5E
:1058800018E6049B624993F80B908978914489F358
:10589000080983F80B9000293FF40AAE0520494619
:1058A0002FF076FDDAF8900604E6049B93F8019059
:1058B0009144B9F1640FA8BF4FF0640929EAE9796E
:1058C00083F801902FF08CFD514B9A78002A3FF419
:1058D000EFAD032049462FF05BFDDAF89006E9E5CD
:1058E0004B4B9A78049B86F30801D972002A3FF447
:1058F000AFAC05202FF04CFDDAF89006A8E4642E3A
:10590000049BA8BF642626EAE6765E702FF068FD49
:105910003F4B9A78002A3FF499AC032031462FF090
:1059200037FDDAF8900693E4642E394BA8BF64265D
:1059300026EAE6769978049BF5B29D7129B1314645
:105940001B2000922FF024FD009A1B2A3FF47EAC0E
:105950002F4B9A78049BDD71002A3FF477AC1C2012
:1059600031462FF015FDDAF8900671E4284B86F3E6
:1059700008069978049BF5B2DD7029B131461920EB
:1059800000922FF005FD009A192A3FF45FAC204BDE
:105990009A78049B1D71002A3FF458AC1A203146B6
:1059A0002FF0F6FCDAF8900652E4B6F5FA6FA8BFCD
:1059B0004FF4FA6626EAE676B5B2154B85819A78F9
:1059C000002A3FF445AC1F2031462FF0E1FCDAF805
:1059D00090063DE4642EA8BF642626EAE676F5B27A
:1059E000B6E786F30806F5B2D1E7642E084B3146D8
:1059F000A8BF642101299A78B8BF012180F8471017
:105A0000002A3FF425AC17202FF0C2FC1EE400BF93
:105A1000347E0020B6F5FA6FBA4BA8BF4FF4FA6691
:105A200026EAE6769978B5B2458239B11E2031462C
:105A300000922FF0ADFCDAF89006009A1E2ABCD135
:105A400006E4B04B9A78049B86F308015971002A4A
:105A50003FF4FEAB15202FF09BFCDAF89006FFF721
:105A6000F7BBC82EA8BFC82626EAE676F5B2A54B36
:105A700085729A78002A3FF4EBAB142031462FF060
:105A800087FCDAF89006FFF7E3BBC82EA8BFC8264C
:105A900026EAE676F5B29B4B45729A78002A3FF4E7
:105AA000D7AB132031462FF073FCDAF89006FFF7DE
:105AB000CFBBC82EA8BFC82626EAE676F5B2914B22
:105AC00005729A78002A3FF4C3AB122031462FF0BA
:105AD0005FFCDAF89006FFF7BBBB86F30806F5B269
:105AE000FFF7ADBB874BC82E31469A78A8BFC821B7
:105AF00021EAE1718175002A3FF4AAAB0B202FF057
:105B000047FCDAF89006FFF7A3BB7E4BC82E314660
:105B10009A78A8BFC82121EAE1714175002A3FF4B3
:105B200097AB0A202FF034FCDAF89006FFF790BB11
:105B3000744BC82E31469A78A8BFC82121EAE1717A
:105B40000175002A3FF484AB09202FF021FCDAF81C
:105B50009006FFF77DBBC82E6A4BA8BFC82626EA71
:105B6000E6769978F5B2057439B111203146009284
:105B70002FF00EFCDAF89006009A112A7FF477AF26
:105B8000FFF766BBC82E5F4BA8BFC82626EAE6769D
:105B90009978F5B2C57339B11020314600922FF0D3
:105BA000F7FBDAF89006009A102A7FF474AFFFF73B
:105BB0004FBBC82E534BA8BFC82626EAE676997875
:105BC000F5B2857339B10F20314600922FF0E0FB1A
:105BD000DAF89006009A0F2A7FF471AFFFF738BB0E
:105BE000DAF890062CF016FD4FF0FF39FFF76EB88B
:105BF0002FF0E0FA444B93F82030FEF755BB01211B
:105C0000B14022EA010207F5FA718AF88C26A960F0
:105C1000FFF763B8491B0C4424B2AAF84646FFF7C5
:105C20005BBB3A4A116811F020017EF479A99AF819
:105C300045260120572A8AF8480600F008815E07A9
:105C400002D55A2A00F09E815D2A00F094815E2AD6
:105C500000F08A815B2A00F07881562A00F0A58145
:105C6000972A3EF47FABA72A00F054823B889D0719
:105C700040F03682A2F1B703072B00F2A581DFE8DE
:105C800013F0BB02A301A301A301B902A301B70250
:105C9000AE021F4B1B78002B3EF468AB1A4BDB782F
:105CA000002B7EF463AB9AF849360133DBB2032B49
:105CB0008AF849367EF65AABF9F7AEFAFEF722B902
:105CC00014480379002B5FD04FF0C80CB2F5617F08
:105CD0004DDA4FF000094A46407890423FF47EAAE0
:105CE00010460592FEF720F8064B059A9978002990
:105CF00040F0DA800132D2B2FFF76BBA6425FEF7CA
:105D000067B800BF347E0020607B0020047E002046
:105D1000454E0020E8980020B4F5FA7FFEF626AB49
:105D20009AF84836002B7EF421AB019AC8491278C4
:105D30000B60012312EA03048AF8483629D0F9F7E8
:105D40006BFAC44B0293C44B1B68FEF713BBB0EE57
:105D5000670AFFF7DAB8CAF83831BF4BBD4A1B688B
:105D60000292FEF707BB4FF00009FFF737BA40F683
:105D700033099145A8BF9146A9F5617999FBFCF9D2
:105D80005FFA89F94A46A7E74FF4966999FBFCFC4C
:105D90009CE70F2021F08EF8B049BAF846360A6821
:105DA0008AF84846FA3B22F02002AAF84636AA4B67
:105DB0000A60A84A1B680292FEF7DCBA03932EF031
:105DC0001FFE039B00287EF42CA9B8F1000F7EF47F
:105DD00028A9029A2AB1DAF840319B1A2344CAF85A
:105DE00040310023CAF83C319D4B9FED9E7A5B7891
:105DF000202F07EE903A00F08D80F8EEE77A67EEFC
:105E0000877AFCEEE77A17EE905AFEF7CCB90126B6
:105E10003346FFF76EB903263346FFF76AB9022609
:105E20003346FFF766B907263346FFF762B9062601
:105E30003346FFF75EB905263346FFF75AB9042605
:105E40003346FFF756B908263346FFF752B986495D
:105E5000864A8C8B8649106842F2107202FB04F26B
:105E6000B2FBF0F2C1F8B020190603D517F0F4F92F
:105E7000794B1B68774A0292126852077EF57AAA1C
:105E80000A22AAF8BE20FEF775BA7A493268CB69B1
:105E900013448B61BBF1000F3DF47FAFFEF703BEEF
:105EA00022F024FBFEF7C6BF49460C202FF070FA03
:105EB000059A1FE70E2031462FF06AFADAF89006AD
:105EC000FFF7C6B9B8F1000F3EF493A99AF844362B
:105ED000002B3DF4C3AF20F0D5FF00238AF84436F1
:105EE000FDF7BCBFACEB0E0191427EF7C6A8881A45
:105EF0006422A1F57A7102FB00F292FBF1F2D2B2B8
:105F0000FEF7B9B80E2049462FF042FADAF89006AB
:105F1000FFF7D0BA584ADAF840315849F8EEE77A34
:105F2000A2FB0323019A67EE877A12789B09FCEEA5
:105F3000E77ACB8002F00102002317EE905A8B80A3
:105F4000002A3DF487AFFEF70ABA4D4A4D494E4B41
:105F50001160022001221A703E4B029321F0C2F818
:105F60003D4B1B68FEF706BA454A48491160464B4F
:105F700002220320EFE7424A45491160424B0022CA
:105F80000120E8E79AF84B269AF84A36A2B983F03E
:105F900001038AF84A366BB90C2020F08BFF2D4B99
:105FA00002932D4B1B68FEF7E5B908F0B7FB9AF892
:105FB000452655E60B20F0E7264B8AF84B168AF863
:105FC0004C060293FDF7B1BF792A00F083807A2A4C
:105FD00037D09E2A03D10021012031F0CFFB9AF85F
:105FE00045369D2B03D10021FF2031F0C7FB9AF8E5
:105FF0004536AE2B03D10121002031F0BFFB9AF8CA
:106000004536AD2B03D1FF21002031F0B7FB9AF8C4
:106010004536EF2B5BD0FD2B56D0FB2B51D0FE2B02
:106020004CD0F72B38D07B2B7EF4A0A94FF4FA612B
:106030000220FDF703FE074B0293074B1B68FEF798
:1060400099B9144A137A43F001031372CFE700BFE2
:106050004C7E00209C720020B0A00020047E002016
:10606000984400200024744980A00020A0A00020B3
:10607000F8990020607B0020D34D6210F884002046
:10608000348000201C5E0020E89800207C5E002008
:10609000BC5D0020A462002000210420FDF7CEFD9D
:1060A000BAF84626554B56491B680291963AAAF80B
:1060B000462600228AF84826FEF75CB90021032014
:1060C000ECE700210220E9E700210120E6E70021BA
:1060D0000846E3E74B4A137A23F0010313727EE785
:1060E0000021A2F1B7030A91072B3FF66DAF01A182
:1060F00051F823F075610108C95F0108C95F010803
:10610000C95F01086D610108C95F01086361010889
:10611000276101083C49394B0A781B6842F00402A8
:106120000A70FDF7FDBE0223ADF82830374BBDF8ED
:1061300028409989DA89BDF82A00214402449981CE
:10614000DA8108F0EBFABAF846262D492B4B02917A
:10615000FA3A00211B68AAF846268AF84816FEF784
:1061600009B94FF6FE73ADF82830DFE70223ADF82A
:106170002A30DBE74FF6FE73ADF82A30D6E7F9F7A1
:106180004BF88AF84486FDF769BE9AF844362C44E9
:10619000CAF83441002B3DF461AE9CE6ACEB090C2F
:1061A0006245BDF6A4AFACEB02026421ACF57A7C8B
:1061B00001FB02F292FBFCF2D2B2FDF796BFACEB10
:1061C0000E0191427DF775AF881A6422A1F57A71AC
:1061D00002FB00F292FBF1F2D2B2FDF768BF02209F
:1061E000FDF7A2FD064B0293044B1B68FEF7C2B8F5
:1061F0000320F5E70020F3E70120F1E7B0A000203D
:106200009C720020A4620020247E002034410020E3
:106210001F4B187810B31F4A138903B31E4A9FED12
:106220001F6AD2ED026A07EE903AF8EEE66AF8EEDF
:10623000677A07EE103A77EEE66AB8EEC77A66EE4E
:10624000866AC6EE877AFDEEE77A17EE900A642832
:10625000A8BF642020EAE070C0B27047704710B455
:106260000F4B54781B88117804FB1032091B6423F0
:1062700000FB01F003FB02F3B3FBF0F06428A8BFBE
:10628000642020EAE070C0B25DF8044B704700BFA4
:106290008A7B00209C7B0020AC7B00200000C84251
:1062A000847B00202DE9F04F83B000254348009502
:1062B0000090009B424ADFF8248192F821C092F8B6
:1062C0002D70D6693C330093009B1B6801950190AB
:1062D000019840300190019D0FFA8CF0D2E9091429
:1062E000D5F800E036F8105026F8103038B211FA20
:1062F0008EF134F8106024F810E03248B8F80090BD
:10630000B0F800809069304C10FA83F3A1EB060ED0
:10631000581BB4F800A092F8205092F82C40B0FB23
:10632000F5F6BEFBF4F340F6E4411FFA86FB9BB2A0
:1063300001FB03F301FB0BF191FBFAF189B293FB33
:10634000F1F347F22471A3EB090308FB03131F4980
:10635000C2F824E00CF1010C81FB03E1906107F12C
:10636000010E1B481B4FDFF87880DB17C3EBA1132E
:106370009CFBF5F105FB11C59EFBF4F104FB11E458
:1063800082F8215082F82D40A7F8B46602781F2ABF
:1063900008BF114A1BB208BF1380A8F80030074B92
:1063A0006FF004021A609A68012142F480029A6038
:1063B00087F8B61603B0BDE8F08F00BF002001409B
:1063C000200000203E8700203A870020D34D621035
:1063D000F58400208C2B0020F88400203C870020CE
:1063E0003065002008B5F7F7CDFD00B108BDBDE868
:1063F000084057E7064A074BB2F8B4261B8840F618
:10640000E44000FB02F090FBF3F080B2704700BF65
:106410008C2B00203A870020F8B50146FFF7EAFFF1
:106420000F4A104BB2F90260B2F900701D780E4CA1
:1064300000FB01F0020B42F2107303FB02F393FB2B
:10644000F7F3334484FB0310222D4FEAE373C3EBCD
:10645000A00000D0F8BD054B1A805880F8BD00BFE1
:106460002E5D0020F584002067666666F8840020B3
:10647000704B1B78002B3AD070B56F4B6F4D9B79EA
:10648000D5F8B846C5F8B806013B041B032B00F24B
:106490008780DFE803F04702312B2EF045FF684B81
:1064A00068491A784B8802F0010200287ED06648BD
:1064B000C5F8B830D0ED037A002A40F08F8003FB96
:1064C00004F007EE900ADFED616A614AB8EEE77A00
:1064D000D5ED2D7AE7EE267AC2E90033BDEEE77AF4
:1064E000C5ED2D7A85ED2C7A82ED027A70BD584A81
:1064F000C2E9003393607047564B1B681B01F5D50A
:10650000FF201DF077FE18B103780A2B74D9002004
:1065100003464F4AC5F8BC06C5F8C036C2E9003389
:10652000906070BD4C4A4D4BD27933F81260B6B2D0
:106530003046FFF771FF07EE906AC5F88800B8EEA5
:10654000670A4748F1F70CFFBCEEC00A10EE103A9C
:1065500098B2FFF761FFD5F88810D5ED207ADFED0E
:106560003B6A3B4B3F4AC5F8840001FB04F407EE4D
:10657000104AB8EEC77A1860E7EE267A10785960AC
:106580002228BDEEE77AC5ED207A17EE102A83EDBA
:10659000027A85ED1F7AA9D1334B9980DA8070BDDC
:1065A0002B4B0022C3E900229A6070BD294E366849
:1065B000F6067FF57CAFC5F8B830002A3FF47FAF10
:1065C000B1F90010294A00FB01F082FB0012C0174C
:1065D000C0EBA2100344C5F8B83070E7FDEEE77ACF
:1065E000234E17EE900AA0F57A7000FB00F2A6FB8E
:1065F000026200EB1210E3E71E4A1F4B51881A6833
:10660000D0ED027ADFED1D6A1D4C436802FB01F2FA
:1066100007EE102AF8EEE77AB8EE477AA4FB0121DC
:10662000E7EE267A03EBD103FDEEE77A17EE900A48
:106630006FE700BF8A7B00209C7B00208C2B002012
:106640005E7B0020365D00208C7B00202FE33E31F6
:10665000AC7B0020B0A000201C87002040870020D9
:10666000182C0020F5840020F8840020D34D6210FF
:106670001F85EB515C7D0020408500207D219534F5
:10668000CDCCCCCC2DE9F047444B5B79012B30D0FD
:10669000022B0ED0424B00221A60424B1B78022B79
:1066A00005D13F4A404B5188128819805A80BDE875
:1066B000F0873E4B1B681B01EFD5FF201DF09AFDB4
:1066C000002868D003780A2B57D99FED390A002398
:1066D000384C04F12C006385F1F742FEBCEEC00A91
:1066E00010EE103A9BB223852D4A618D51801380A4
:1066F000D3E7314A314B92782E4C33F81270304E3A
:10670000304D1FFA87FA07EE90AA04F15400B8EE54
:10671000670AF1F725FEFFF76DFEBCEEC00A377879
:106720007378B67810EE102A07FB00F190B201FBE7
:1067300000F1A5FB012144F6FB78C3EB033908EB1C
:106740005111B1FBF9F1B1FBF6F189B2A4F8501087
:10675000FFF750FE07FB0AF707FB00F3A5FB032337
:106760000F4A08EB5313B3FBF9F3B3FBF6F39BB2F9
:10677000A4F85230538011808FE7B0F902201249FB
:10678000D31781FB0212C3EBA2039BB207EE903A30
:10679000B8EE670A9CE7074C238DA5E79C7B002099
:1067A000847B0020F5840020F8840020B0A0002025
:1067B000000000008C2B00201C8700204087002058
:1067C000295D00201F85EB5167666666174A3423F2
:1067D00003FB002009B1C368B3B970B5144DD5F8F7
:1067E000C446002C0FDDD5F8C83698420ED005F50A
:1067F000D9663346002203E053F8041F884208D0CC
:1068000001329442F8D170BD1FF0D0BF002205F5CF
:10681000D9669000011DA21A920031443044013C17
:1068200031F015F8C5F8C44670BD00BF7C1E0020CD
:106830008C2B00202DE9F04F2DED088B664C9BB082
:10684000F6F71AF806F00CFBF8F7C2FA6278BE2ADF
:1068500055D0F4F751FF07F097FE01F099FB02F0D5
:106860000DFF054601F04AFC45B12378AB2B05D15D
:1068700006225A495A48F4F7E3FB08B108F0B2F986
:10688000584C594D94F80C3BAA78584E43F00103EC
:1068900084F80C3B564B1A70564B1B68336027F03C
:1068A00051FE0121022006F02BFC07F0B1FB3368FA
:1068B00013F0080FB2460BD04F4B1A7A0A2A07D8AA
:1068C0000123934040F20342134201D027F0BCFC65
:1068D0006B79022B18D8494903EB43025200881800
:1068E0008A5A4188B2FBF1F1454A4A434549096851
:1068F0008A4209D0444A136072B630F02DFF07F087
:106900000FFE0028ABD1A4E7642003F051FA01F098
:106910006FFD3E483E4B3F4F002200F11308115CD3
:1069200008EB0206002507EB010916F801EFBEF19E
:10693000000F05D099F80CC0F44508BF83F868C073
:1069400096F804E0BEF1000F05D017F801C0F44539
:1069500008BF83F869C00135042DE6D1B3F868504B
:106960003DB104EB810185185D66C1F8103B03F56C
:10697000F6732432482AD2D1282200212648DAF898
:106980000050DFF8949030F07BFF224ADFF88CC093
:10699000937A069392F80BB0937D92F81780079341
:1069A00005F040070020052305924FF0FF0E1CF96B
:1069B000011F00EB09060729B17131DC059A525C11
:1069C000002A37D1059A1144097B99BB013B86F80F
:1069D00006E0DBB22EE000BF00400008B9CE04089C
:1069E000EF9800208C2B0020E8980020B0A0002019
:1069F000F5840020BC62002068AF0020A094040849
:106A000040420F00B0A20020D8C20020B494040875
:106A1000C032002098AF002098B80020FB940408F2
:106A20001E2940F05584002FD0D0069A12B9079A3B
:106A3000002ACBD008302828B9D184F8283BB74B9E
:106A4000B74E1A78B74BB8481A70B378B749B84AF6
:106A5000053B042B05F4805500F2508400230360AD
:106A6000F389DFEDB47A9FEDB47A06EE903AF8EE52
:106A7000E66A66EEA77A002D00F03A8437EE877A50
:106A800081ED007A9FEDAD7AAD4B136077EE877A9A
:106A9000AC4BAD4AC3ED007AAC4B1A60AC4B9B8A51
:106AA000C3F5FA6307EE903AAA4BF8EEE77AC3ED26
:106AB000007A2EF0C5F9DAF80030B08AD90444BF64
:106AC000A54B9888B378042BA44B08BF00201978F5
:106AD00026F048FD94F80C3B43F0040384F80C3B8B
:106AE000DAF80030DA0740F1498426F0D1FCB4F836
:106AF0002E5B9B4B94F82A0B1D80002D40F04584A3
:106B000001F0F6FE974A9849106094F82B2B00325A
:106B100018BF01220A7058B194F82C3BC571002BA4
:106B20004FF0250282710CBF0121112106F038FAC5
:106B3000002007F055F98D4B8D4F8E4803F130063C
:106B40004FF0000ED3F804C0BCF1000F47D093F90A
:106B5000002093F8089002EB4205120117F8058017
:106B6000C14508BF00EB020907EB050108BF89F822
:106B700004804D7893F80A908978A94504BF00EB0A
:106B8000020989F8055093F80C90894504BF00EB81
:106B9000020989F8061093F80990C14504BF00EB7B
:106BA000020989F8048093F80B80A84504BF00EB24
:106BB000020888F805505D7B8D4204BF8518A971D5
:106BC00081180D795DB14D794DB18D793DB140F8A8
:106BD00002C09A7BCA71DA7B0A7281F80CE010332A
:106BE000B342AFD1644F00254FF03508E85D60B186
:106BF00001F07EFE064640B180F80680C571202176
:106C000006F0CEF9304606F06DFA01350B2DEDD1C8
:106C100094F8440B60B101F06BFE054640B1362399
:106C200083710023C37124F0ADF9284606F05AFAA7
:106C300094F8450B60B101F05BFE054640B1362388
:106C400083710123C37124F09DF9284606F04AFAA6
:106C50000020F6F771FE0120F6F76EFE474F4FF069
:106C60000009474B03EB0902059252680692002A7D
:106C700000F08C8013F90960242202FB06F57819D4
:106C8000002130F0FDFD3F4BDDF8148003EB860B57
:106C900013F8263007939BF80130089304230993D7
:106CA000254498F80800079B984208D1184601F03F
